 navPlugin

 Timestamp is 614c8002 (Thu Sep 23 13:24:18 2021)

 Preferred load address is 10000000

 Start         Length     Name                   Class
 0001:00000000 00000063H .text$di                CODE
 0001:00000070 0000308cH .text$mn                CODE
 0001:000030fc 00000729H .text$x                 CODE
 0001:00003825 00000021H .text$yd                CODE
 0002:00000000 000006f0H .idata$5                DATA
 0002:000006f0 00000004H .CRT$XCA                DATA
 0002:000006f4 0000000cH .CRT$XCU                DATA
 0002:00000700 00000004H .CRT$XCZ                DATA
 0002:00000704 00000004H .CRT$XIA                DATA
 0002:00000708 00000004H .CRT$XIAA               DATA
 0002:0000070c 00000004H .CRT$XIC                DATA
 0002:00000710 00000004H .CRT$XIZ                DATA
 0002:00000718 000015a8H .rdata                  DATA
 0002:00001cc0 000009a8H .rdata$r                DATA
 0002:00002668 00000004H .rtc$IAA                DATA
 0002:0000266c 00000004H .rtc$IZZ                DATA
 0002:00002670 00000004H .rtc$TAA                DATA
 0002:00002674 00000004H .rtc$TZZ                DATA
 0002:00002678 00000814H .xdata$x                DATA
 0002:00002e90 0000005dH .edata                  DATA
 0002:00002ef0 0000003cH .idata$2                DATA
 0002:00002f2c 00000014H .idata$3                DATA
 0002:00002f40 000006f0H .idata$4                DATA
 0002:00003630 00004618H .idata$6                DATA
 0003:00000000 000000a4H .data                   DATA
 0003:000000a4 00000390H .data$r                 DATA
 0003:00000438 000003a4H .bss                    DATA
 0004:00000000 000000a0H .rsrc$01                DATA
 0004:000000a0 00000608H .rsrc$02                DATA

  Address         Publics by Value              Rva+Base       Lib:Object

 0000:00000000       ___safe_se_handler_table   00000000     <absolute>
 0000:00000000       ___safe_se_handler_count   00000000     <absolute>
 0000:00000000       ___guard_fids_count        00000000     <absolute>
 0000:00000000       ___guard_flags             00000000     <absolute>
 0000:00000000       ___guard_fids_table        00000000     <absolute>
 0000:00000000       ___ImageBase               10000000     <linker-defined>
 0001:00000070       ??0config@@QAE@ABVQString@@@Z 10001070 f   config.obj
 0001:000000c6       ??0navEntry@@QAE@ABVQString@@0ABVQPixmap@@@Z 100010c6 f i config.obj
 0001:00000129       ??1?$QDict@V?$QPtrList@VnavEntry@@@@@@UAE@XZ 10001129 f i config.obj
 0001:0000015c       ??1?$QPtrList@VnavEntry@@@@UAE@XZ 1000115c f i config.obj
 0001:0000018f       ??1config@@UAE@XZ          1000118f f   config.obj
 0001:000001c5       ??1navEntry@@QAE@XZ        100011c5 f i config.obj
 0001:00000205       ??_E?$QDict@V?$QPtrList@VnavEntry@@@@@@UAEPAXI@Z 10001205 f i config.obj
 0001:00000205       ??_G?$QDict@V?$QPtrList@VnavEntry@@@@@@UAEPAXI@Z 10001205 f i config.obj
 0001:00000224       ??_G?$QPtrList@VnavEntry@@@@UAEPAXI@Z 10001224 f i config.obj
 0001:00000224       ??_E?$QPtrList@VnavEntry@@@@UAEPAXI@Z 10001224 f i config.obj
 0001:00000243       ??_Econfig@@UAEPAXI@Z      10001243 f i config.obj
 0001:00000243       ??_Gconfig@@UAEPAXI@Z      10001243 f i config.obj
 0001:00000262       ?clear@?$QDict@V?$QPtrList@VnavEntry@@@@@@UAEXXZ 10001262 f i config.obj
 0001:00000268       ?clear@?$QPtrList@VQPopupMenu@@@@UAEXXZ 10001268 f i navPlugin.obj
 0001:00000268       ?clear@?$QPtrList@VnavEntry@@@@UAEXXZ 10001268 f i config.obj
 0001:0000026e       ?count@?$QDict@V?$QPtrList@VnavEntry@@@@@@UBEIXZ 1000126e f i config.obj
 0001:00000272       ?count@?$QPtrList@VnavEntry@@@@UBEIXZ 10001272 f i config.obj
 0001:00000272       ?count@?$QPtrList@VQPopupMenu@@@@UBEIXZ 10001272 f i navPlugin.obj
 0001:00000276       ?deleteItem@?$QDict@V?$QPtrList@VnavEntry@@@@@@EAEXPAX@Z 10001276 f i config.obj
 0001:00000291       ?deleteItem@?$QPtrList@VnavEntry@@@@EAEXPAX@Z 10001291 f i config.obj
 0001:000002b5       ?getKeys@config@@QAE?AVQStringList@@XZ 100012b5 f   config.obj
 0001:000004cf       ?getNavEntry@config@@QAE?AV?$QPtrList@VnavEntry@@@@ABVQString@@AAV3@@Z 100014cf f   config.obj
 0001:00000a5f       ??0navIconViewItem@@QAE@PAVQIconView@@ABVQString@@1@Z 10001a5f f   navIconViewItem.obj
 0001:00000aa9       ??0navIconViewItem@@QAE@PAVQIconView@@ABVQString@@1ABVQPixmap@@@Z 10001aa9 f   navIconViewItem.obj
 0001:00000af6       ??1navIconViewItem@@UAE@XZ 10001af6 f   navIconViewItem.obj
 0001:00000b2c       ??_GnavIconViewItem@@UAEPAXI@Z 10001b2c f i navIconViewItem.obj
 0001:00000b2c       ??_EnavIconViewItem@@UAEPAXI@Z 10001b2c f i navIconViewItem.obj
 0001:00000b4b       ??0config_plugin_base@@QAE@ABVQString@@00@Z 10001b4b f i navPlugin.obj
 0001:00000bd8       ??0navPlugin@@QAE@ABVQString@@00@Z 10001bd8 f   navPlugin.obj
 0001:00000dde       ??1?$QPtrList@VQPopupMenu@@@@UAE@XZ 10001dde f i navPlugin.obj
 0001:00000e11       ??1QDockWindowList@@UAE@XZ 10001e11 f i navPlugin.obj
 0001:00000e5a       ??1QPopupMenuList@@UAE@XZ  10001e5a f i navPlugin.obj
 0001:00000e8c       ??1config_plugin_base@@UAE@XZ 10001e8c f i navPlugin.obj
 0001:00000ee6       ??1navPlugin@@UAE@XZ       10001ee6 f   navPlugin.obj
 0001:00000ef8       ??_Econfig_plugin_base@@WCI@AEPAXI@Z 10001ef8 f i navPlugin.obj
 0001:00000f00       ??_EnavPlugin@@WCI@AEPAXI@Z 10001f00 f i navPlugin.obj
 0001:00000f08       ??_E?$QPtrList@VQPopupMenu@@@@UAEPAXI@Z 10001f08 f i navPlugin.obj
 0001:00000f08       ??_G?$QPtrList@VQPopupMenu@@@@UAEPAXI@Z 10001f08 f i navPlugin.obj
 0001:00000f27       ??_GQDockWindowList@@UAEPAXI@Z 10001f27 f i navPlugin.obj
 0001:00000f27       ??_EQDockWindowList@@UAEPAXI@Z 10001f27 f i navPlugin.obj
 0001:00000f46       ??_GQPopupMenuList@@UAEPAXI@Z 10001f46 f i navPlugin.obj
 0001:00000f46       ??_EQPopupMenuList@@UAEPAXI@Z 10001f46 f i navPlugin.obj
 0001:00000f65       ??_Econfig_plugin_base@@UAEPAXI@Z 10001f65 f i navPlugin.obj
 0001:00000f65       ??_Gconfig_plugin_base@@UAEPAXI@Z 10001f65 f i navPlugin.obj
 0001:00000f84       ??_GnavPlugin@@UAEPAXI@Z   10001f84 f i navPlugin.obj
 0001:00000f84       ??_EnavPlugin@@UAEPAXI@Z   10001f84 f i navPlugin.obj
 0001:00000fa3       ?about@config_plugin_base@@UAE?AVQString@@XZ 10001fa3 f i navPlugin.obj
 0001:00000ff9       ?about@navPlugin@@UAE?AVQString@@XZ 10001ff9 f   navPlugin.obj
 0001:000010a1       ?activate@navPlugin@@UAEX_N@Z 100020a1 f   navPlugin.obj
 0001:000010a1       ?activate@config_plugin_base@@UAEX_N@Z 100020a1 f   navPlugin.obj
 0001:000010a1       ?reply@config_plugin_base@@UAEXPAVresponse@@@Z 100020a1 f   navPlugin.obj
 0001:000010a4       ?apply@navPlugin@@UAEXXZ   100020a4 f i navPlugin.obj
 0001:000010a4       ?apply@config_plugin_base@@UAEXXZ 100020a4 f i navPlugin.obj
 0001:000010a5       ?closeEvent@config_plugin_base@@UAEXPAVQCloseEvent@@@Z 100020a5 f i navPlugin.obj
 0001:000010b3       ?closeEvent@navPlugin@@UAEXPAVQCloseEvent@@@Z 100020b3 f   navPlugin.obj
 0001:000010bd       ?db@@YAXABVQString@@@Z     100020bd f   navPlugin.obj
 0001:00001105       ?deleteItem@?$QPtrList@VQPopupMenu@@@@EAEXPAX@Z 10002105 f i navPlugin.obj
 0001:00001120       ?iconClicked@navPlugin@@QAEXHPAVQIconViewItem@@ABVQPoint@@@Z 10002120 f   navPlugin.obj
 0001:00001135       ?iconClicked@navPlugin@@QAEXPAVQIconViewItem@@@Z 10002135 f   navPlugin.obj
 0001:0000117f       ?isDirty@config_plugin_base@@UAE_NXZ 1000217f f i navPlugin.obj
 0001:0000117f       ?isDirty@navPlugin@@UAE_NXZ 1000217f f i navPlugin.obj
 0001:0000117f       ?validate@config_plugin_base@@UAE_NXZ 1000217f f i navPlugin.obj
 0001:00001182       ?menus@config_plugin_base@@UAE?AVQPopupMenuList@@XZ 10002182 f   navPlugin.obj
 0001:00001182       ?menus@navPlugin@@UAE?AVQPopupMenuList@@XZ 10002182 f   navPlugin.obj
 0001:000011a5       ?metaObject@navPlugin@@UBEPAVQMetaObject@@XZ 100021a5 f i navPlugin.obj
 0001:000011aa       ?navigate@config_plugin_base@@UAEXABVQString@@0@Z 100021aa f i navPlugin.obj
 0001:000011ad       ?navigate@navPlugin@@UAEXABVQString@@0@Z 100021ad f   navPlugin.obj
 0001:00001229       ?onItem@navPlugin@@QAEXPAVQIconViewItem@@@Z 10002229 f   navPlugin.obj
 0001:00001269       ?onViewport@navPlugin@@QAEXXZ 10002269 f   navPlugin.obj
 0001:00001271       ?reply@navPlugin@@UAEXPAVresponse@@@Z 10002271 f   navPlugin.obj
 0001:000013b3       ?resizeEvent@navPlugin@@UAEXPAVQResizeEvent@@@Z 100023b3 f   navPlugin.obj
 0001:000013e2       ?textStatus@response@@QAE?AVQString@@W4status@1@@Z 100023e2 f i navPlugin.obj
 0001:00001431       ?toolbars@config_plugin_base@@UAE?AVQDockWindowList@@XZ 10002431 f   navPlugin.obj
 0001:00001431       ?toolbars@navPlugin@@UAE?AVQDockWindowList@@XZ 10002431 f   navPlugin.obj
 0001:00001454       ??0navPluginDlg@@QAE@ABVQString@@PAVQWidget@@PBDI@Z 10002454 f   navPlugindlgimpl.obj
 0001:0000147c       ??1navPluginDlg@@UAE@XZ    1000247c f   navPlugindlgimpl.obj
 0001:0000148e       ??_EnavPluginDlg@@WCI@AEPAXI@Z 1000248e f i navPlugindlgimpl.obj
 0001:00001496       ??_GnavPluginDlg@@UAEPAXI@Z 10002496 f i navPlugindlgimpl.obj
 0001:00001496       ??_EnavPluginDlg@@UAEPAXI@Z 10002496 f i navPlugindlgimpl.obj
 0001:000014b5       ?metaObject@navPluginDlg@@UBEPAVQMetaObject@@XZ 100024b5 f i navPlugindlgimpl.obj
 0001:000014ba       ??_Econfig_plugin_desc_base@@UAEPAXI@Z 100024ba f i plugindesc.obj
 0001:000014ba       ??_Gplugindesc@@UAEPAXI@Z  100024ba f i plugindesc.obj
 0001:000014ba       ??_Eplugindesc@@UAEPAXI@Z  100024ba f i plugindesc.obj
 0001:000014ba       ??_Gconfig_plugin_desc_base@@UAEPAXI@Z 100024ba f i plugindesc.obj
 0001:000014da       ?create@plugindesc@@UAEPAVconfig_plugin_base@@ABVQString@@00@Z 100024da f   plugindesc.obj
 0001:00001512       ?keys@plugindesc@@UAE?AVQStringList@@ABVQString@@0@Z 10002512 f   plugindesc.obj
 0001:00001558       ?pixmap@plugindesc@@UAE?AVQPixmap@@ABVQString@@@Z 10002558 f   plugindesc.obj
 0001:00001577       _load_bncs_config_plugin_desc 10002577 f   plugindesc.obj
 0001:0000158d       ?className@navPlugin@@UBEPBDXZ 1000258d f   moc_navPlugin.obj
 0001:00001593       ?command@navPlugin@@IAEXVQString@@0@Z 10002593 f   moc_navPlugin.obj
 0001:00001653       ?qt_cast@navPlugin@@UAEPAXPBD@Z 10002653 f   moc_navPlugin.obj
 0001:00001681       ?qt_emit@navPlugin@@UAE_NHPAUQUObject@@@Z 10002681 f   moc_navPlugin.obj
 0001:000016e5       ?qt_invoke@navPlugin@@UAE_NHPAUQUObject@@@Z 100026e5 f   moc_navPlugin.obj
 0001:0000174d       ?qt_property@navPlugin@@UAE_NHHPAVQVariant@@@Z 1000274d f   moc_navPlugin.obj
 0001:0000174d       ?qt_property@navPluginDlgBase@@UAE_NHHPAVQVariant@@@Z 1000274d f   moc_navPlugindlg.obj
 0001:00001757       ?staticMetaObject@navPlugin@@SAPAVQMetaObject@@XZ 10002757 f   moc_navPlugin.obj
 0001:000018a9       ?className@navPluginDlgBase@@UBEPBDXZ 100028a9 f   moc_navPlugindlg.obj
 0001:000018af       ?qt_cast@navPluginDlgBase@@UAEPAXPBD@Z 100028af f   moc_navPlugindlg.obj
 0001:000018dd       ?qt_emit@navPluginDlgBase@@UAE_NHPAUQUObject@@@Z 100028dd f   moc_navPlugindlg.obj
 0001:000018e7       ?qt_invoke@navPluginDlgBase@@UAE_NHPAUQUObject@@@Z 100028e7 f   moc_navPlugindlg.obj
 0001:00001919       ?staticMetaObject@navPluginDlgBase@@SAPAVQMetaObject@@XZ 10002919 f   moc_navPlugindlg.obj
 0001:00001963       ?tr@navPluginDlgBase@@SA?AVQString@@PBD0@Z 10002963 f   moc_navPlugindlg.obj
 0001:000019a6       ?className@navPluginDlg@@UBEPBDXZ 100029a6 f   moc_navPlugindlgimpl.obj
 0001:000019ac       ?command@navPluginDlg@@IAEXVQString@@0@Z 100029ac f   moc_navPlugindlgimpl.obj
 0001:00001a6c       ?qt_cast@navPluginDlg@@UAEPAXPBD@Z 10002a6c f   moc_navPlugindlgimpl.obj
 0001:00001a99       ?qt_emit@navPluginDlg@@UAE_NHPAUQUObject@@@Z 10002a99 f   moc_navPlugindlgimpl.obj
 0001:00001afc       ?qt_invoke@navPluginDlg@@UAE_NHPAUQUObject@@@Z 10002afc f   moc_navPlugindlgimpl.obj
 0001:00001b05       ?qt_property@navPluginDlg@@UAE_NHHPAVQVariant@@@Z 10002b05 f   moc_navPlugindlgimpl.obj
 0001:00001b0e       ?staticMetaObject@navPluginDlg@@SAPAVQMetaObject@@XZ 10002b0e f   moc_navPlugindlgimpl.obj
 0001:00001ba2       ??0navPluginDlgBase@@QAE@PAVQWidget@@PBDI@Z 10002ba2 f   navPlugindlg.obj
 0001:00001d47       ??1navPluginDlgBase@@UAE@XZ 10002d47 f   navPlugindlg.obj
 0001:00001d5a       ??_EQIconView@@WCI@AEPAXI@Z 10002d5a f i navPlugindlg.obj
 0001:00001d62       ??_EQLabel@@WCI@AEPAXI@Z   10002d62 f i navPlugindlg.obj
 0001:00001d6a       ??_EQVBoxLayout@@WCI@AEPAXI@Z 10002d6a f i navPlugindlg.obj
 0001:00001d72       ??_EnavPluginDlgBase@@WCI@AEPAXI@Z 10002d72 f i navPlugindlg.obj
 0001:00001d7a       ??_EQIconView@@UAEPAXI@Z   10002d7a f i navPlugindlg.obj
 0001:00001d7a       ??_GQIconView@@UAEPAXI@Z   10002d7a f i navPlugindlg.obj
 0001:00001d9a       ??_EQLabel@@UAEPAXI@Z      10002d9a f i navPlugindlg.obj
 0001:00001d9a       ??_GQLabel@@UAEPAXI@Z      10002d9a f i navPlugindlg.obj
 0001:00001dba       ??_GQVBoxLayout@@UAEPAXI@Z 10002dba f i navPlugindlg.obj
 0001:00001dba       ??_EQVBoxLayout@@UAEPAXI@Z 10002dba f i navPlugindlg.obj
 0001:00001dda       ??_EnavPluginDlgBase@@UAEPAXI@Z 10002dda f i navPlugindlg.obj
 0001:00001dda       ??_GnavPluginDlgBase@@UAEPAXI@Z 10002dda f i navPlugindlg.obj
 0001:00001df9       ?languageChange@navPluginDlgBase@@MAEXXZ 10002df9 f   navPlugindlg.obj
 0001:00001e4d       ?metaObject@navPluginDlgBase@@UBEPAVQMetaObject@@XZ 10002e4d f i navPlugindlg.obj
 0001:00001e52       ?compareItems@QGList@@MAEHPAX0@Z 10002e52 f   qt-mt323:qt-mt323.dll
 0001:00001e58       ?newItem@QPtrCollection@@MAEPAXPAX@Z 10002e58 f   qt-mt323:qt-mt323.dll
 0001:00001e5e       ?read@QGDict@@MAEAAVQDataStream@@AAV2@AAPAX@Z 10002e5e f   qt-mt323:qt-mt323.dll
 0001:00001e64       ?read@QGList@@MAEAAVQDataStream@@AAV2@AAPAX@Z 10002e64 f   qt-mt323:qt-mt323.dll
 0001:00001e6a       ?write@QGDict@@MBEAAVQDataStream@@AAV2@PAX@Z 10002e6a f   qt-mt323:qt-mt323.dll
 0001:00001e70       ?write@QGList@@MBEAAVQDataStream@@AAV2@PAX@Z 10002e70 f   qt-mt323:qt-mt323.dll
 0001:00001e76       ?acceptDrop@QIconViewItem@@UBE_NPBVQMimeSource@@@Z 10002e76 f   qt-mt323:qt-mt323.dll
 0001:00001e7c       ?calcRect@QIconViewItem@@MAEXABVQString@@@Z 10002e7c f   qt-mt323:qt-mt323.dll
 0001:00001e82       ?compare@QIconViewItem@@UBEHPAV1@@Z 10002e82 f   qt-mt323:qt-mt323.dll
 0001:00001e88       ?dragEntered@QIconViewItem@@MAEXXZ 10002e88 f   qt-mt323:qt-mt323.dll
 0001:00001e8e       ?dragLeft@QIconViewItem@@MAEXXZ 10002e8e f   qt-mt323:qt-mt323.dll
 0001:00001e94       ?dropped@QIconViewItem@@MAEXPAVQDropEvent@@ABV?$QValueList@VQIconDragItem@@@@@Z 10002e94 f   qt-mt323:qt-mt323.dll
 0001:00001e9a       ?key@QIconViewItem@@UBE?AVQString@@XZ 10002e9a f   qt-mt323:qt-mt323.dll
 0001:00001ea0       ?move@QIconViewItem@@UAE_NABVQPoint@@@Z 10002ea0 f   qt-mt323:qt-mt323.dll
 0001:00001ea6       ?move@QIconViewItem@@UAE_NHH@Z 10002ea6 f   qt-mt323:qt-mt323.dll
 0001:00001eac       ?moveBy@QIconViewItem@@UAEXABVQPoint@@@Z 10002eac f   qt-mt323:qt-mt323.dll
 0001:00001eb2       ?moveBy@QIconViewItem@@UAEXHH@Z 10002eb2 f   qt-mt323:qt-mt323.dll
 0001:00001eb8       ?paintFocus@QIconViewItem@@MAEXPAVQPainter@@ABVQColorGroup@@@Z 10002eb8 f   qt-mt323:qt-mt323.dll
 0001:00001ebe       ?paintItem@QIconViewItem@@MAEXPAVQPainter@@ABVQColorGroup@@@Z 10002ebe f   qt-mt323:qt-mt323.dll
 0001:00001ec4       ?picture@QIconViewItem@@UBEPAVQPicture@@XZ 10002ec4 f   qt-mt323:qt-mt323.dll
 0001:00001eca       ?pixmap@QIconViewItem@@UBEPAVQPixmap@@XZ 10002eca f   qt-mt323:qt-mt323.dll
 0001:00001ed0       ?removeRenameBox@QIconViewItem@@MAEXXZ 10002ed0 f   qt-mt323:qt-mt323.dll
 0001:00001ed6       ?repaint@QIconViewItem@@UAEXXZ 10002ed6 f   qt-mt323:qt-mt323.dll
 0001:00001edc       ?rtti@QIconViewItem@@UBEHXZ 10002edc f   qt-mt323:qt-mt323.dll
 0001:00001ee2       ?setDragEnabled@QIconViewItem@@UAEX_N@Z 10002ee2 f   qt-mt323:qt-mt323.dll
 0001:00001ee8       ?setDropEnabled@QIconViewItem@@UAEX_N@Z 10002ee8 f   qt-mt323:qt-mt323.dll
 0001:00001eee       ?setKey@QIconViewItem@@UAEXABVQString@@@Z 10002eee f   qt-mt323:qt-mt323.dll
 0001:00001ef4       ?setPicture@QIconViewItem@@UAEXABVQPicture@@@Z 10002ef4 f   qt-mt323:qt-mt323.dll
 0001:00001efa       ?setPixmap@QIconViewItem@@UAEXABVQPixmap@@@Z 10002efa f   qt-mt323:qt-mt323.dll
 0001:00001f00       ?setPixmap@QIconViewItem@@UAEXABVQPixmap@@_N1@Z 10002f00 f   qt-mt323:qt-mt323.dll
 0001:00001f06       ?setRenameEnabled@QIconViewItem@@UAEX_N@Z 10002f06 f   qt-mt323:qt-mt323.dll
 0001:00001f0c       ?setSelectable@QIconViewItem@@UAEX_N@Z 10002f0c f   qt-mt323:qt-mt323.dll
 0001:00001f12       ?setSelected@QIconViewItem@@UAEX_N0@Z 10002f12 f   qt-mt323:qt-mt323.dll
 0001:00001f18       ?setSelected@QIconViewItem@@UAEX_N@Z 10002f18 f   qt-mt323:qt-mt323.dll
 0001:00001f1e       ?setText@QIconViewItem@@UAEXABVQString@@@Z 10002f1e f   qt-mt323:qt-mt323.dll
 0001:00001f24       ?setText@QIconViewItem@@UAEXABVQString@@_N1@Z 10002f24 f   qt-mt323:qt-mt323.dll
 0001:00001f2a       ?text@QIconViewItem@@UBE?AVQString@@XZ 10002f2a f   qt-mt323:qt-mt323.dll
 0001:00001f30       ?setName@QWidget@@UAEXPBD@Z 10002f30 f   qt-mt323:qt-mt323.dll
 0001:00001f36       ?closeEvent@QWidget@@MAEXPAVQCloseEvent@@@Z 10002f36 f   qt-mt323:qt-mt323.dll
 0001:00001f3c       ?adjustSize@QWidget@@UAEXXZ 10002f3c f   qt-mt323:qt-mt323.dll
 0001:00001f42       ?checkConnectArgs@QObject@@MAE_NPBDPBV1@0@Z 10002f42 f   qt-mt323:qt-mt323.dll
 0001:00001f48       ?childEvent@QObject@@MAEXPAVQChildEvent@@@Z 10002f48 f   qt-mt323:qt-mt323.dll
 0001:00001f4e       ?className@QWidget@@UBEPBDXZ 10002f4e f   qt-mt323:qt-mt323.dll
 0001:00001f54       ?clear@?$QPtrList@VQDockWindow@@@@UAEXXZ 10002f54 f   qt-mt323:qt-mt323.dll
 0001:00001f5a       ?close@QWidget@@UAE_N_N@Z  10002f5a f   qt-mt323:qt-mt323.dll
 0001:00001f60       ?cmd@QPaintDevice@@MAE_NHPAVQPainter@@PATQPDevCmdParam@@@Z 10002f60 f   qt-mt323:qt-mt323.dll
 0001:00001f66       ?connectNotify@QObject@@MAEXPBD@Z 10002f66 f   qt-mt323:qt-mt323.dll
 0001:00001f6c       ?contextMenuEvent@QWidget@@MAEXPAVQContextMenuEvent@@@Z 10002f6c f   qt-mt323:qt-mt323.dll
 0001:00001f72       ?count@?$QPtrList@VQDockWindow@@@@UBEIXZ 10002f72 f   qt-mt323:qt-mt323.dll
 0001:00001f78       ?create@QWidget@@MAEXPAUHWND__@@_N1@Z 10002f78 f   qt-mt323:qt-mt323.dll
 0001:00001f7e       ?customEvent@QObject@@MAEXPAVQCustomEvent@@@Z 10002f7e f   qt-mt323:qt-mt323.dll
 0001:00001f84       ?customWhatsThis@QWidget@@UBE_NXZ 10002f84 f   qt-mt323:qt-mt323.dll
 0001:00001f8a       ?deleteItem@?$QPtrList@VQDockWindow@@@@EAEXPAX@Z 10002f8a f   qt-mt323:qt-mt323.dll
 0001:00001f90       ?destroy@QWidget@@MAEX_N0@Z 10002f90 f   qt-mt323:qt-mt323.dll
 0001:00001f96       ?disconnectNotify@QObject@@MAEXPBD@Z 10002f96 f   qt-mt323:qt-mt323.dll
 0001:00001f9c       ?dragEnterEvent@QWidget@@MAEXPAVQDragEnterEvent@@@Z 10002f9c f   qt-mt323:qt-mt323.dll
 0001:00001fa2       ?dragLeaveEvent@QWidget@@MAEXPAVQDragLeaveEvent@@@Z 10002fa2 f   qt-mt323:qt-mt323.dll
 0001:00001fa8       ?dragMoveEvent@QWidget@@MAEXPAVQDragMoveEvent@@@Z 10002fa8 f   qt-mt323:qt-mt323.dll
 0001:00001fae       ?dropEvent@QWidget@@MAEXPAVQDropEvent@@@Z 10002fae f   qt-mt323:qt-mt323.dll
 0001:00001fb4       ?enabledChange@QWidget@@MAEX_N@Z 10002fb4 f   qt-mt323:qt-mt323.dll
 0001:00001fba       ?enterEvent@QWidget@@MAEXPAVQEvent@@@Z 10002fba f   qt-mt323:qt-mt323.dll
 0001:00001fc0       ?event@QWidget@@MAE_NPAVQEvent@@@Z 10002fc0 f   qt-mt323:qt-mt323.dll
 0001:00001fc6       ?eventFilter@QObject@@UAE_NPAV1@PAVQEvent@@@Z 10002fc6 f   qt-mt323:qt-mt323.dll
 0001:00001fcc       ?focusInEvent@QWidget@@MAEXPAVQFocusEvent@@@Z 10002fcc f   qt-mt323:qt-mt323.dll
 0001:00001fd2       ?focusNextPrevChild@QWidget@@MAE_N_N@Z 10002fd2 f   qt-mt323:qt-mt323.dll
 0001:00001fd8       ?focusOutEvent@QWidget@@MAEXPAVQFocusEvent@@@Z 10002fd8 f   qt-mt323:qt-mt323.dll
 0001:00001fde       ?fontChange@QWidget@@MAEXABVQFont@@@Z 10002fde f   qt-mt323:qt-mt323.dll
 0001:00001fe4       ?fontInf@QPaintDevice@@MBEHPAVQFont@@H@Z 10002fe4 f   qt-mt323:qt-mt323.dll
 0001:00001fea       ?fontMet@QPaintDevice@@MBEHPAVQFont@@HPBDH@Z 10002fea f   qt-mt323:qt-mt323.dll
 0001:00001ff0       ?handle@QPaintDevice@@UBEPAUHDC__@@XZ 10002ff0 f   qt-mt323:qt-mt323.dll
 0001:00001ff6       ?heightForWidth@QWidget@@UBEHH@Z 10002ff6 f   qt-mt323:qt-mt323.dll
 0001:00001ffe       ?hide@QWidget@@UAEXXZ      10002ffe f   qt-mt323:qt-mt323.dll
 0001:00002004       ?hideEvent@QWidget@@MAEXPAVQHideEvent@@@Z 10003004 f   qt-mt323:qt-mt323.dll
 0001:0000200a       ?imComposeEvent@QWidget@@MAEXPAVQIMEvent@@@Z 1000300a f   qt-mt323:qt-mt323.dll
 0001:00002010       ?imEndEvent@QWidget@@MAEXPAVQIMEvent@@@Z 10003010 f   qt-mt323:qt-mt323.dll
 0001:00002016       ?imStartEvent@QWidget@@MAEXPAVQIMEvent@@@Z 10003016 f   qt-mt323:qt-mt323.dll
 0001:0000201c       ?insertChild@QObject@@UAEXPAV1@@Z 1000301c f   qt-mt323:qt-mt323.dll
 0001:00002022       ?keyPressEvent@QWidget@@MAEXPAVQKeyEvent@@@Z 10003022 f   qt-mt323:qt-mt323.dll
 0001:00002028       ?keyReleaseEvent@QWidget@@MAEXPAVQKeyEvent@@@Z 10003028 f   qt-mt323:qt-mt323.dll
 0001:0000202e       ?leaveEvent@QWidget@@MAEXPAVQEvent@@@Z 1000302e f   qt-mt323:qt-mt323.dll
 0001:00002034       ?metaObject@QWidget@@UBEPAVQMetaObject@@XZ 10003034 f   qt-mt323:qt-mt323.dll
 0001:0000203a       ?metric@QWidget@@MBEHH@Z   1000303a f   qt-mt323:qt-mt323.dll
 0001:00002040       ?minimumSizeHint@QWidget@@UBE?AVQSize@@XZ 10003040 f   qt-mt323:qt-mt323.dll
 0001:00002046       ?mouseDoubleClickEvent@QWidget@@MAEXPAVQMouseEvent@@@Z 10003046 f   qt-mt323:qt-mt323.dll
 0001:0000204c       ?mouseMoveEvent@QWidget@@MAEXPAVQMouseEvent@@@Z 1000304c f   qt-mt323:qt-mt323.dll
 0001:00002052       ?mousePressEvent@QWidget@@MAEXPAVQMouseEvent@@@Z 10003052 f   qt-mt323:qt-mt323.dll
 0001:00002058       ?mouseReleaseEvent@QWidget@@MAEXPAVQMouseEvent@@@Z 10003058 f   qt-mt323:qt-mt323.dll
 0001:0000205e       ?move@QWidget@@UAEXHH@Z    1000305e f   qt-mt323:qt-mt323.dll
 0001:00002064       ?moveEvent@QWidget@@MAEXPAVQMoveEvent@@@Z 10003064 f   qt-mt323:qt-mt323.dll
 0001:0000206a       ?paintEvent@QWidget@@MAEXPAVQPaintEvent@@@Z 1000306a f   qt-mt323:qt-mt323.dll
 0001:00002070       ?paletteChange@QWidget@@MAEXABVQPalette@@@Z 10003070 f   qt-mt323:qt-mt323.dll
 0001:00002076       ?polish@QWidget@@UAEXXZ    10003076 f   qt-mt323:qt-mt323.dll
 0001:0000207c       ?property@QObject@@UBE?AVQVariant@@PBD@Z 1000307c f   qt-mt323:qt-mt323.dll
 0001:00002082       ?qt_cast@QWidget@@UAEPAXPBD@Z 10003082 f   qt-mt323:qt-mt323.dll
 0001:00002088       ?qt_emit@QWidget@@UAE_NHPAUQUObject@@@Z 10003088 f   qt-mt323:qt-mt323.dll
 0001:0000208e       ?qt_invoke@QWidget@@UAE_NHPAUQUObject@@@Z 1000308e f   qt-mt323:qt-mt323.dll
 0001:00002094       ?qt_property@QWidget@@UAE_NHHPAVQVariant@@@Z 10003094 f   qt-mt323:qt-mt323.dll
 0001:0000209a       ?removeChild@QObject@@UAEXPAV1@@Z 1000309a f   qt-mt323:qt-mt323.dll
 0001:000020a0       ?reparent@QWidget@@UAEXPAV1@IABVQPoint@@_N@Z 100030a0 f   qt-mt323:qt-mt323.dll
 0001:000020a6       ?resize@QWidget@@UAEXHH@Z  100030a6 f   qt-mt323:qt-mt323.dll
 0001:000020ac       ?resizeEvent@QWidget@@MAEXPAVQResizeEvent@@@Z 100030ac f   qt-mt323:qt-mt323.dll
 0001:000020b2       ?resolution@QPaintDevice@@UBEHXZ 100030b2 f   qt-mt323:qt-mt323.dll
 0001:000020b8       ?setAcceptDrops@QWidget@@UAEX_N@Z 100030b8 f   qt-mt323:qt-mt323.dll
 0001:000020be       ?setActiveWindow@QWidget@@UAEXXZ 100030be f   qt-mt323:qt-mt323.dll
 0001:000020c4       ?setAutoMask@QWidget@@UAEX_N@Z 100030c4 f   qt-mt323:qt-mt323.dll
 0001:000020ca       ?setBackgroundColor@QWidget@@UAEXABVQColor@@@Z 100030ca f   qt-mt323:qt-mt323.dll
 0001:000020d0       ?setBackgroundMode@QWidget@@UAEXW4BackgroundMode@Qt@@@Z 100030d0 f   qt-mt323:qt-mt323.dll
 0001:000020d6       ?setBackgroundOrigin@QWidget@@UAEXW4BackgroundOrigin@1@@Z 100030d6 f   qt-mt323:qt-mt323.dll
 0001:000020dc       ?setBackgroundPixmap@QWidget@@UAEXABVQPixmap@@@Z 100030dc f   qt-mt323:qt-mt323.dll
 0001:000020e2       ?setCaption@QWidget@@UAEXABVQString@@@Z 100030e2 f   qt-mt323:qt-mt323.dll
 0001:000020e8       ?setCursor@QWidget@@UAEXABVQCursor@@@Z 100030e8 f   qt-mt323:qt-mt323.dll
 0001:000020ee       ?setEnabled@QWidget@@UAEX_N@Z 100030ee f   qt-mt323:qt-mt323.dll
 0001:000020f4       ?setEraseColor@QWidget@@UAEXABVQColor@@@Z 100030f4 f   qt-mt323:qt-mt323.dll
 0001:000020fa       ?setErasePixmap@QWidget@@UAEXABVQPixmap@@@Z 100030fa f   qt-mt323:qt-mt323.dll
 0001:00002100       ?setFocus@QWidget@@UAEXXZ  10003100 f   qt-mt323:qt-mt323.dll
 0001:00002106       ?setFocusPolicy@QWidget@@UAEXW4FocusPolicy@1@@Z 10003106 f   qt-mt323:qt-mt323.dll
 0001:0000210c       ?setFocusProxy@QWidget@@UAEXPAV1@@Z 1000310c f   qt-mt323:qt-mt323.dll
 0001:00002112       ?setFont@QWidget@@UAEXABVQFont@@@Z 10003112 f   qt-mt323:qt-mt323.dll
 0001:00002118       ?setGeometry@QWidget@@UAEXABVQRect@@@Z 10003118 f   qt-mt323:qt-mt323.dll
 0001:0000211e       ?setGeometry@QWidget@@UAEXHHHH@Z 1000311e f   qt-mt323:qt-mt323.dll
 0001:00002124       ?setIcon@QWidget@@UAEXABVQPixmap@@@Z 10003124 f   qt-mt323:qt-mt323.dll
 0001:0000212a       ?setIconText@QWidget@@UAEXABVQString@@@Z 1000312a f   qt-mt323:qt-mt323.dll
 0001:00002130       ?setKeyCompression@QWidget@@MAEX_N@Z 10003130 f   qt-mt323:qt-mt323.dll
 0001:00002136       ?setMask@QWidget@@UAEXABVQBitmap@@@Z 10003136 f   qt-mt323:qt-mt323.dll
 0001:0000213c       ?setMask@QWidget@@UAEXABVQRegion@@@Z 1000313c f   qt-mt323:qt-mt323.dll
 0001:00002142       ?setMaximumSize@QWidget@@UAEXHH@Z 10003142 f   qt-mt323:qt-mt323.dll
 0001:00002148       ?setMicroFocusHint@QWidget@@MAEXHHHH_NPAVQFont@@@Z 10003148 f   qt-mt323:qt-mt323.dll
 0001:0000214e       ?setMinimumSize@QWidget@@UAEXHH@Z 1000314e f   qt-mt323:qt-mt323.dll
 0001:00002154       ?setMouseTracking@QWidget@@UAEX_N@Z 10003154 f   qt-mt323:qt-mt323.dll
 0001:0000215a       ?setPalette@QWidget@@UAEXABVQPalette@@@Z 1000315a f   qt-mt323:qt-mt323.dll
 0001:00002160       ?setPaletteBackgroundColor@QWidget@@UAEXABVQColor@@@Z 10003160 f   qt-mt323:qt-mt323.dll
 0001:00002166       ?setPaletteBackgroundPixmap@QWidget@@UAEXABVQPixmap@@@Z 10003166 f   qt-mt323:qt-mt323.dll
 0001:0000216c       ?setProperty@QObject@@UAE_NPBDABVQVariant@@@Z 1000316c f   qt-mt323:qt-mt323.dll
 0001:00002172       ?setResolution@QPaintDevice@@UAEXH@Z 10003172 f   qt-mt323:qt-mt323.dll
 0001:00002178       ?setSizeIncrement@QWidget@@UAEXHH@Z 10003178 f   qt-mt323:qt-mt323.dll
 0001:0000217e       ?setSizePolicy@QWidget@@UAEXVQSizePolicy@@@Z 1000317e f   qt-mt323:qt-mt323.dll
 0001:00002184       ?setUpdatesEnabled@QWidget@@UAEX_N@Z 10003184 f   qt-mt323:qt-mt323.dll
 0001:0000218a       ?setWFlags@QWidget@@MAEXI@Z 1000318a f   qt-mt323:qt-mt323.dll
 0001:00002190       ?setWState@QWidget@@MAEXI@Z 10003190 f   qt-mt323:qt-mt323.dll
 0001:00002196       ?show@QWidget@@UAEXXZ      10003196 f   qt-mt323:qt-mt323.dll
 0001:0000219c       ?showEvent@QWidget@@MAEXPAVQShowEvent@@@Z 1000319c f   qt-mt323:qt-mt323.dll
 0001:000021a2       ?showMaximized@QWidget@@UAEXXZ 100031a2 f   qt-mt323:qt-mt323.dll
 0001:000021a8       ?showMinimized@QWidget@@UAEXXZ 100031a8 f   qt-mt323:qt-mt323.dll
 0001:000021ae       ?showNormal@QWidget@@UAEXXZ 100031ae f   qt-mt323:qt-mt323.dll
 0001:000021b4       ?sizeHint@QWidget@@UBE?AVQSize@@XZ 100031b4 f   qt-mt323:qt-mt323.dll
 0001:000021ba       ?sizePolicy@QWidget@@UBE?AVQSizePolicy@@XZ 100031ba f   qt-mt323:qt-mt323.dll
 0001:000021c0       ?styleChange@QWidget@@MAEXAAVQStyle@@@Z 100031c0 f   qt-mt323:qt-mt323.dll
 0001:000021c6       ?tabletEvent@QWidget@@MAEXPAVQTabletEvent@@@Z 100031c6 f   qt-mt323:qt-mt323.dll
 0001:000021cc       ?timerEvent@QObject@@MAEXPAVQTimerEvent@@@Z 100031cc f   qt-mt323:qt-mt323.dll
 0001:000021d2       ?unsetCursor@QWidget@@UAEXXZ 100031d2 f   qt-mt323:qt-mt323.dll
 0001:000021d8       ?updateMask@QWidget@@MAEXXZ 100031d8 f   qt-mt323:qt-mt323.dll
 0001:000021de       ?wheelEvent@QWidget@@MAEXPAVQWheelEvent@@@Z 100031de f   qt-mt323:qt-mt323.dll
 0001:000021e4       ?winEvent@QWidget@@MAE_NPAUtagMSG@@@Z 100031e4 f   qt-mt323:qt-mt323.dll
 0001:000021ea       ?windowActivationChange@QWidget@@MAEX_N@Z 100031ea f   qt-mt323:qt-mt323.dll
 0001:000021f0       ?addChild@QScrollView@@UAEXPAVQWidget@@HH@Z 100031f0 f   qt-mt323:qt-mt323.dll
 0001:000021f6       ?addItem@QBoxLayout@@UAEXPAVQLayoutItem@@@Z 100031f6 f   qt-mt323:qt-mt323.dll
 0001:000021fc       ?adjustItems@QIconView@@MAEXXZ 100031fc f   qt-mt323:qt-mt323.dll
 0001:00002202       ?arrangeItemsInGrid@QIconView@@UAEXABVQSize@@_N@Z 10003202 f   qt-mt323:qt-mt323.dll
 0001:00002208       ?arrangeItemsInGrid@QIconView@@UAEX_N@Z 10003208 f   qt-mt323:qt-mt323.dll
 0001:0000220e       ?childEvent@QLayout@@MAEXPAVQChildEvent@@@Z 1000320e f   qt-mt323:qt-mt323.dll
 0001:00002214       ?className@QIconView@@UBEPBDXZ 10003214 f   qt-mt323:qt-mt323.dll
 0001:0000221a       ?className@QLabel@@UBEPBDXZ 1000321a f   qt-mt323:qt-mt323.dll
 0001:00002220       ?className@QVBoxLayout@@UBEPBDXZ 10003220 f   qt-mt323:qt-mt323.dll
 0001:00002226       ?clear@QIconView@@UAEXXZ   10003226 f   qt-mt323:qt-mt323.dll
 0001:0000222c       ?clearSelection@QIconView@@UAEXXZ 1000322c f   qt-mt323:qt-mt323.dll
 0001:00002232       ?contentsContextMenuEvent@QIconView@@MAEXPAVQContextMenuEvent@@@Z 10003232 f   qt-mt323:qt-mt323.dll
 0001:00002238       ?contentsDragEnterEvent@QIconView@@MAEXPAVQDragEnterEvent@@@Z 10003238 f   qt-mt323:qt-mt323.dll
 0001:0000223e       ?contentsDragLeaveEvent@QIconView@@MAEXPAVQDragLeaveEvent@@@Z 1000323e f   qt-mt323:qt-mt323.dll
 0001:00002244       ?contentsDragMoveEvent@QIconView@@MAEXPAVQDragMoveEvent@@@Z 10003244 f   qt-mt323:qt-mt323.dll
 0001:0000224a       ?contentsDropEvent@QIconView@@MAEXPAVQDropEvent@@@Z 1000324a f   qt-mt323:qt-mt323.dll
 0001:00002250       ?contentsMouseDoubleClickEvent@QIconView@@MAEXPAVQMouseEvent@@@Z 10003250 f   qt-mt323:qt-mt323.dll
 0001:00002256       ?contentsMouseMoveEvent@QIconView@@MAEXPAVQMouseEvent@@@Z 10003256 f   qt-mt323:qt-mt323.dll
 0001:0000225c       ?contentsMousePressEvent@QIconView@@MAEXPAVQMouseEvent@@@Z 1000325c f   qt-mt323:qt-mt323.dll
 0001:00002262       ?contentsMouseReleaseEvent@QIconView@@MAEXPAVQMouseEvent@@@Z 10003262 f   qt-mt323:qt-mt323.dll
 0001:00002268       ?contentsWheelEvent@QScrollView@@MAEXPAVQWheelEvent@@@Z 10003268 f   qt-mt323:qt-mt323.dll
 0001:0000226e       ?contextMenuEvent@QScrollView@@MAEXPAVQContextMenuEvent@@@Z 1000326e f   qt-mt323:qt-mt323.dll
 0001:00002274       ?doAutoScroll@QIconView@@MAEXXZ 10003274 f   qt-mt323:qt-mt323.dll
 0001:0000227a       ?dragObject@QIconView@@MAEPAVQDragObject@@XZ 1000327a f   qt-mt323:qt-mt323.dll
 0001:00002280       ?drawBackground@QIconView@@MAEXPAVQPainter@@ABVQRect@@@Z 10003280 f   qt-mt323:qt-mt323.dll
 0001:00002286       ?drawContents@QIconView@@EAEXPAVQPainter@@@Z 10003286 f   qt-mt323:qt-mt323.dll
 0001:0000228c       ?drawContents@QIconView@@MAEXPAVQPainter@@HHHH@Z 1000328c f   qt-mt323:qt-mt323.dll
 0001:00002292       ?drawContents@QLabel@@MAEXPAVQPainter@@@Z 10003292 f   qt-mt323:qt-mt323.dll
 0001:00002298       ?drawContentsOffset@QScrollView@@MAEXPAVQPainter@@HHHHHH@Z 10003298 f   qt-mt323:qt-mt323.dll
 0001:0000229e       ?drawDragShapes@QIconView@@EAEXABVQPoint@@@Z 1000329e f   qt-mt323:qt-mt323.dll
 0001:000022a4       ?drawFrame@QFrame@@MAEXPAVQPainter@@@Z 100032a4 f   qt-mt323:qt-mt323.dll
 0001:000022aa       ?drawRubber@QIconView@@MAEXPAVQPainter@@@Z 100032aa f   qt-mt323:qt-mt323.dll
 0001:000022b0       ?enterEvent@QIconView@@MAEXPAVQEvent@@@Z 100032b0 f   qt-mt323:qt-mt323.dll
 0001:000022b6       ?event@QObject@@UAE_NPAVQEvent@@@Z 100032b6 f   qt-mt323:qt-mt323.dll
 0001:000022bc       ?eventFilter@QIconView@@UAE_NPAVQObject@@PAVQEvent@@@Z 100032bc f   qt-mt323:qt-mt323.dll
 0001:000022c2       ?eventFilter@QLayout@@MAE_NPAVQObject@@PAVQEvent@@@Z 100032c2 f   qt-mt323:qt-mt323.dll
 0001:000022c8       ?expanding@QBoxLayout@@UBE?AW4ExpandData@QSizePolicy@@XZ 100032c8 f   qt-mt323:qt-mt323.dll
 0001:000022ce       ?focusInEvent@QIconView@@MAEXPAVQFocusEvent@@@Z 100032ce f   qt-mt323:qt-mt323.dll
 0001:000022d4       ?focusNextPrevChild@QScrollView@@MAE_N_N@Z 100032d4 f   qt-mt323:qt-mt323.dll
 0001:000022da       ?focusOutEvent@QIconView@@MAEXPAVQFocusEvent@@@Z 100032da f   qt-mt323:qt-mt323.dll
 0001:000022e0       ?fontChange@QLabel@@MAEXABVQFont@@@Z 100032e0 f   qt-mt323:qt-mt323.dll
 0001:000022e6       ?fontChange@QScrollView@@MAEXABVQFont@@@Z 100032e6 f   qt-mt323:qt-mt323.dll
 0001:000022ec       ?frameChanged@QFrame@@MAEXXZ 100032ec f   qt-mt323:qt-mt323.dll
 0001:000022f2       ?frameChanged@QScrollView@@MAEXXZ 100032f2 f   qt-mt323:qt-mt323.dll
 0001:000022f8       ?geometry@QLayout@@UBE?AVQRect@@XZ 100032f8 f   qt-mt323:qt-mt323.dll
 0001:000022fe       ?hasHeightForWidth@QBoxLayout@@UBE_NXZ 100032fe f   qt-mt323:qt-mt323.dll
 0001:00002304       ?heightForWidth@QBoxLayout@@UBEHH@Z 10003304 f   qt-mt323:qt-mt323.dll
 0001:0000230a       ?heightForWidth@QLabel@@UBEHH@Z 1000330a f   qt-mt323:qt-mt323.dll
 0001:00002310       ?initDragEnter@QIconView@@EAEXPAVQDropEvent@@@Z 10003310 f   qt-mt323:qt-mt323.dll
 0001:00002316       ?insertInGrid@QIconView@@MAEXPAVQIconViewItem@@@Z 10003316 f   qt-mt323:qt-mt323.dll
 0001:0000231c       ?insertItem@QIconView@@UAEXPAVQIconViewItem@@0@Z 1000331c f   qt-mt323:qt-mt323.dll
 0001:00002322       ?invalidate@QBoxLayout@@UAEXXZ 10003322 f   qt-mt323:qt-mt323.dll
 0001:00002328       ?invertSelection@QIconView@@UAEXXZ 10003328 f   qt-mt323:qt-mt323.dll
 0001:0000232e       ?isEmpty@QLayout@@UBE_NXZ  1000332e f   qt-mt323:qt-mt323.dll
 0001:00002334       ?iterator@QBoxLayout@@UAE?AVQLayoutIterator@@XZ 10003334 f   qt-mt323:qt-mt323.dll
 0001:0000233a       ?keyPressEvent@QIconView@@MAEXPAVQKeyEvent@@@Z 1000333a f   qt-mt323:qt-mt323.dll
 0001:00002340       ?layout@QLayout@@UAEPAV1@XZ 10003340 f   qt-mt323:qt-mt323.dll
 0001:00002346       ?maximumSize@QBoxLayout@@UBE?AVQSize@@XZ 10003346 f   qt-mt323:qt-mt323.dll
 0001:0000234c       ?metaObject@QIconView@@UBEPAVQMetaObject@@XZ 1000334c f   qt-mt323:qt-mt323.dll
 0001:00002352       ?metaObject@QLabel@@UBEPAVQMetaObject@@XZ 10003352 f   qt-mt323:qt-mt323.dll
 0001:00002358       ?metaObject@QVBoxLayout@@UBEPAVQMetaObject@@XZ 10003358 f   qt-mt323:qt-mt323.dll
 0001:0000235e       ?minimumSize@QBoxLayout@@UBE?AVQSize@@XZ 1000335e f   qt-mt323:qt-mt323.dll
 0001:00002364       ?minimumSizeHint@QIconView@@UBE?AVQSize@@XZ 10003364 f   qt-mt323:qt-mt323.dll
 0001:0000236a       ?minimumSizeHint@QLabel@@UBE?AVQSize@@XZ 1000336a f   qt-mt323:qt-mt323.dll
 0001:00002370       ?mouseDoubleClickEvent@QScrollView@@MAEXPAVQMouseEvent@@@Z 10003370 f   qt-mt323:qt-mt323.dll
 0001:00002376       ?mouseMoveEvent@QScrollView@@MAEXPAVQMouseEvent@@@Z 10003376 f   qt-mt323:qt-mt323.dll
 0001:0000237c       ?mousePressEvent@QScrollView@@MAEXPAVQMouseEvent@@@Z 1000337c f   qt-mt323:qt-mt323.dll
 0001:00002382       ?mouseReleaseEvent@QScrollView@@MAEXPAVQMouseEvent@@@Z 10003382 f   qt-mt323:qt-mt323.dll
 0001:00002388       ?moveChild@QScrollView@@UAEXPAVQWidget@@HH@Z 10003388 f   qt-mt323:qt-mt323.dll
 0001:0000238e       ?paintEvent@QFrame@@MAEXPAVQPaintEvent@@@Z 1000338e f   qt-mt323:qt-mt323.dll
 0001:00002394       ?qt_cast@QIconView@@UAEPAXPBD@Z 10003394 f   qt-mt323:qt-mt323.dll
 0001:0000239a       ?qt_cast@QLabel@@UAEPAXPBD@Z 1000339a f   qt-mt323:qt-mt323.dll
 0001:000023a0       ?qt_cast@QVBoxLayout@@UAEPAXPBD@Z 100033a0 f   qt-mt323:qt-mt323.dll
 0001:000023a6       ?qt_emit@QIconView@@UAE_NHPAUQUObject@@@Z 100033a6 f   qt-mt323:qt-mt323.dll
 0001:000023ac       ?qt_emit@QLabel@@UAE_NHPAUQUObject@@@Z 100033ac f   qt-mt323:qt-mt323.dll
 0001:000023b2       ?qt_emit@QVBoxLayout@@UAE_NHPAUQUObject@@@Z 100033b2 f   qt-mt323:qt-mt323.dll
 0001:000023b8       ?qt_invoke@QIconView@@UAE_NHPAUQUObject@@@Z 100033b8 f   qt-mt323:qt-mt323.dll
 0001:000023be       ?qt_invoke@QLabel@@UAE_NHPAUQUObject@@@Z 100033be f   qt-mt323:qt-mt323.dll
 0001:000023c4       ?qt_invoke@QVBoxLayout@@UAE_NHPAUQUObject@@@Z 100033c4 f   qt-mt323:qt-mt323.dll
 0001:000023ca       ?qt_property@QIconView@@UAE_NHHPAVQVariant@@@Z 100033ca f   qt-mt323:qt-mt323.dll
 0001:000023d0       ?qt_property@QLabel@@UAE_NHHPAVQVariant@@@Z 100033d0 f   qt-mt323:qt-mt323.dll
 0001:000023d6       ?qt_property@QVBoxLayout@@UAE_NHHPAVQVariant@@@Z 100033d6 f   qt-mt323:qt-mt323.dll
 0001:000023dc       ?removeChild@QScrollView@@UAEXPAVQObject@@@Z 100033dc f   qt-mt323:qt-mt323.dll
 0001:000023e2       ?repaintItem@QIconView@@UAEXPAVQIconViewItem@@@Z 100033e2 f   qt-mt323:qt-mt323.dll
 0001:000023e8       ?resize@QScrollView@@UAEXHH@Z 100033e8 f   qt-mt323:qt-mt323.dll
 0001:000023ee       ?resizeContents@QScrollView@@UAEXHH@Z 100033ee f   qt-mt323:qt-mt323.dll
 0001:000023f4       ?resizeEvent@QIconView@@MAEXPAVQResizeEvent@@@Z 100033f4 f   qt-mt323:qt-mt323.dll
 0001:000023fa       ?resizeEvent@QLabel@@MAEXPAVQResizeEvent@@@Z 100033fa f   qt-mt323:qt-mt323.dll
 0001:00002400       ?selectAll@QIconView@@UAEX_N@Z 10003400 f   qt-mt323:qt-mt323.dll
 0001:00002406       ?setAlignment@QLabel@@UAEXH@Z 10003406 f   qt-mt323:qt-mt323.dll
 0001:0000240c       ?setAlignment@QLayoutItem@@UAEXH@Z 1000340c f   qt-mt323:qt-mt323.dll
 0001:00002412       ?setArrangement@QIconView@@UAEXW4Arrangement@1@@Z 10003412 f   qt-mt323:qt-mt323.dll
 0001:00002418       ?setAutoAdd@QLayout@@UAEX_N@Z 10003418 f   qt-mt323:qt-mt323.dll
 0001:0000241e       ?setAutoArrange@QIconView@@UAEX_N@Z 1000341e f   qt-mt323:qt-mt323.dll
 0001:00002424       ?setAutoResize@QLabel@@UAEX_N@Z 10003424 f   qt-mt323:qt-mt323.dll
 0001:0000242a       ?setBuddy@QLabel@@UAEXPAVQWidget@@@Z 1000342a f   qt-mt323:qt-mt323.dll
 0001:00002430       ?setContentsPos@QIconView@@UAEXHH@Z 10003430 f   qt-mt323:qt-mt323.dll
 0001:00002436       ?setCornerWidget@QScrollView@@UAEXPAVQWidget@@@Z 10003436 f   qt-mt323:qt-mt323.dll
 0001:0000243c       ?setCurrentItem@QIconView@@UAEXPAVQIconViewItem@@@Z 1000343c f   qt-mt323:qt-mt323.dll
 0001:00002442       ?setDragAutoScroll@QScrollView@@UAEX_N@Z 10003442 f   qt-mt323:qt-mt323.dll
 0001:00002448       ?setEnabled@QScrollView@@UAEX_N@Z 10003448 f   qt-mt323:qt-mt323.dll
 0001:0000244e       ?setFont@QIconView@@UAEXABVQFont@@@Z 1000344e f   qt-mt323:qt-mt323.dll
 0001:00002454       ?setFont@QLabel@@UAEXABVQFont@@@Z 10003454 f   qt-mt323:qt-mt323.dll
 0001:0000245a       ?setFrameRect@QFrame@@UAEXABVQRect@@@Z 1000345a f   qt-mt323:qt-mt323.dll
 0001:00002460       ?setFrameStyle@QFrame@@UAEXH@Z 10003460 f   qt-mt323:qt-mt323.dll
 0001:00002466       ?setGeometry@QBoxLayout@@UAEXABVQRect@@@Z 10003466 f   qt-mt323:qt-mt323.dll
 0001:0000246c       ?setGridX@QIconView@@UAEXH@Z 1000346c f   qt-mt323:qt-mt323.dll
 0001:00002472       ?setGridY@QIconView@@UAEXH@Z 10003472 f   qt-mt323:qt-mt323.dll
 0001:00002478       ?setHBarGeometry@QScrollView@@MAEXAAVQScrollBar@@HHHH@Z 10003478 f   qt-mt323:qt-mt323.dll
 0001:0000247e       ?setHScrollBarMode@QScrollView@@UAEXW4ScrollBarMode@1@@Z 1000347e f   qt-mt323:qt-mt323.dll
 0001:00002484       ?setItemTextBackground@QIconView@@UAEXABVQBrush@@@Z 10003484 f   qt-mt323:qt-mt323.dll
 0001:0000248a       ?setItemTextPos@QIconView@@UAEXW4ItemTextPos@1@@Z 1000348a f   qt-mt323:qt-mt323.dll
 0001:00002490       ?setItemsMovable@QIconView@@UAEX_N@Z 10003490 f   qt-mt323:qt-mt323.dll
 0001:00002496       ?setLineWidth@QFrame@@UAEXH@Z 10003496 f   qt-mt323:qt-mt323.dll
 0001:0000249c       ?setMargin@QFrame@@UAEXH@Z 1000349c f   qt-mt323:qt-mt323.dll
 0001:000024a2       ?setMargin@QLayout@@UAEXH@Z 100034a2 f   qt-mt323:qt-mt323.dll
 0001:000024a8       ?setMargins@QScrollView@@MAEXHHHH@Z 100034a8 f   qt-mt323:qt-mt323.dll
 0001:000024ae       ?setMaxItemTextLength@QIconView@@UAEXH@Z 100034ae f   qt-mt323:qt-mt323.dll
 0001:000024b4       ?setMaxItemWidth@QIconView@@UAEXH@Z 100034b4 f   qt-mt323:qt-mt323.dll
 0001:000024ba       ?setMenuBar@QLayout@@UAEXPAVQMenuBar@@@Z 100034ba f   qt-mt323:qt-mt323.dll
 0001:000024c0       ?setMidLineWidth@QFrame@@UAEXH@Z 100034c0 f   qt-mt323:qt-mt323.dll
 0001:000024c6       ?setMovie@QLabel@@UAEXABVQMovie@@@Z 100034c6 f   qt-mt323:qt-mt323.dll
 0001:000024cc       ?setName@QObject@@UAEXPBD@Z 100034cc f   qt-mt323:qt-mt323.dll
 0001:000024d2       ?setNum@QLabel@@UAEXH@Z    100034d2 f   qt-mt323:qt-mt323.dll
 0001:000024d8       ?setNum@QLabel@@UAEXN@Z    100034d8 f   qt-mt323:qt-mt323.dll
 0001:000024de       ?setPalette@QIconView@@UAEXABVQPalette@@@Z 100034de f   qt-mt323:qt-mt323.dll
 0001:000024e4       ?setPicture@QLabel@@UAEXABVQPicture@@@Z 100034e4 f   qt-mt323:qt-mt323.dll
 0001:000024ea       ?setPixmap@QLabel@@UAEXABVQPixmap@@@Z 100034ea f   qt-mt323:qt-mt323.dll
 0001:000024f0       ?setResizeMode@QIconView@@UAEXW4ResizeMode@1@@Z 100034f0 f   qt-mt323:qt-mt323.dll
 0001:000024f6       ?setResizePolicy@QScrollView@@UAEXW4ResizePolicy@1@@Z 100034f6 f   qt-mt323:qt-mt323.dll
 0001:000024fc       ?setSelected@QIconView@@UAEXPAVQIconViewItem@@_N1@Z 100034fc f   qt-mt323:qt-mt323.dll
 0001:00002502       ?setSelectionMode@QIconView@@UAEXW4SelectionMode@1@@Z 10003502 f   qt-mt323:qt-mt323.dll
 0001:00002508       ?setShowToolTips@QIconView@@UAEX_N@Z 10003508 f   qt-mt323:qt-mt323.dll
 0001:0000250e       ?setSpacing@QIconView@@UAEXH@Z 1000350e f   qt-mt323:qt-mt323.dll
 0001:00002514       ?setSpacing@QLayout@@UAEXH@Z 10003514 f   qt-mt323:qt-mt323.dll
 0001:0000251a       ?setText@QLabel@@UAEXABVQString@@@Z 1000351a f   qt-mt323:qt-mt323.dll
 0001:00002520       ?setVBarGeometry@QScrollView@@MAEXAAVQScrollBar@@HHHH@Z 10003520 f   qt-mt323:qt-mt323.dll
 0001:00002526       ?setVScrollBarMode@QScrollView@@UAEXW4ScrollBarMode@1@@Z 10003526 f   qt-mt323:qt-mt323.dll
 0001:0000252c       ?setWordWrapIconText@QIconView@@UAEX_N@Z 1000352c f   qt-mt323:qt-mt323.dll
 0001:00002532       ?show@QScrollView@@UAEXXZ  10003532 f   qt-mt323:qt-mt323.dll
 0001:00002538       ?showEvent@QIconView@@UAEXPAVQShowEvent@@@Z 10003538 f   qt-mt323:qt-mt323.dll
 0001:0000253e       ?sizeHint@QBoxLayout@@UBE?AVQSize@@XZ 1000353e f   qt-mt323:qt-mt323.dll
 0001:00002544       ?sizeHint@QIconView@@UBE?AVQSize@@XZ 10003544 f   qt-mt323:qt-mt323.dll
 0001:0000254a       ?sizeHint@QLabel@@UBE?AVQSize@@XZ 1000354a f   qt-mt323:qt-mt323.dll
 0001:00002550       ?slotUpdate@QIconView@@MAEXXZ 10003550 f   qt-mt323:qt-mt323.dll
 0001:00002556       ?sort@QIconView@@UAEX_N@Z  10003556 f   qt-mt323:qt-mt323.dll
 0001:0000255c       ?spacerItem@QLayoutItem@@UAEPAVQSpacerItem@@XZ 1000355c f   qt-mt323:qt-mt323.dll
 0001:00002562       ?startDrag@QIconView@@MAEXXZ 10003562 f   qt-mt323:qt-mt323.dll
 0001:00002568       ?styleChange@QFrame@@MAEXAAVQStyle@@@Z 10003568 f   qt-mt323:qt-mt323.dll
 0001:0000256e       ?styleChange@QIconView@@MAEXAAVQStyle@@@Z 1000356e f   qt-mt323:qt-mt323.dll
 0001:00002574       ?takeItem@QIconView@@UAEXPAVQIconViewItem@@@Z 10003574 f   qt-mt323:qt-mt323.dll
 0001:0000257a       ?updateContents@QIconView@@UAEXXZ 1000357a f   qt-mt323:qt-mt323.dll
 0001:00002580       ?viewportContextMenuEvent@QScrollView@@MAEXPAVQContextMenuEvent@@@Z 10003580 f   qt-mt323:qt-mt323.dll
 0001:00002586       ?viewportDragEnterEvent@QScrollView@@MAEXPAVQDragEnterEvent@@@Z 10003586 f   qt-mt323:qt-mt323.dll
 0001:0000258c       ?viewportDragLeaveEvent@QScrollView@@MAEXPAVQDragLeaveEvent@@@Z 1000358c f   qt-mt323:qt-mt323.dll
 0001:00002592       ?viewportDragMoveEvent@QScrollView@@MAEXPAVQDragMoveEvent@@@Z 10003592 f   qt-mt323:qt-mt323.dll
 0001:00002598       ?viewportDropEvent@QScrollView@@MAEXPAVQDropEvent@@@Z 10003598 f   qt-mt323:qt-mt323.dll
 0001:0000259e       ?viewportMouseDoubleClickEvent@QScrollView@@MAEXPAVQMouseEvent@@@Z 1000359e f   qt-mt323:qt-mt323.dll
 0001:000025a4       ?viewportMouseMoveEvent@QScrollView@@MAEXPAVQMouseEvent@@@Z 100035a4 f   qt-mt323:qt-mt323.dll
 0001:000025aa       ?viewportMousePressEvent@QScrollView@@MAEXPAVQMouseEvent@@@Z 100035aa f   qt-mt323:qt-mt323.dll
 0001:000025b0       ?viewportMouseReleaseEvent@QScrollView@@MAEXPAVQMouseEvent@@@Z 100035b0 f   qt-mt323:qt-mt323.dll
 0001:000025b6       ?viewportPaintEvent@QScrollView@@MAEXPAVQPaintEvent@@@Z 100035b6 f   qt-mt323:qt-mt323.dll
 0001:000025bc       ?viewportResizeEvent@QScrollView@@MAEXPAVQResizeEvent@@@Z 100035bc f   qt-mt323:qt-mt323.dll
 0001:000025c2       ?viewportWheelEvent@QScrollView@@MAEXPAVQWheelEvent@@@Z 100035c2 f   qt-mt323:qt-mt323.dll
 0001:000025c8       ?wheelEvent@QScrollView@@MAEXPAVQWheelEvent@@@Z 100035c8 f   qt-mt323:qt-mt323.dll
 0001:000025ce       ?widget@QLayoutItem@@UAEPAVQWidget@@XZ 100035ce f   qt-mt323:qt-mt323.dll
 0001:000025d4       ?windowActivationChange@QIconView@@MAEX_N@Z 100035d4 f   qt-mt323:qt-mt323.dll
 0001:000025da       ??2@YAPAXI@Z               100035da f   MSVCRT:MSVCR120.dll
 0001:000025e0       ??3@YAXPAX@Z               100035e0 f   MSVCRT:MSVCR120.dll
 0001:000025e6       @__security_check_cookie@4 100035e6 f   MSVCRT:secchk.obj
 0001:000025f5       __EH_epilog3               100035f5 f   MSVCRT:ehprolg3.obj
 0001:00002609       __EH_epilog3_GS            10003609 f   MSVCRT:ehprolg3.obj
 0001:00002618       __EH_prolog3               10003618 f   MSVCRT:ehprolg3.obj
 0001:0000264b       __EH_prolog3_GS            1000364b f   MSVCRT:ehprolg3.obj
 0001:00002682       ___CxxFrameHandler3        10003682 f   MSVCRT:MSVCR120.dll
 0001:00002688       ??_Etype_info@@UAEPAXI@Z   10003688 f i MSVCRT:ti_inst.obj
 0001:000026d2       __purecall                 100036d2 f   MSVCRT:MSVCR120.dll
 0001:000026d8       ??_L@YGXPAXIHP6EX0@Z1@Z    100036d8 f   MSVCRT:ehvecctr.obj
 0001:0000273a       ??_M@YGXPAXIHP6EX0@Z@Z     1000373a f   MSVCRT:ehvecdtr.obj
 0001:000027a9       ?__ArrayUnwind@@YGXPAXIHP6EX0@Z@Z 100037a9 f   MSVCRT:ehvecdtr.obj
 0001:00002807       ___atonexitinit            10003807 f   MSVCRT:atonexit.obj
 0001:00002843       __onexit                   10003843 f   MSVCRT:atonexit.obj
 0001:000028ec       _atexit                    100038ec f   MSVCRT:atonexit.obj
 0001:0000294d       __CRT_INIT@12              1000394d f   MSVCRT:crtdll.obj
 0001:00002b44       __DllMainCRTStartup@12     10003b44 f   MSVCRT:crtdll.obj
 0001:00002c9a       ___raise_securityfailure   10003c9a f   MSVCRT:gs_report.obj
 0001:00002cd7       ___report_gsfailure        10003cd7 f   MSVCRT:gs_report.obj
 0001:00002dd2       ??1type_info@@UAE@XZ       10003dd2 f   MSVCRT:MSVCR120.dll
 0001:00002de0       __SEH_prolog4              10003de0 f   MSVCRT:sehprolg4.obj
 0001:00002e25       __SEH_epilog4              10003e25 f   MSVCRT:sehprolg4.obj
 0001:00002e39       __except_handler4          10003e39 f   MSVCRT:chandler4gs.obj
 0001:00002e5c       ?terminate@@YAXXZ          10003e5c f   MSVCRT:MSVCR120.dll
 0001:00002e62       __lock                     10003e62 f   MSVCRT:MSVCR120.dll
 0001:00002e68       __unlock                   10003e68 f   MSVCRT:MSVCR120.dll
 0001:00002e6e       ___dllonexit               10003e6e f   MSVCRT:MSVCR120.dll
 0001:00002e74       ___CppXcptFilter           10003e74 f   MSVCRT:MSVCR120.dll
 0001:00002e7a       __amsg_exit                10003e7a f   MSVCRT:MSVCR120.dll
 0001:00002e80       __FindPESection            10003e80 f   MSVCRT:pesect.obj
 0001:00002ed0       __IsNonwritableInCurrentImage 10003ed0 f   MSVCRT:pesect.obj
 0001:00002f90       __ValidateImageBase        10003f90 f   MSVCRT:pesect.obj
 0001:00002fc1       ___security_init_cookie    10003fc1 f   MSVCRT:gs_support.obj
 0001:0000305d       _DllMain@12                1000405d f   MSVCRT:dllmain.obj
 0001:0000307f       __RTC_Initialize           1000407f f   MSVCRT:initsect.obj
 0001:0000309f       __RTC_Terminate            1000409f f   MSVCRT:initsect.obj
 0001:000030c0       __initterm                 100040c0 f   MSVCRT:MSVCR120.dll
 0001:000030c6       __initterm_e               100040c6 f   MSVCRT:MSVCR120.dll
 0001:000030cc       ___clean_type_info_names   100040cc f   MSVCRT:tncleanup.obj
 0001:000030d8       __crt_debugger_hook        100040d8 f   MSVCRT:MSVCR120.dll
 0001:000030de       ___crtUnhandledException   100040de f   MSVCRT:MSVCR120.dll
 0001:000030e4       ___crtTerminateProcess     100040e4 f   MSVCRT:MSVCR120.dll
 0001:000030ea       __except_handler4_common   100040ea f   MSVCRT:MSVCR120.dll
 0001:000030f0       ___clean_type_info_names_internal 100040f0 f   MSVCRT:MSVCR120.dll
 0001:000030f6       _IsProcessorFeaturePresent@4 100040f6 f   kernel32:KERNEL32.dll
 0002:00000000       __imp__GetSystemTimeAsFileTime@4 10005000     kernel32:KERNEL32.dll
 0002:00000004       __imp__GetCurrentThreadId@0 10005004     kernel32:KERNEL32.dll
 0002:00000008       __imp__GetCurrentProcessId@0 10005008     kernel32:KERNEL32.dll
 0002:0000000c       __imp__QueryPerformanceCounter@4 1000500c     kernel32:KERNEL32.dll
 0002:00000010       __imp__IsProcessorFeaturePresent@4 10005010     kernel32:KERNEL32.dll
 0002:00000014       __imp__IsDebuggerPresent@0 10005014     kernel32:KERNEL32.dll
 0002:00000018       __imp__DecodePointer@4     10005018     kernel32:KERNEL32.dll
 0002:0000001c       __imp__EncodePointer@4     1000501c     kernel32:KERNEL32.dll
 0002:00000020       __imp__DisableThreadLibraryCalls@4 10005020     kernel32:KERNEL32.dll
 0002:00000024       \177KERNEL32_NULL_THUNK_DATA 10005024     kernel32:KERNEL32.dll
 0002:00000028       __imp____clean_type_info_names_internal 10005028     MSVCRT:MSVCR120.dll
 0002:0000002c       __imp____crtTerminateProcess 1000502c     MSVCRT:MSVCR120.dll
 0002:00000030       __imp____crtUnhandledException 10005030     MSVCRT:MSVCR120.dll
 0002:00000034       __imp___crt_debugger_hook  10005034     MSVCRT:MSVCR120.dll
 0002:00000038       __imp___initterm_e         10005038     MSVCRT:MSVCR120.dll
 0002:0000003c       __imp___initterm           1000503c     MSVCRT:MSVCR120.dll
 0002:00000040       __imp___malloc_crt         10005040     MSVCRT:MSVCR120.dll
 0002:00000044       __imp__free                10005044     MSVCRT:MSVCR120.dll
 0002:00000048       __imp___amsg_exit          10005048     MSVCRT:MSVCR120.dll
 0002:0000004c       __imp____CppXcptFilter     1000504c     MSVCRT:MSVCR120.dll
 0002:00000050       __imp___onexit             10005050     MSVCRT:MSVCR120.dll
 0002:00000054       __imp____dllonexit         10005054     MSVCRT:MSVCR120.dll
 0002:00000058       __imp___calloc_crt         10005058     MSVCRT:MSVCR120.dll
 0002:0000005c       __imp___unlock             1000505c     MSVCRT:MSVCR120.dll
 0002:00000060       __imp___lock               10005060     MSVCRT:MSVCR120.dll
 0002:00000064       __imp_?terminate@@YAXXZ    10005064     MSVCRT:MSVCR120.dll
 0002:00000068       __imp_??1type_info@@UAE@XZ 10005068     MSVCRT:MSVCR120.dll
 0002:0000006c       __imp___purecall           1000506c     MSVCRT:MSVCR120.dll
 0002:00000070       __imp____CxxFrameHandler3  10005070     MSVCRT:MSVCR120.dll
 0002:00000074       __imp_??3@YAXPAX@Z         10005074     MSVCRT:MSVCR120.dll
 0002:00000078       __imp_??2@YAPAXI@Z         10005078     MSVCRT:MSVCR120.dll
 0002:0000007c       __imp___except_handler4_common 1000507c     MSVCRT:MSVCR120.dll
 0002:00000080       \177MSVCR120_NULL_THUNK_DATA 10005080     MSVCRT:MSVCR120.dll
 0002:00000084       __imp_?documentElement@QDomDocument@@QBE?AVQDomElement@@XZ 10005084     qt-mt323:qt-mt323.dll
 0002:00000088       __imp_?setContent@QDomDocument@@QAE_NPAVQIODevice@@PAVQString@@PAH2@Z 10005088     qt-mt323:qt-mt323.dll
 0002:0000008c       __imp_??1QDomElement@@UAE@XZ 1000508c     qt-mt323:qt-mt323.dll
 0002:00000090       __imp_?attribute@QDomElement@@QBE?AVQString@@ABV2@0@Z 10005090     qt-mt323:qt-mt323.dll
 0002:00000094       __imp_?tagName@QDomElement@@QBE?AVQString@@XZ 10005094     qt-mt323:qt-mt323.dll
 0002:00000098       __imp_??0QFile@@QAE@ABVQString@@@Z 10005098     qt-mt323:qt-mt323.dll
 0002:0000009c       __imp_??1QFile@@UAE@XZ     1000509c     qt-mt323:qt-mt323.dll
 0002:000000a0       __imp_?open@QFile@@UAE_NH@Z 100050a0     qt-mt323:qt-mt323.dll
 0002:000000a4       __imp_?close@QFile@@UAEXXZ 100050a4     qt-mt323:qt-mt323.dll
 0002:000000a8       __imp_?compareItems@QGList@@MAEHPAX0@Z 100050a8     qt-mt323:qt-mt323.dll
 0002:000000ac       __imp_?newItem@QPtrCollection@@MAEPAXPAX@Z 100050ac     qt-mt323:qt-mt323.dll
 0002:000000b0       __imp_?read@QGDict@@MAEAAVQDataStream@@AAV2@AAPAX@Z 100050b0     qt-mt323:qt-mt323.dll
 0002:000000b4       __imp_?read@QGList@@MAEAAVQDataStream@@AAV2@AAPAX@Z 100050b4     qt-mt323:qt-mt323.dll
 0002:000000b8       __imp_?write@QGDict@@MBEAAVQDataStream@@AAV2@PAX@Z 100050b8     qt-mt323:qt-mt323.dll
 0002:000000bc       __imp_?write@QGList@@MBEAAVQDataStream@@AAV2@PAX@Z 100050bc     qt-mt323:qt-mt323.dll
 0002:000000c0       __imp_?null@QString@@2V1@A 100050c0     qt-mt323:qt-mt323.dll
 0002:000000c4       __imp_??0QIconViewItem@@QAE@PAVQIconView@@ABVQString@@@Z 100050c4     qt-mt323:qt-mt323.dll
 0002:000000c8       __imp_??0QIconViewItem@@QAE@PAVQIconView@@ABVQString@@ABVQPixmap@@@Z 100050c8     qt-mt323:qt-mt323.dll
 0002:000000cc       __imp_??1QIconViewItem@@UAE@XZ 100050cc     qt-mt323:qt-mt323.dll
 0002:000000d0       __imp_?acceptDrop@QIconViewItem@@UBE_NPBVQMimeSource@@@Z 100050d0     qt-mt323:qt-mt323.dll
 0002:000000d4       __imp_?calcRect@QIconViewItem@@MAEXABVQString@@@Z 100050d4     qt-mt323:qt-mt323.dll
 0002:000000d8       __imp_?compare@QIconViewItem@@UBEHPAV1@@Z 100050d8     qt-mt323:qt-mt323.dll
 0002:000000dc       __imp_?dragEntered@QIconViewItem@@MAEXXZ 100050dc     qt-mt323:qt-mt323.dll
 0002:000000e0       __imp_?dragLeft@QIconViewItem@@MAEXXZ 100050e0     qt-mt323:qt-mt323.dll
 0002:000000e4       __imp_?dropped@QIconViewItem@@MAEXPAVQDropEvent@@ABV?$QValueList@VQIconDragItem@@@@@Z 100050e4     qt-mt323:qt-mt323.dll
 0002:000000e8       __imp_?key@QIconViewItem@@UBE?AVQString@@XZ 100050e8     qt-mt323:qt-mt323.dll
 0002:000000ec       __imp_?move@QIconViewItem@@UAE_NABVQPoint@@@Z 100050ec     qt-mt323:qt-mt323.dll
 0002:000000f0       __imp_?move@QIconViewItem@@UAE_NHH@Z 100050f0     qt-mt323:qt-mt323.dll
 0002:000000f4       __imp_?moveBy@QIconViewItem@@UAEXABVQPoint@@@Z 100050f4     qt-mt323:qt-mt323.dll
 0002:000000f8       __imp_?moveBy@QIconViewItem@@UAEXHH@Z 100050f8     qt-mt323:qt-mt323.dll
 0002:000000fc       __imp_?paintFocus@QIconViewItem@@MAEXPAVQPainter@@ABVQColorGroup@@@Z 100050fc     qt-mt323:qt-mt323.dll
 0002:00000100       __imp_?paintItem@QIconViewItem@@MAEXPAVQPainter@@ABVQColorGroup@@@Z 10005100     qt-mt323:qt-mt323.dll
 0002:00000104       __imp_?picture@QIconViewItem@@UBEPAVQPicture@@XZ 10005104     qt-mt323:qt-mt323.dll
 0002:00000108       __imp_?pixmap@QIconViewItem@@UBEPAVQPixmap@@XZ 10005108     qt-mt323:qt-mt323.dll
 0002:0000010c       __imp_?removeRenameBox@QIconViewItem@@MAEXXZ 1000510c     qt-mt323:qt-mt323.dll
 0002:00000110       __imp_?repaint@QIconViewItem@@UAEXXZ 10005110     qt-mt323:qt-mt323.dll
 0002:00000114       __imp_?rtti@QIconViewItem@@UBEHXZ 10005114     qt-mt323:qt-mt323.dll
 0002:00000118       __imp_?setDragEnabled@QIconViewItem@@UAEX_N@Z 10005118     qt-mt323:qt-mt323.dll
 0002:0000011c       __imp_?setDropEnabled@QIconViewItem@@UAEX_N@Z 1000511c     qt-mt323:qt-mt323.dll
 0002:00000120       __imp_?setKey@QIconViewItem@@UAEXABVQString@@@Z 10005120     qt-mt323:qt-mt323.dll
 0002:00000124       __imp_?setPicture@QIconViewItem@@UAEXABVQPicture@@@Z 10005124     qt-mt323:qt-mt323.dll
 0002:00000128       __imp_?setPixmap@QIconViewItem@@UAEXABVQPixmap@@@Z 10005128     qt-mt323:qt-mt323.dll
 0002:0000012c       __imp_?setPixmap@QIconViewItem@@UAEXABVQPixmap@@_N1@Z 1000512c     qt-mt323:qt-mt323.dll
 0002:00000130       __imp_?setRenameEnabled@QIconViewItem@@UAEX_N@Z 10005130     qt-mt323:qt-mt323.dll
 0002:00000134       __imp_?setSelectable@QIconViewItem@@UAEX_N@Z 10005134     qt-mt323:qt-mt323.dll
 0002:00000138       __imp_?setSelected@QIconViewItem@@UAEX_N0@Z 10005138     qt-mt323:qt-mt323.dll
 0002:0000013c       __imp_?setSelected@QIconViewItem@@UAEX_N@Z 1000513c     qt-mt323:qt-mt323.dll
 0002:00000140       __imp_?setText@QIconViewItem@@UAEXABVQString@@@Z 10005140     qt-mt323:qt-mt323.dll
 0002:00000144       __imp_?setText@QIconViewItem@@UAEXABVQString@@_N1@Z 10005144     qt-mt323:qt-mt323.dll
 0002:00000148       __imp_?text@QIconViewItem@@UBE?AVQString@@XZ 10005148     qt-mt323:qt-mt323.dll
 0002:0000014c       __imp_??0QString@@QAE@ABV0@@Z 1000514c     qt-mt323:qt-mt323.dll
 0002:00000150       __imp_?arg@QString@@QBE?AV1@ABV1@H@Z 10005150     qt-mt323:qt-mt323.dll
 0002:00000154       __imp_?ascii@QString@@QBEPBDXZ 10005154     qt-mt323:qt-mt323.dll
 0002:00000158       __imp_??H@YA?BVQString@@PBDABV0@@Z 10005158     qt-mt323:qt-mt323.dll
 0002:0000015c       __imp_?first@QGList@@IAEPAXXZ 1000515c     qt-mt323:qt-mt323.dll
 0002:00000160       __imp_?next@QGList@@IAEPAXXZ 10005160     qt-mt323:qt-mt323.dll
 0002:00000164       __imp_?connect@QObject@@SA_NPBV1@PBD01@Z 10005164     qt-mt323:qt-mt323.dll
 0002:00000168       __imp_??0QWidget@@QAE@PAV0@PBDI@Z 10005168     qt-mt323:qt-mt323.dll
 0002:0000016c       __imp_??1QWidget@@UAE@XZ   1000516c     qt-mt323:qt-mt323.dll
 0002:00000170       __imp_?setName@QWidget@@UAEXPBD@Z 10005170     qt-mt323:qt-mt323.dll
 0002:00000174       __imp_?rect@QWidget@@QBE?AVQRect@@XZ 10005174     qt-mt323:qt-mt323.dll
 0002:00000178       __imp_?closeEvent@QWidget@@MAEXPAVQCloseEvent@@@Z 10005178     qt-mt323:qt-mt323.dll
 0002:0000017c       __imp_??1?$QPtrList@VQDockWindow@@@@UAE@XZ 1000517c     qt-mt323:qt-mt323.dll
 0002:00000180       __imp_??0QCursor@@QAE@H@Z  10005180     qt-mt323:qt-mt323.dll
 0002:00000184       __imp_??1QCursor@@QAE@XZ   10005184     qt-mt323:qt-mt323.dll
 0002:00000188       __imp_?adjustSize@QWidget@@UAEXXZ 10005188     qt-mt323:qt-mt323.dll
 0002:0000018c       __imp_?checkConnectArgs@QObject@@MAE_NPBDPBV1@0@Z 1000518c     qt-mt323:qt-mt323.dll
 0002:00000190       __imp_?childEvent@QObject@@MAEXPAVQChildEvent@@@Z 10005190     qt-mt323:qt-mt323.dll
 0002:00000194       __imp_?className@QWidget@@UBEPBDXZ 10005194     qt-mt323:qt-mt323.dll
 0002:00000198       __imp_?clear@?$QPtrList@VQDockWindow@@@@UAEXXZ 10005198     qt-mt323:qt-mt323.dll
 0002:0000019c       __imp_?close@QWidget@@UAE_N_N@Z 1000519c     qt-mt323:qt-mt323.dll
 0002:000001a0       __imp_?cmd@QPaintDevice@@MAE_NHPAVQPainter@@PATQPDevCmdParam@@@Z 100051a0     qt-mt323:qt-mt323.dll
 0002:000001a4       __imp_?connectNotify@QObject@@MAEXPBD@Z 100051a4     qt-mt323:qt-mt323.dll
 0002:000001a8       __imp_?contextMenuEvent@QWidget@@MAEXPAVQContextMenuEvent@@@Z 100051a8     qt-mt323:qt-mt323.dll
 0002:000001ac       __imp_?count@?$QPtrList@VQDockWindow@@@@UBEIXZ 100051ac     qt-mt323:qt-mt323.dll
 0002:000001b0       __imp_?create@QWidget@@MAEXPAUHWND__@@_N1@Z 100051b0     qt-mt323:qt-mt323.dll
 0002:000001b4       __imp_?customEvent@QObject@@MAEXPAVQCustomEvent@@@Z 100051b4     qt-mt323:qt-mt323.dll
 0002:000001b8       __imp_?customWhatsThis@QWidget@@UBE_NXZ 100051b8     qt-mt323:qt-mt323.dll
 0002:000001bc       __imp_?deleteItem@?$QPtrList@VQDockWindow@@@@EAEXPAX@Z 100051bc     qt-mt323:qt-mt323.dll
 0002:000001c0       __imp_?destroy@QWidget@@MAEX_N0@Z 100051c0     qt-mt323:qt-mt323.dll
 0002:000001c4       __imp_?disconnectNotify@QObject@@MAEXPBD@Z 100051c4     qt-mt323:qt-mt323.dll
 0002:000001c8       __imp_?dragEnterEvent@QWidget@@MAEXPAVQDragEnterEvent@@@Z 100051c8     qt-mt323:qt-mt323.dll
 0002:000001cc       __imp_?dragLeaveEvent@QWidget@@MAEXPAVQDragLeaveEvent@@@Z 100051cc     qt-mt323:qt-mt323.dll
 0002:000001d0       __imp_?dragMoveEvent@QWidget@@MAEXPAVQDragMoveEvent@@@Z 100051d0     qt-mt323:qt-mt323.dll
 0002:000001d4       __imp_?dropEvent@QWidget@@MAEXPAVQDropEvent@@@Z 100051d4     qt-mt323:qt-mt323.dll
 0002:000001d8       __imp_?enabledChange@QWidget@@MAEX_N@Z 100051d8     qt-mt323:qt-mt323.dll
 0002:000001dc       __imp_?enterEvent@QWidget@@MAEXPAVQEvent@@@Z 100051dc     qt-mt323:qt-mt323.dll
 0002:000001e0       __imp_?event@QWidget@@MAE_NPAVQEvent@@@Z 100051e0     qt-mt323:qt-mt323.dll
 0002:000001e4       __imp_?eventFilter@QObject@@UAE_NPAV1@PAVQEvent@@@Z 100051e4     qt-mt323:qt-mt323.dll
 0002:000001e8       __imp_?focusInEvent@QWidget@@MAEXPAVQFocusEvent@@@Z 100051e8     qt-mt323:qt-mt323.dll
 0002:000001ec       __imp_?focusNextPrevChild@QWidget@@MAE_N_N@Z 100051ec     qt-mt323:qt-mt323.dll
 0002:000001f0       __imp_?focusOutEvent@QWidget@@MAEXPAVQFocusEvent@@@Z 100051f0     qt-mt323:qt-mt323.dll
 0002:000001f4       __imp_?fontChange@QWidget@@MAEXABVQFont@@@Z 100051f4     qt-mt323:qt-mt323.dll
 0002:000001f8       __imp_?fontInf@QPaintDevice@@MBEHPAVQFont@@H@Z 100051f8     qt-mt323:qt-mt323.dll
 0002:000001fc       __imp_?fontMet@QPaintDevice@@MBEHPAVQFont@@HPBDH@Z 100051fc     qt-mt323:qt-mt323.dll
 0002:00000200       __imp_?handle@QPaintDevice@@UBEPAUHDC__@@XZ 10005200     qt-mt323:qt-mt323.dll
 0002:00000204       __imp_?heightForWidth@QWidget@@UBEHH@Z 10005204     qt-mt323:qt-mt323.dll
 0002:00000208       __imp_?hide@QWidget@@UAEXXZ 10005208     qt-mt323:qt-mt323.dll
 0002:0000020c       __imp_?hideEvent@QWidget@@MAEXPAVQHideEvent@@@Z 1000520c     qt-mt323:qt-mt323.dll
 0002:00000210       __imp_?imComposeEvent@QWidget@@MAEXPAVQIMEvent@@@Z 10005210     qt-mt323:qt-mt323.dll
 0002:00000214       __imp_?imEndEvent@QWidget@@MAEXPAVQIMEvent@@@Z 10005214     qt-mt323:qt-mt323.dll
 0002:00000218       __imp_?imStartEvent@QWidget@@MAEXPAVQIMEvent@@@Z 10005218     qt-mt323:qt-mt323.dll
 0002:0000021c       __imp_?insertChild@QObject@@UAEXPAV1@@Z 1000521c     qt-mt323:qt-mt323.dll
 0002:00000220       __imp_?keyPressEvent@QWidget@@MAEXPAVQKeyEvent@@@Z 10005220     qt-mt323:qt-mt323.dll
 0002:00000224       __imp_?keyReleaseEvent@QWidget@@MAEXPAVQKeyEvent@@@Z 10005224     qt-mt323:qt-mt323.dll
 0002:00000228       __imp_?leaveEvent@QWidget@@MAEXPAVQEvent@@@Z 10005228     qt-mt323:qt-mt323.dll
 0002:0000022c       __imp_?metaObject@QWidget@@UBEPAVQMetaObject@@XZ 1000522c     qt-mt323:qt-mt323.dll
 0002:00000230       __imp_?metric@QWidget@@MBEHH@Z 10005230     qt-mt323:qt-mt323.dll
 0002:00000234       __imp_?minimumSizeHint@QWidget@@UBE?AVQSize@@XZ 10005234     qt-mt323:qt-mt323.dll
 0002:00000238       __imp_?mouseDoubleClickEvent@QWidget@@MAEXPAVQMouseEvent@@@Z 10005238     qt-mt323:qt-mt323.dll
 0002:0000023c       __imp_?mouseMoveEvent@QWidget@@MAEXPAVQMouseEvent@@@Z 1000523c     qt-mt323:qt-mt323.dll
 0002:00000240       __imp_?mousePressEvent@QWidget@@MAEXPAVQMouseEvent@@@Z 10005240     qt-mt323:qt-mt323.dll
 0002:00000244       __imp_?mouseReleaseEvent@QWidget@@MAEXPAVQMouseEvent@@@Z 10005244     qt-mt323:qt-mt323.dll
 0002:00000248       __imp_?move@QWidget@@UAEXHH@Z 10005248     qt-mt323:qt-mt323.dll
 0002:0000024c       __imp_?moveEvent@QWidget@@MAEXPAVQMoveEvent@@@Z 1000524c     qt-mt323:qt-mt323.dll
 0002:00000250       __imp_?paintEvent@QWidget@@MAEXPAVQPaintEvent@@@Z 10005250     qt-mt323:qt-mt323.dll
 0002:00000254       __imp_?paletteChange@QWidget@@MAEXABVQPalette@@@Z 10005254     qt-mt323:qt-mt323.dll
 0002:00000258       __imp_?polish@QWidget@@UAEXXZ 10005258     qt-mt323:qt-mt323.dll
 0002:0000025c       __imp_?property@QObject@@UBE?AVQVariant@@PBD@Z 1000525c     qt-mt323:qt-mt323.dll
 0002:00000260       __imp_?qt_cast@QWidget@@UAEPAXPBD@Z 10005260     qt-mt323:qt-mt323.dll
 0002:00000264       __imp_?qt_emit@QWidget@@UAE_NHPAUQUObject@@@Z 10005264     qt-mt323:qt-mt323.dll
 0002:00000268       __imp_?qt_invoke@QWidget@@UAE_NHPAUQUObject@@@Z 10005268     qt-mt323:qt-mt323.dll
 0002:0000026c       __imp_?qt_property@QWidget@@UAE_NHHPAVQVariant@@@Z 1000526c     qt-mt323:qt-mt323.dll
 0002:00000270       __imp_?removeChild@QObject@@UAEXPAV1@@Z 10005270     qt-mt323:qt-mt323.dll
 0002:00000274       __imp_?reparent@QWidget@@UAEXPAV1@IABVQPoint@@_N@Z 10005274     qt-mt323:qt-mt323.dll
 0002:00000278       __imp_?resize@QWidget@@UAEXHH@Z 10005278     qt-mt323:qt-mt323.dll
 0002:0000027c       __imp_?resizeEvent@QWidget@@MAEXPAVQResizeEvent@@@Z 1000527c     qt-mt323:qt-mt323.dll
 0002:00000280       __imp_?resolution@QPaintDevice@@UBEHXZ 10005280     qt-mt323:qt-mt323.dll
 0002:00000284       __imp_?setAcceptDrops@QWidget@@UAEX_N@Z 10005284     qt-mt323:qt-mt323.dll
 0002:00000288       __imp_?setActiveWindow@QWidget@@UAEXXZ 10005288     qt-mt323:qt-mt323.dll
 0002:0000028c       __imp_?setAutoMask@QWidget@@UAEX_N@Z 1000528c     qt-mt323:qt-mt323.dll
 0002:00000290       __imp_?setBackgroundColor@QWidget@@UAEXABVQColor@@@Z 10005290     qt-mt323:qt-mt323.dll
 0002:00000294       __imp_?setBackgroundMode@QWidget@@UAEXW4BackgroundMode@Qt@@@Z 10005294     qt-mt323:qt-mt323.dll
 0002:00000298       __imp_?setBackgroundOrigin@QWidget@@UAEXW4BackgroundOrigin@1@@Z 10005298     qt-mt323:qt-mt323.dll
 0002:0000029c       __imp_?setBackgroundPixmap@QWidget@@UAEXABVQPixmap@@@Z 1000529c     qt-mt323:qt-mt323.dll
 0002:000002a0       __imp_?setCaption@QWidget@@UAEXABVQString@@@Z 100052a0     qt-mt323:qt-mt323.dll
 0002:000002a4       __imp_?setCursor@QWidget@@UAEXABVQCursor@@@Z 100052a4     qt-mt323:qt-mt323.dll
 0002:000002a8       __imp_?setEnabled@QWidget@@UAEX_N@Z 100052a8     qt-mt323:qt-mt323.dll
 0002:000002ac       __imp_?setEraseColor@QWidget@@UAEXABVQColor@@@Z 100052ac     qt-mt323:qt-mt323.dll
 0002:000002b0       __imp_?setErasePixmap@QWidget@@UAEXABVQPixmap@@@Z 100052b0     qt-mt323:qt-mt323.dll
 0002:000002b4       __imp_?setFocus@QWidget@@UAEXXZ 100052b4     qt-mt323:qt-mt323.dll
 0002:000002b8       __imp_?setFocusPolicy@QWidget@@UAEXW4FocusPolicy@1@@Z 100052b8     qt-mt323:qt-mt323.dll
 0002:000002bc       __imp_?setFocusProxy@QWidget@@UAEXPAV1@@Z 100052bc     qt-mt323:qt-mt323.dll
 0002:000002c0       __imp_?setFont@QWidget@@UAEXABVQFont@@@Z 100052c0     qt-mt323:qt-mt323.dll
 0002:000002c4       __imp_?setGeometry@QWidget@@UAEXABVQRect@@@Z 100052c4     qt-mt323:qt-mt323.dll
 0002:000002c8       __imp_?setGeometry@QWidget@@UAEXHHHH@Z 100052c8     qt-mt323:qt-mt323.dll
 0002:000002cc       __imp_?setIcon@QWidget@@UAEXABVQPixmap@@@Z 100052cc     qt-mt323:qt-mt323.dll
 0002:000002d0       __imp_?setIconText@QWidget@@UAEXABVQString@@@Z 100052d0     qt-mt323:qt-mt323.dll
 0002:000002d4       __imp_?setKeyCompression@QWidget@@MAEX_N@Z 100052d4     qt-mt323:qt-mt323.dll
 0002:000002d8       __imp_?setMask@QWidget@@UAEXABVQBitmap@@@Z 100052d8     qt-mt323:qt-mt323.dll
 0002:000002dc       __imp_?setMask@QWidget@@UAEXABVQRegion@@@Z 100052dc     qt-mt323:qt-mt323.dll
 0002:000002e0       __imp_?setMaximumSize@QWidget@@UAEXHH@Z 100052e0     qt-mt323:qt-mt323.dll
 0002:000002e4       __imp_?setMicroFocusHint@QWidget@@MAEXHHHH_NPAVQFont@@@Z 100052e4     qt-mt323:qt-mt323.dll
 0002:000002e8       __imp_?setMinimumSize@QWidget@@UAEXHH@Z 100052e8     qt-mt323:qt-mt323.dll
 0002:000002ec       __imp_?setMouseTracking@QWidget@@UAEX_N@Z 100052ec     qt-mt323:qt-mt323.dll
 0002:000002f0       __imp_?setPalette@QWidget@@UAEXABVQPalette@@@Z 100052f0     qt-mt323:qt-mt323.dll
 0002:000002f4       __imp_?setPaletteBackgroundColor@QWidget@@UAEXABVQColor@@@Z 100052f4     qt-mt323:qt-mt323.dll
 0002:000002f8       __imp_?setPaletteBackgroundPixmap@QWidget@@UAEXABVQPixmap@@@Z 100052f8     qt-mt323:qt-mt323.dll
 0002:000002fc       __imp_?setProperty@QObject@@UAE_NPBDABVQVariant@@@Z 100052fc     qt-mt323:qt-mt323.dll
 0002:00000300       __imp_?setResolution@QPaintDevice@@UAEXH@Z 10005300     qt-mt323:qt-mt323.dll
 0002:00000304       __imp_?setSizeIncrement@QWidget@@UAEXHH@Z 10005304     qt-mt323:qt-mt323.dll
 0002:00000308       __imp_?setSizePolicy@QWidget@@UAEXVQSizePolicy@@@Z 10005308     qt-mt323:qt-mt323.dll
 0002:0000030c       __imp_?setUpdatesEnabled@QWidget@@UAEX_N@Z 1000530c     qt-mt323:qt-mt323.dll
 0002:00000310       __imp_?setWFlags@QWidget@@MAEXI@Z 10005310     qt-mt323:qt-mt323.dll
 0002:00000314       __imp_?setWState@QWidget@@MAEXI@Z 10005314     qt-mt323:qt-mt323.dll
 0002:00000318       __imp_?show@QWidget@@UAEXXZ 10005318     qt-mt323:qt-mt323.dll
 0002:0000031c       __imp_?showEvent@QWidget@@MAEXPAVQShowEvent@@@Z 1000531c     qt-mt323:qt-mt323.dll
 0002:00000320       __imp_?showMaximized@QWidget@@UAEXXZ 10005320     qt-mt323:qt-mt323.dll
 0002:00000324       __imp_?showMinimized@QWidget@@UAEXXZ 10005324     qt-mt323:qt-mt323.dll
 0002:00000328       __imp_?showNormal@QWidget@@UAEXXZ 10005328     qt-mt323:qt-mt323.dll
 0002:0000032c       __imp_?sizeHint@QWidget@@UBE?AVQSize@@XZ 1000532c     qt-mt323:qt-mt323.dll
 0002:00000330       __imp_?sizePolicy@QWidget@@UBE?AVQSizePolicy@@XZ 10005330     qt-mt323:qt-mt323.dll
 0002:00000334       __imp_?styleChange@QWidget@@MAEXAAVQStyle@@@Z 10005334     qt-mt323:qt-mt323.dll
 0002:00000338       __imp_?tabletEvent@QWidget@@MAEXPAVQTabletEvent@@@Z 10005338     qt-mt323:qt-mt323.dll
 0002:0000033c       __imp_?timerEvent@QObject@@MAEXPAVQTimerEvent@@@Z 1000533c     qt-mt323:qt-mt323.dll
 0002:00000340       __imp_?unsetCursor@QWidget@@UAEXXZ 10005340     qt-mt323:qt-mt323.dll
 0002:00000344       __imp_?updateMask@QWidget@@MAEXXZ 10005344     qt-mt323:qt-mt323.dll
 0002:00000348       __imp_?wheelEvent@QWidget@@MAEXPAVQWheelEvent@@@Z 10005348     qt-mt323:qt-mt323.dll
 0002:0000034c       __imp_?winEvent@QWidget@@MAE_NPAUtagMSG@@@Z 1000534c     qt-mt323:qt-mt323.dll
 0002:00000350       __imp_?windowActivationChange@QWidget@@MAEX_N@Z 10005350     qt-mt323:qt-mt323.dll
 0002:00000354       __imp_??_7?$QPtrList@VQDockWindow@@@@6B@ 10005354     qt-mt323:qt-mt323.dll
 0002:00000358       __imp_??0QPixmap@@QAE@QAPBD@Z 10005358     qt-mt323:qt-mt323.dll
 0002:0000035c       __imp_?qstrcmp@@YAHPBD0@Z  1000535c     qt-mt323:qt-mt323.dll
 0002:00000360       __imp_?fromLatin1@QString@@SA?AV1@PBDH@Z 10005360     qt-mt323:qt-mt323.dll
 0002:00000364       __imp_?receivers@QObject@@IBEPAVQConnectionList@@H@Z 10005364     qt-mt323:qt-mt323.dll
 0002:00000368       __imp_?activate_signal@QObject@@IAEXPAVQConnectionList@@PAUQUObject@@@Z 10005368     qt-mt323:qt-mt323.dll
 0002:0000036c       __imp_?staticMetaObject@QWidget@@SAPAVQMetaObject@@XZ 1000536c     qt-mt323:qt-mt323.dll
 0002:00000370       __imp_?new_metaobject@QMetaObject@@SAPAV1@PBDPAV1@QBUQMetaData@@H2HQBVQMetaProperty@@HQBUQMetaEnum@@HQBUQClassInfo@@H@Z 10005370     qt-mt323:qt-mt323.dll
 0002:00000374       __imp_??1QDomDocument@@UAE@XZ 10005374     qt-mt323:qt-mt323.dll
 0002:00000378       __imp_??1QMetaObjectCleanUp@@QAE@XZ 10005378     qt-mt323:qt-mt323.dll
 0002:0000037c       __imp_?setMetaObject@QMetaObjectCleanUp@@QAEXAAPAVQMetaObject@@@Z 1000537c     qt-mt323:qt-mt323.dll
 0002:00000380       __imp_?translate@QApplication@@QBE?AVQString@@PBD00W4Encoding@1@@Z 10005380     qt-mt323:qt-mt323.dll
 0002:00000384       __imp_??0QUObject@@QAE@XZ  10005384     qt-mt323:qt-mt323.dll
 0002:00000388       __imp_??1QUObject@@QAE@XZ  10005388     qt-mt323:qt-mt323.dll
 0002:0000038c       __imp_?set@QUType_QString@@QAEXPAUQUObject@@ABVQString@@@Z 1000538c     qt-mt323:qt-mt323.dll
 0002:00000390       __imp_?qApp@@3PAVQApplication@@A 10005390     qt-mt323:qt-mt323.dll
 0002:00000394       __imp_?static_QUType_ptr@@3UQUType_ptr@@A 10005394     qt-mt323:qt-mt323.dll
 0002:00000398       __imp_?static_QUType_int@@3UQUType_int@@A 10005398     qt-mt323:qt-mt323.dll
 0002:0000039c       __imp_?static_QUType_QString@@3UQUType_QString@@A 1000539c     qt-mt323:qt-mt323.dll
 0002:000003a0       __imp_?static_QUType_varptr@@3UQUType_varptr@@A 100053a0     qt-mt323:qt-mt323.dll
 0002:000003a4       __imp_?resize@QWidget@@QAEXABVQSize@@@Z 100053a4     qt-mt323:qt-mt323.dll
 0002:000003a8       __imp_?setFrameShape@QFrame@@QAEXW4Shape@1@@Z 100053a8     qt-mt323:qt-mt323.dll
 0002:000003ac       __imp_?setFrameShadow@QFrame@@QAEXW4Shadow@1@@Z 100053ac     qt-mt323:qt-mt323.dll
 0002:000003b0       __imp_??0QLabel@@QAE@PAVQWidget@@PBDI@Z 100053b0     qt-mt323:qt-mt323.dll
 0002:000003b4       __imp_??1QLabel@@UAE@XZ    100053b4     qt-mt323:qt-mt323.dll
 0002:000003b8       __imp_??0QIconView@@QAE@PAVQWidget@@PBDI@Z 100053b8     qt-mt323:qt-mt323.dll
 0002:000003bc       __imp_??1QIconView@@UAE@XZ 100053bc     qt-mt323:qt-mt323.dll
 0002:000003c0       __imp_?addWidget@QBoxLayout@@QAEXPAVQWidget@@HH@Z 100053c0     qt-mt323:qt-mt323.dll
 0002:000003c4       __imp_??0QVBoxLayout@@QAE@PAVQWidget@@HHPBD@Z 100053c4     qt-mt323:qt-mt323.dll
 0002:000003c8       __imp_??1QVBoxLayout@@UAE@XZ 100053c8     qt-mt323:qt-mt323.dll
 0002:000003cc       __imp_?addChild@QScrollView@@UAEXPAVQWidget@@HH@Z 100053cc     qt-mt323:qt-mt323.dll
 0002:000003d0       __imp_?addItem@QBoxLayout@@UAEXPAVQLayoutItem@@@Z 100053d0     qt-mt323:qt-mt323.dll
 0002:000003d4       __imp_?adjustItems@QIconView@@MAEXXZ 100053d4     qt-mt323:qt-mt323.dll
 0002:000003d8       __imp_?arrangeItemsInGrid@QIconView@@UAEXABVQSize@@_N@Z 100053d8     qt-mt323:qt-mt323.dll
 0002:000003dc       __imp_?arrangeItemsInGrid@QIconView@@UAEX_N@Z 100053dc     qt-mt323:qt-mt323.dll
 0002:000003e0       __imp_?childEvent@QLayout@@MAEXPAVQChildEvent@@@Z 100053e0     qt-mt323:qt-mt323.dll
 0002:000003e4       __imp_?className@QIconView@@UBEPBDXZ 100053e4     qt-mt323:qt-mt323.dll
 0002:000003e8       __imp_?className@QLabel@@UBEPBDXZ 100053e8     qt-mt323:qt-mt323.dll
 0002:000003ec       __imp_?className@QVBoxLayout@@UBEPBDXZ 100053ec     qt-mt323:qt-mt323.dll
 0002:000003f0       __imp_?clear@QIconView@@UAEXXZ 100053f0     qt-mt323:qt-mt323.dll
 0002:000003f4       __imp_?clearSelection@QIconView@@UAEXXZ 100053f4     qt-mt323:qt-mt323.dll
 0002:000003f8       __imp_?contentsContextMenuEvent@QIconView@@MAEXPAVQContextMenuEvent@@@Z 100053f8     qt-mt323:qt-mt323.dll
 0002:000003fc       __imp_?contentsDragEnterEvent@QIconView@@MAEXPAVQDragEnterEvent@@@Z 100053fc     qt-mt323:qt-mt323.dll
 0002:00000400       __imp_?contentsDragLeaveEvent@QIconView@@MAEXPAVQDragLeaveEvent@@@Z 10005400     qt-mt323:qt-mt323.dll
 0002:00000404       __imp_?contentsDragMoveEvent@QIconView@@MAEXPAVQDragMoveEvent@@@Z 10005404     qt-mt323:qt-mt323.dll
 0002:00000408       __imp_?contentsDropEvent@QIconView@@MAEXPAVQDropEvent@@@Z 10005408     qt-mt323:qt-mt323.dll
 0002:0000040c       __imp_?contentsMouseDoubleClickEvent@QIconView@@MAEXPAVQMouseEvent@@@Z 1000540c     qt-mt323:qt-mt323.dll
 0002:00000410       __imp_?contentsMouseMoveEvent@QIconView@@MAEXPAVQMouseEvent@@@Z 10005410     qt-mt323:qt-mt323.dll
 0002:00000414       __imp_?contentsMousePressEvent@QIconView@@MAEXPAVQMouseEvent@@@Z 10005414     qt-mt323:qt-mt323.dll
 0002:00000418       __imp_?contentsMouseReleaseEvent@QIconView@@MAEXPAVQMouseEvent@@@Z 10005418     qt-mt323:qt-mt323.dll
 0002:0000041c       __imp_?contentsWheelEvent@QScrollView@@MAEXPAVQWheelEvent@@@Z 1000541c     qt-mt323:qt-mt323.dll
 0002:00000420       __imp_?contextMenuEvent@QScrollView@@MAEXPAVQContextMenuEvent@@@Z 10005420     qt-mt323:qt-mt323.dll
 0002:00000424       __imp_?doAutoScroll@QIconView@@MAEXXZ 10005424     qt-mt323:qt-mt323.dll
 0002:00000428       __imp_?dragObject@QIconView@@MAEPAVQDragObject@@XZ 10005428     qt-mt323:qt-mt323.dll
 0002:0000042c       __imp_?drawBackground@QIconView@@MAEXPAVQPainter@@ABVQRect@@@Z 1000542c     qt-mt323:qt-mt323.dll
 0002:00000430       __imp_?drawContents@QIconView@@EAEXPAVQPainter@@@Z 10005430     qt-mt323:qt-mt323.dll
 0002:00000434       __imp_?drawContents@QIconView@@MAEXPAVQPainter@@HHHH@Z 10005434     qt-mt323:qt-mt323.dll
 0002:00000438       __imp_?drawContents@QLabel@@MAEXPAVQPainter@@@Z 10005438     qt-mt323:qt-mt323.dll
 0002:0000043c       __imp_?drawContentsOffset@QScrollView@@MAEXPAVQPainter@@HHHHHH@Z 1000543c     qt-mt323:qt-mt323.dll
 0002:00000440       __imp_?drawDragShapes@QIconView@@EAEXABVQPoint@@@Z 10005440     qt-mt323:qt-mt323.dll
 0002:00000444       __imp_?drawFrame@QFrame@@MAEXPAVQPainter@@@Z 10005444     qt-mt323:qt-mt323.dll
 0002:00000448       __imp_?drawRubber@QIconView@@MAEXPAVQPainter@@@Z 10005448     qt-mt323:qt-mt323.dll
 0002:0000044c       __imp_?enterEvent@QIconView@@MAEXPAVQEvent@@@Z 1000544c     qt-mt323:qt-mt323.dll
 0002:00000450       __imp_?event@QObject@@UAE_NPAVQEvent@@@Z 10005450     qt-mt323:qt-mt323.dll
 0002:00000454       __imp_?eventFilter@QIconView@@UAE_NPAVQObject@@PAVQEvent@@@Z 10005454     qt-mt323:qt-mt323.dll
 0002:00000458       __imp_?eventFilter@QLayout@@MAE_NPAVQObject@@PAVQEvent@@@Z 10005458     qt-mt323:qt-mt323.dll
 0002:0000045c       __imp_?expanding@QBoxLayout@@UBE?AW4ExpandData@QSizePolicy@@XZ 1000545c     qt-mt323:qt-mt323.dll
 0002:00000460       __imp_?focusInEvent@QIconView@@MAEXPAVQFocusEvent@@@Z 10005460     qt-mt323:qt-mt323.dll
 0002:00000464       __imp_?focusNextPrevChild@QScrollView@@MAE_N_N@Z 10005464     qt-mt323:qt-mt323.dll
 0002:00000468       __imp_?focusOutEvent@QIconView@@MAEXPAVQFocusEvent@@@Z 10005468     qt-mt323:qt-mt323.dll
 0002:0000046c       __imp_?fontChange@QLabel@@MAEXABVQFont@@@Z 1000546c     qt-mt323:qt-mt323.dll
 0002:00000470       __imp_?fontChange@QScrollView@@MAEXABVQFont@@@Z 10005470     qt-mt323:qt-mt323.dll
 0002:00000474       __imp_?frameChanged@QFrame@@MAEXXZ 10005474     qt-mt323:qt-mt323.dll
 0002:00000478       __imp_?frameChanged@QScrollView@@MAEXXZ 10005478     qt-mt323:qt-mt323.dll
 0002:0000047c       __imp_?geometry@QLayout@@UBE?AVQRect@@XZ 1000547c     qt-mt323:qt-mt323.dll
 0002:00000480       __imp_?hasHeightForWidth@QBoxLayout@@UBE_NXZ 10005480     qt-mt323:qt-mt323.dll
 0002:00000484       __imp_?heightForWidth@QBoxLayout@@UBEHH@Z 10005484     qt-mt323:qt-mt323.dll
 0002:00000488       __imp_?heightForWidth@QLabel@@UBEHH@Z 10005488     qt-mt323:qt-mt323.dll
 0002:0000048c       __imp_?initDragEnter@QIconView@@EAEXPAVQDropEvent@@@Z 1000548c     qt-mt323:qt-mt323.dll
 0002:00000490       __imp_?insertInGrid@QIconView@@MAEXPAVQIconViewItem@@@Z 10005490     qt-mt323:qt-mt323.dll
 0002:00000494       __imp_?insertItem@QIconView@@UAEXPAVQIconViewItem@@0@Z 10005494     qt-mt323:qt-mt323.dll
 0002:00000498       __imp_?invalidate@QBoxLayout@@UAEXXZ 10005498     qt-mt323:qt-mt323.dll
 0002:0000049c       __imp_?invertSelection@QIconView@@UAEXXZ 1000549c     qt-mt323:qt-mt323.dll
 0002:000004a0       __imp_?isEmpty@QLayout@@UBE_NXZ 100054a0     qt-mt323:qt-mt323.dll
 0002:000004a4       __imp_?iterator@QBoxLayout@@UAE?AVQLayoutIterator@@XZ 100054a4     qt-mt323:qt-mt323.dll
 0002:000004a8       __imp_?keyPressEvent@QIconView@@MAEXPAVQKeyEvent@@@Z 100054a8     qt-mt323:qt-mt323.dll
 0002:000004ac       __imp_?layout@QLayout@@UAEPAV1@XZ 100054ac     qt-mt323:qt-mt323.dll
 0002:000004b0       __imp_?maximumSize@QBoxLayout@@UBE?AVQSize@@XZ 100054b0     qt-mt323:qt-mt323.dll
 0002:000004b4       __imp_?metaObject@QIconView@@UBEPAVQMetaObject@@XZ 100054b4     qt-mt323:qt-mt323.dll
 0002:000004b8       __imp_?metaObject@QLabel@@UBEPAVQMetaObject@@XZ 100054b8     qt-mt323:qt-mt323.dll
 0002:000004bc       __imp_?metaObject@QVBoxLayout@@UBEPAVQMetaObject@@XZ 100054bc     qt-mt323:qt-mt323.dll
 0002:000004c0       __imp_?minimumSize@QBoxLayout@@UBE?AVQSize@@XZ 100054c0     qt-mt323:qt-mt323.dll
 0002:000004c4       __imp_?minimumSizeHint@QIconView@@UBE?AVQSize@@XZ 100054c4     qt-mt323:qt-mt323.dll
 0002:000004c8       __imp_?minimumSizeHint@QLabel@@UBE?AVQSize@@XZ 100054c8     qt-mt323:qt-mt323.dll
 0002:000004cc       __imp_?mouseDoubleClickEvent@QScrollView@@MAEXPAVQMouseEvent@@@Z 100054cc     qt-mt323:qt-mt323.dll
 0002:000004d0       __imp_?mouseMoveEvent@QScrollView@@MAEXPAVQMouseEvent@@@Z 100054d0     qt-mt323:qt-mt323.dll
 0002:000004d4       __imp_?mousePressEvent@QScrollView@@MAEXPAVQMouseEvent@@@Z 100054d4     qt-mt323:qt-mt323.dll
 0002:000004d8       __imp_?mouseReleaseEvent@QScrollView@@MAEXPAVQMouseEvent@@@Z 100054d8     qt-mt323:qt-mt323.dll
 0002:000004dc       __imp_?moveChild@QScrollView@@UAEXPAVQWidget@@HH@Z 100054dc     qt-mt323:qt-mt323.dll
 0002:000004e0       __imp_?paintEvent@QFrame@@MAEXPAVQPaintEvent@@@Z 100054e0     qt-mt323:qt-mt323.dll
 0002:000004e4       __imp_?qt_cast@QIconView@@UAEPAXPBD@Z 100054e4     qt-mt323:qt-mt323.dll
 0002:000004e8       __imp_?qt_cast@QLabel@@UAEPAXPBD@Z 100054e8     qt-mt323:qt-mt323.dll
 0002:000004ec       __imp_?qt_cast@QVBoxLayout@@UAEPAXPBD@Z 100054ec     qt-mt323:qt-mt323.dll
 0002:000004f0       __imp_?qt_emit@QIconView@@UAE_NHPAUQUObject@@@Z 100054f0     qt-mt323:qt-mt323.dll
 0002:000004f4       __imp_?qt_emit@QLabel@@UAE_NHPAUQUObject@@@Z 100054f4     qt-mt323:qt-mt323.dll
 0002:000004f8       __imp_?qt_emit@QVBoxLayout@@UAE_NHPAUQUObject@@@Z 100054f8     qt-mt323:qt-mt323.dll
 0002:000004fc       __imp_?qt_invoke@QIconView@@UAE_NHPAUQUObject@@@Z 100054fc     qt-mt323:qt-mt323.dll
 0002:00000500       __imp_?qt_invoke@QLabel@@UAE_NHPAUQUObject@@@Z 10005500     qt-mt323:qt-mt323.dll
 0002:00000504       __imp_?qt_invoke@QVBoxLayout@@UAE_NHPAUQUObject@@@Z 10005504     qt-mt323:qt-mt323.dll
 0002:00000508       __imp_?qt_property@QIconView@@UAE_NHHPAVQVariant@@@Z 10005508     qt-mt323:qt-mt323.dll
 0002:0000050c       __imp_?qt_property@QLabel@@UAE_NHHPAVQVariant@@@Z 1000550c     qt-mt323:qt-mt323.dll
 0002:00000510       __imp_?qt_property@QVBoxLayout@@UAE_NHHPAVQVariant@@@Z 10005510     qt-mt323:qt-mt323.dll
 0002:00000514       __imp_?removeChild@QScrollView@@UAEXPAVQObject@@@Z 10005514     qt-mt323:qt-mt323.dll
 0002:00000518       __imp_?repaintItem@QIconView@@UAEXPAVQIconViewItem@@@Z 10005518     qt-mt323:qt-mt323.dll
 0002:0000051c       __imp_?resize@QScrollView@@UAEXHH@Z 1000551c     qt-mt323:qt-mt323.dll
 0002:00000520       __imp_?resizeContents@QScrollView@@UAEXHH@Z 10005520     qt-mt323:qt-mt323.dll
 0002:00000524       __imp_?resizeEvent@QIconView@@MAEXPAVQResizeEvent@@@Z 10005524     qt-mt323:qt-mt323.dll
 0002:00000528       __imp_?resizeEvent@QLabel@@MAEXPAVQResizeEvent@@@Z 10005528     qt-mt323:qt-mt323.dll
 0002:0000052c       __imp_?selectAll@QIconView@@UAEX_N@Z 1000552c     qt-mt323:qt-mt323.dll
 0002:00000530       __imp_?setAlignment@QLabel@@UAEXH@Z 10005530     qt-mt323:qt-mt323.dll
 0002:00000534       __imp_?setAlignment@QLayoutItem@@UAEXH@Z 10005534     qt-mt323:qt-mt323.dll
 0002:00000538       __imp_?setArrangement@QIconView@@UAEXW4Arrangement@1@@Z 10005538     qt-mt323:qt-mt323.dll
 0002:0000053c       __imp_?setAutoAdd@QLayout@@UAEX_N@Z 1000553c     qt-mt323:qt-mt323.dll
 0002:00000540       __imp_?setAutoArrange@QIconView@@UAEX_N@Z 10005540     qt-mt323:qt-mt323.dll
 0002:00000544       __imp_?setAutoResize@QLabel@@UAEX_N@Z 10005544     qt-mt323:qt-mt323.dll
 0002:00000548       __imp_?setBuddy@QLabel@@UAEXPAVQWidget@@@Z 10005548     qt-mt323:qt-mt323.dll
 0002:0000054c       __imp_?setContentsPos@QIconView@@UAEXHH@Z 1000554c     qt-mt323:qt-mt323.dll
 0002:00000550       __imp_?setCornerWidget@QScrollView@@UAEXPAVQWidget@@@Z 10005550     qt-mt323:qt-mt323.dll
 0002:00000554       __imp_?setCurrentItem@QIconView@@UAEXPAVQIconViewItem@@@Z 10005554     qt-mt323:qt-mt323.dll
 0002:00000558       __imp_?setDragAutoScroll@QScrollView@@UAEX_N@Z 10005558     qt-mt323:qt-mt323.dll
 0002:0000055c       __imp_?setEnabled@QScrollView@@UAEX_N@Z 1000555c     qt-mt323:qt-mt323.dll
 0002:00000560       __imp_?setFont@QIconView@@UAEXABVQFont@@@Z 10005560     qt-mt323:qt-mt323.dll
 0002:00000564       __imp_?setFont@QLabel@@UAEXABVQFont@@@Z 10005564     qt-mt323:qt-mt323.dll
 0002:00000568       __imp_?setFrameRect@QFrame@@UAEXABVQRect@@@Z 10005568     qt-mt323:qt-mt323.dll
 0002:0000056c       __imp_?setFrameStyle@QFrame@@UAEXH@Z 1000556c     qt-mt323:qt-mt323.dll
 0002:00000570       __imp_?setGeometry@QBoxLayout@@UAEXABVQRect@@@Z 10005570     qt-mt323:qt-mt323.dll
 0002:00000574       __imp_?setGridX@QIconView@@UAEXH@Z 10005574     qt-mt323:qt-mt323.dll
 0002:00000578       __imp_?setGridY@QIconView@@UAEXH@Z 10005578     qt-mt323:qt-mt323.dll
 0002:0000057c       __imp_?setHBarGeometry@QScrollView@@MAEXAAVQScrollBar@@HHHH@Z 1000557c     qt-mt323:qt-mt323.dll
 0002:00000580       __imp_?setHScrollBarMode@QScrollView@@UAEXW4ScrollBarMode@1@@Z 10005580     qt-mt323:qt-mt323.dll
 0002:00000584       __imp_?setItemTextBackground@QIconView@@UAEXABVQBrush@@@Z 10005584     qt-mt323:qt-mt323.dll
 0002:00000588       __imp_?setItemTextPos@QIconView@@UAEXW4ItemTextPos@1@@Z 10005588     qt-mt323:qt-mt323.dll
 0002:0000058c       __imp_?setItemsMovable@QIconView@@UAEX_N@Z 1000558c     qt-mt323:qt-mt323.dll
 0002:00000590       __imp_?setLineWidth@QFrame@@UAEXH@Z 10005590     qt-mt323:qt-mt323.dll
 0002:00000594       __imp_?setMargin@QFrame@@UAEXH@Z 10005594     qt-mt323:qt-mt323.dll
 0002:00000598       __imp_?setMargin@QLayout@@UAEXH@Z 10005598     qt-mt323:qt-mt323.dll
 0002:0000059c       __imp_?setMargins@QScrollView@@MAEXHHHH@Z 1000559c     qt-mt323:qt-mt323.dll
 0002:000005a0       __imp_?setMaxItemTextLength@QIconView@@UAEXH@Z 100055a0     qt-mt323:qt-mt323.dll
 0002:000005a4       __imp_?setMaxItemWidth@QIconView@@UAEXH@Z 100055a4     qt-mt323:qt-mt323.dll
 0002:000005a8       __imp_?setMenuBar@QLayout@@UAEXPAVQMenuBar@@@Z 100055a8     qt-mt323:qt-mt323.dll
 0002:000005ac       __imp_?setMidLineWidth@QFrame@@UAEXH@Z 100055ac     qt-mt323:qt-mt323.dll
 0002:000005b0       __imp_?setMovie@QLabel@@UAEXABVQMovie@@@Z 100055b0     qt-mt323:qt-mt323.dll
 0002:000005b4       __imp_?setName@QObject@@UAEXPBD@Z 100055b4     qt-mt323:qt-mt323.dll
 0002:000005b8       __imp_?setNum@QLabel@@UAEXH@Z 100055b8     qt-mt323:qt-mt323.dll
 0002:000005bc       __imp_?setNum@QLabel@@UAEXN@Z 100055bc     qt-mt323:qt-mt323.dll
 0002:000005c0       __imp_?setPalette@QIconView@@UAEXABVQPalette@@@Z 100055c0     qt-mt323:qt-mt323.dll
 0002:000005c4       __imp_?setPicture@QLabel@@UAEXABVQPicture@@@Z 100055c4     qt-mt323:qt-mt323.dll
 0002:000005c8       __imp_?setPixmap@QLabel@@UAEXABVQPixmap@@@Z 100055c8     qt-mt323:qt-mt323.dll
 0002:000005cc       __imp_?setResizeMode@QIconView@@UAEXW4ResizeMode@1@@Z 100055cc     qt-mt323:qt-mt323.dll
 0002:000005d0       __imp_?setResizePolicy@QScrollView@@UAEXW4ResizePolicy@1@@Z 100055d0     qt-mt323:qt-mt323.dll
 0002:000005d4       __imp_?setSelected@QIconView@@UAEXPAVQIconViewItem@@_N1@Z 100055d4     qt-mt323:qt-mt323.dll
 0002:000005d8       __imp_?setSelectionMode@QIconView@@UAEXW4SelectionMode@1@@Z 100055d8     qt-mt323:qt-mt323.dll
 0002:000005dc       __imp_?setShowToolTips@QIconView@@UAEX_N@Z 100055dc     qt-mt323:qt-mt323.dll
 0002:000005e0       __imp_?setSpacing@QIconView@@UAEXH@Z 100055e0     qt-mt323:qt-mt323.dll
 0002:000005e4       __imp_?setSpacing@QLayout@@UAEXH@Z 100055e4     qt-mt323:qt-mt323.dll
 0002:000005e8       __imp_?setText@QLabel@@UAEXABVQString@@@Z 100055e8     qt-mt323:qt-mt323.dll
 0002:000005ec       __imp_?setVBarGeometry@QScrollView@@MAEXAAVQScrollBar@@HHHH@Z 100055ec     qt-mt323:qt-mt323.dll
 0002:000005f0       __imp_?setVScrollBarMode@QScrollView@@UAEXW4ScrollBarMode@1@@Z 100055f0     qt-mt323:qt-mt323.dll
 0002:000005f4       __imp_?setWordWrapIconText@QIconView@@UAEX_N@Z 100055f4     qt-mt323:qt-mt323.dll
 0002:000005f8       __imp_?show@QScrollView@@UAEXXZ 100055f8     qt-mt323:qt-mt323.dll
 0002:000005fc       __imp_?showEvent@QIconView@@UAEXPAVQShowEvent@@@Z 100055fc     qt-mt323:qt-mt323.dll
 0002:00000600       __imp_?sizeHint@QBoxLayout@@UBE?AVQSize@@XZ 10005600     qt-mt323:qt-mt323.dll
 0002:00000604       __imp_?sizeHint@QIconView@@UBE?AVQSize@@XZ 10005604     qt-mt323:qt-mt323.dll
 0002:00000608       __imp_?sizeHint@QLabel@@UBE?AVQSize@@XZ 10005608     qt-mt323:qt-mt323.dll
 0002:0000060c       __imp_?slotUpdate@QIconView@@MAEXXZ 1000560c     qt-mt323:qt-mt323.dll
 0002:00000610       __imp_?sort@QIconView@@UAEX_N@Z 10005610     qt-mt323:qt-mt323.dll
 0002:00000614       __imp_?spacerItem@QLayoutItem@@UAEPAVQSpacerItem@@XZ 10005614     qt-mt323:qt-mt323.dll
 0002:00000618       __imp_?startDrag@QIconView@@MAEXXZ 10005618     qt-mt323:qt-mt323.dll
 0002:0000061c       __imp_?styleChange@QFrame@@MAEXAAVQStyle@@@Z 1000561c     qt-mt323:qt-mt323.dll
 0002:00000620       __imp_?styleChange@QIconView@@MAEXAAVQStyle@@@Z 10005620     qt-mt323:qt-mt323.dll
 0002:00000624       __imp_?takeItem@QIconView@@UAEXPAVQIconViewItem@@@Z 10005624     qt-mt323:qt-mt323.dll
 0002:00000628       __imp_?updateContents@QIconView@@UAEXXZ 10005628     qt-mt323:qt-mt323.dll
 0002:0000062c       __imp_?viewportContextMenuEvent@QScrollView@@MAEXPAVQContextMenuEvent@@@Z 1000562c     qt-mt323:qt-mt323.dll
 0002:00000630       __imp_?viewportDragEnterEvent@QScrollView@@MAEXPAVQDragEnterEvent@@@Z 10005630     qt-mt323:qt-mt323.dll
 0002:00000634       __imp_?viewportDragLeaveEvent@QScrollView@@MAEXPAVQDragLeaveEvent@@@Z 10005634     qt-mt323:qt-mt323.dll
 0002:00000638       __imp_?viewportDragMoveEvent@QScrollView@@MAEXPAVQDragMoveEvent@@@Z 10005638     qt-mt323:qt-mt323.dll
 0002:0000063c       __imp_?viewportDropEvent@QScrollView@@MAEXPAVQDropEvent@@@Z 1000563c     qt-mt323:qt-mt323.dll
 0002:00000640       __imp_?viewportMouseDoubleClickEvent@QScrollView@@MAEXPAVQMouseEvent@@@Z 10005640     qt-mt323:qt-mt323.dll
 0002:00000644       __imp_?viewportMouseMoveEvent@QScrollView@@MAEXPAVQMouseEvent@@@Z 10005644     qt-mt323:qt-mt323.dll
 0002:00000648       __imp_?viewportMousePressEvent@QScrollView@@MAEXPAVQMouseEvent@@@Z 10005648     qt-mt323:qt-mt323.dll
 0002:0000064c       __imp_?viewportMouseReleaseEvent@QScrollView@@MAEXPAVQMouseEvent@@@Z 1000564c     qt-mt323:qt-mt323.dll
 0002:00000650       __imp_?viewportPaintEvent@QScrollView@@MAEXPAVQPaintEvent@@@Z 10005650     qt-mt323:qt-mt323.dll
 0002:00000654       __imp_?viewportResizeEvent@QScrollView@@MAEXPAVQResizeEvent@@@Z 10005654     qt-mt323:qt-mt323.dll
 0002:00000658       __imp_?viewportWheelEvent@QScrollView@@MAEXPAVQWheelEvent@@@Z 10005658     qt-mt323:qt-mt323.dll
 0002:0000065c       __imp_?wheelEvent@QScrollView@@MAEXPAVQWheelEvent@@@Z 1000565c     qt-mt323:qt-mt323.dll
 0002:00000660       __imp_?widget@QLayoutItem@@UAEPAVQWidget@@XZ 10005660     qt-mt323:qt-mt323.dll
 0002:00000664       __imp_?windowActivationChange@QIconView@@MAEX_N@Z 10005664     qt-mt323:qt-mt323.dll
 0002:00000668       __imp_??0QDomDocument@@QAE@XZ 10005668     qt-mt323:qt-mt323.dll
 0002:0000066c       __imp_?toElement@QDomNode@@QAE?AVQDomElement@@XZ 1000566c     qt-mt323:qt-mt323.dll
 0002:00000670       __imp_?isNull@QDomNode@@QBE_NXZ 10005670     qt-mt323:qt-mt323.dll
 0002:00000674       __imp_?nextSibling@QDomNode@@UBE?AV1@XZ 10005674     qt-mt323:qt-mt323.dll
 0002:00000678       __imp_?firstChild@QDomNode@@UBE?AV1@XZ 10005678     qt-mt323:qt-mt323.dll
 0002:0000067c       __imp_??1QDomNode@@UAE@XZ  1000567c     qt-mt323:qt-mt323.dll
 0002:00000680       __imp_??4QDomNode@@QAEAAV0@ABV0@@Z 10005680     qt-mt323:qt-mt323.dll
 0002:00000684       __imp_??4QPixmap@@QAEAAV0@ABV0@@Z 10005684     qt-mt323:qt-mt323.dll
 0002:00000688       __imp_??1QPixmap@@UAE@XZ   10005688     qt-mt323:qt-mt323.dll
 0002:0000068c       __imp_??0QPixmap@@QAE@ABVQString@@PBDW4ColorMode@0@@Z 1000568c     qt-mt323:qt-mt323.dll
 0002:00000690       __imp_??0QPixmap@@QAE@XZ   10005690     qt-mt323:qt-mt323.dll
 0002:00000694       __imp_?clear@QGDict@@MAEXXZ 10005694     qt-mt323:qt-mt323.dll
 0002:00000698       __imp_??1QGDict@@MAE@XZ    10005698     qt-mt323:qt-mt323.dll
 0002:0000069c       __imp_??0QGDict@@IAE@IW4KeyType@0@_N1@Z 1000569c     qt-mt323:qt-mt323.dll
 0002:000006a0       __imp_??1QStringList@@QAE@XZ 100056a0     qt-mt323:qt-mt323.dll
 0002:000006a4       __imp_??0QStringList@@QAE@ABV0@@Z 100056a4     qt-mt323:qt-mt323.dll
 0002:000006a8       __imp_??0QStringList@@QAE@XZ 100056a8     qt-mt323:qt-mt323.dll
 0002:000006ac       __imp_?clear@QGList@@MAEXXZ 100056ac     qt-mt323:qt-mt323.dll
 0002:000006b0       __imp_?append@QGList@@IAEXPAX@Z 100056b0     qt-mt323:qt-mt323.dll
 0002:000006b4       __imp_??1QGList@@MAE@XZ    100056b4     qt-mt323:qt-mt323.dll
 0002:000006b8       __imp_??0QGList@@IAE@ABV0@@Z 100056b8     qt-mt323:qt-mt323.dll
 0002:000006bc       __imp_??6?$QValueList@VQString@@@@QAEAAV0@ABVQString@@@Z 100056bc     qt-mt323:qt-mt323.dll
 0002:000006c0       __imp_??0QGList@@IAE@XZ    100056c0     qt-mt323:qt-mt323.dll
 0002:000006c4       __imp_??H@YA?BVQString@@ABV0@PBD@Z 100056c4     qt-mt323:qt-mt323.dll
 0002:000006c8       __imp_??H@YA?BVQString@@ABV0@0@Z 100056c8     qt-mt323:qt-mt323.dll
 0002:000006cc       __imp_??9@YA_NABVQString@@PBD@Z 100056cc     qt-mt323:qt-mt323.dll
 0002:000006d0       __imp_??9@YA_NABVQString@@0@Z 100056d0     qt-mt323:qt-mt323.dll
 0002:000006d4       __imp_??4QString@@QAEAAV0@ABV0@@Z 100056d4     qt-mt323:qt-mt323.dll
 0002:000006d8       __imp_??1QString@@QAE@XZ   100056d8     qt-mt323:qt-mt323.dll
 0002:000006dc       __imp_??0QString@@QAE@PBD@Z 100056dc     qt-mt323:qt-mt323.dll
 0002:000006e0       __imp_??0QString@@QAE@XZ   100056e0     qt-mt323:qt-mt323.dll
 0002:000006e4       __imp_??0QMetaObjectCleanUp@@QAE@PBDP6APAVQMetaObject@@XZ@Z 100056e4     qt-mt323:qt-mt323.dll
 0002:000006e8       __imp_?qDebug@@YAXPBDZZ    100056e8     qt-mt323:qt-mt323.dll
 0002:000006ec       \177qt-mt323_NULL_THUNK_DATA 100056ec     qt-mt323:qt-mt323.dll
 0002:000006f0       ___xc_a                    100056f0     MSVCRT:cinitexe.obj
 0002:00000700       ___xc_z                    10005700     MSVCRT:cinitexe.obj
 0002:00000704       ___xi_a                    10005704     MSVCRT:cinitexe.obj
 0002:00000710       ___xi_z                    10005710     MSVCRT:cinitexe.obj
 0002:0000071c       ??_7?$QDict@V?$QPtrList@VnavEntry@@@@@@6B@ 1000571c     config.obj
 0002:0000073c       ??_7config@@6B@            1000573c     config.obj
 0002:00000740       ??_C@_0CE@JBMKNNIG@?1config?1plugins?1navPluginConfig?4@ 10005740     config.obj
 0002:00000764       ??_C@_03ICHNJLJF@key?$AA@  10005764     config.obj
 0002:0000076c       ??_7?$QPtrList@VnavEntry@@@@6B@ 1000576c     config.obj
 0002:0000078c       ??_C@_0P@MDLBFJJO@ConfigNavPages?$AA@ 1000578c     config.obj
 0002:000007a0       ??_C@_0FJ@GKBOLBND@?1config?1plugins?1navPluginConfig?4@ 100057a0     config.obj
 0002:000007fc       ??_C@_04BGIHDKAM@page?$AA@ 100057fc     config.obj
 0002:00000804       ??_C@_04EBPADADD@desc?$AA@ 10005804     config.obj
 0002:0000080c       ??_C@_04OHHBHOGB@link?$AA@ 1000580c     config.obj
 0002:00000814       ??_C@_06JJLAMBGK@target?$AA@ 10005814     config.obj
 0002:0000081c       ??_C@_04MEMAJGDJ@name?$AA@ 1000581c     config.obj
 0002:00000824       ??_C@_06MHMEPCAJ@pixmap?$AA@ 10005824     config.obj
 0002:0000082c       ??_C@_0BI@FJBEEGCK@?1config?1plugins?1images?1?$AA@ 1000582c     config.obj
 0002:00000848       ??_7navIconViewItem@@6B@   10005848     navIconViewItem.obj
 0002:000008c8       ??_C@_02GIPFHKNO@OK?$AA@   100058c8     navPlugin.obj
 0002:000008d0       ??_7QDockWindowList@@6B@   100058d0     navPlugin.obj
 0002:000008f4       ??_7?$QPtrList@VQPopupMenu@@@@6B@ 100058f4     navPlugin.obj
 0002:00000918       ??_7QPopupMenuList@@6B@    10005918     navPlugin.obj
 0002:00000938       ??_C@_04OOEBCMBF@FAIL?$AA@ 10005938     navPlugin.obj
 0002:00000940       ??_C@_08OBALAKLA@READONLY?$AA@ 10005940     navPlugin.obj
 0002:0000094c       ??_C@_04KANDKFIK@DONE?$AA@ 1000594c     navPlugin.obj
 0002:00000954       ??_C@_07NFANNNEC@UNKNOWN?$AA@ 10005954     navPlugin.obj
 0002:00000960       ??_7config_plugin_base@@6BQObject@@@ 10005960     navPlugin.obj
 0002:00000b38       ??_7config_plugin_base@@6BQPaintDevice@@@ 10005b38     navPlugin.obj
 0002:00000b58       ??_C@_0EB@GNDACMDJ@?$CC?5?9?5the?5author?5should?5have?5defin@ 10005b58     navPlugin.obj
 0002:00000b9c       ??_C@_0CH@BDPDPLDP@This?5is?5the?5default?5?$CCAbout?$CC?5text@ 10005b9c     navPlugin.obj
 0002:00000bc8       ??_7navPlugin@@6BQObject@@@ 10005bc8     navPlugin.obj
 0002:00000da0       ??_7navPlugin@@6BQPaintDevice@@@ 10005da0     navPlugin.obj
 0002:00000dc0       ??_C@_0M@ICFANPKF@navPlugin?3?5?$AA@ 10005dc0     navPlugin.obj
 0002:00000dcc       ??_C@_0BK@DDOIAGCG@1onItem?$CI?5QIconViewItem?5?$CK?$CJ?$AA@ 10005dcc     navPlugin.obj
 0002:00000de8       ??_C@_0BK@MBLPOLNO@2onItem?$CI?5QIconViewItem?5?$CK?$CJ?$AA@ 10005de8     navPlugin.obj
 0002:00000e04       ??_C@_0O@PNHIJGEL@1onViewport?$CI?$CJ?$AA@ 10005e04     navPlugin.obj
 0002:00000e14       ??_C@_0O@IBBJLDJA@2onViewport?$CI?$CJ?$AA@ 10005e14     navPlugin.obj
 0002:00000e24       ??_C@_0M@LIJDBMP@?$DMh1?$DO?$CF1?$DM?1h1?$DO?$AA@ 10005e24     navPlugin.obj
 0002:00000e30       ??_C@_0DD@DHNGBGLP@1iconClicked?$CI?5int?0?5QIconViewItem@ 10005e30     navPlugin.obj
 0002:00000e64       ??_C@_0DJ@CIHBOPBC@2mouseButtonPressed?$CIint?0?5QIconVi@ 10005e64     navPlugin.obj
 0002:00000ea0       ??_C@_0BO@GMFDFAEH@1iconClicked?$CIQIconViewItem?5?$CK?$CJ?$AA@ 10005ea0     navPlugin.obj
 0002:00000ec0       ??_C@_0CA@COPIKJJM@2returnPressed?$CIQIconViewItem?5?$CK?$CJ?$AA@ 10005ec0     navPlugin.obj
 0002:00000ee0       ??_C@_0BN@CEGLABJP@2command?$CI?5QString?0?5QString?5?$CJ?$AA@ 10005ee0     navPlugin.obj
 0002:00000f00       ??_C@_09JLEOPMAJ@?5?9?5error?$DN?$AA@ 10005f00     navPlugin.obj
 0002:00000f0c       ??_C@_09LBCHCBIC@?5?9?5value?$DN?$AA@ 10005f0c     navPlugin.obj
 0002:00000f18       ??_C@_0P@ELNNACEA@?5?9?5textStatus?$DN?$AA@ 10005f18     navPlugin.obj
 0002:00000f28       ??_C@_0L@LEAPMKGP@Reply?3?5op?$DN?$AA@ 10005f28     navPlugin.obj
 0002:00000f34       ??_C@_0CO@GKAEALGF@Being?5asked?5to?5navigate?5to?5?$CF1?5wi@ 10005f34     navPlugin.obj
 0002:00000f64       ??_C@_0DL@CNOANKPE@?$DMh3?$DOGeneric?5Navigation?5Plugin?$DM?1h@ 10005f64     navPlugin.obj
 0002:00000fa0       ??_C@_08JNNCPLF@13?324?316?$AA@ 10005fa0     navPlugin.obj
 0002:00000fac       ??_C@_0M@JEDEHNP@Sep?523?52021?$AA@ 10005fac     navPlugin.obj
 0002:00000fb8       ??_C@_08NCKPMOJE@navigate?$AA@ 10005fb8     navPlugin.obj
 0002:00000fc8       ??_7navPluginDlg@@6BQObject@@@ 10005fc8     navPlugindlgimpl.obj
 0002:00001180       ??_7navPluginDlg@@6BQPaintDevice@@@ 10006180     navPlugindlgimpl.obj
 0002:000011a0       ??_C@_09FNFPFPED@14?514?53?51?$AA@ 100061a0     plugindesc.obj
 0002:000011ac       ??_C@_0M@KEPPNGJB@?$CD?5c?5?$CD000000?$AA@ 100061ac     plugindesc.obj
 0002:000011b8       ??_C@_0M@HFCLKLOA@a?5c?5?$CD808080?$AA@ 100061b8     plugindesc.obj
 0002:000011c4       ??_C@_0M@HNGHCCNN@?4?5c?5?$CDffffff?$AA@ 100061c4     plugindesc.obj
 0002:000011d0       ??_C@_0P@HFKAALMG@?4?4?4?4?4?4?4?4?4?4?4?4?4?4?$AA@ 100061d0     plugindesc.obj
 0002:000011e0       ??_C@_0P@MLHMKILI@?4?4?4?4?4?4?4?$CD?$CD?$CD?$CD?4?4?4?$AA@ 100061e0     plugindesc.obj
 0002:000011f0       ??_C@_0P@OHHKDNPB@?4?4?4?4?4?4?$CD?$CD?4?4?$CD?4?4?4?$AA@ 100061f0     plugindesc.obj
 0002:00001200       ??_C@_0P@ODMLFBBG@?4?4?4?4?4?$CD?4?$CD?4?4?$CD?4?4?4?$AA@ 10006200     plugindesc.obj
 0002:00001210       ??_C@_0P@GPOCJCDB@?4?4?4?4?$CD?4?4?$CDa?4?$CD?4?4?4?$AA@ 10006210     plugindesc.obj
 0002:00001220       ??_C@_0P@EHLPPKKI@?4?4?4?$CD?$CD?$CD?$CD?$CD?4?4?$CD?4?4?4?$AA@ 10006220     plugindesc.obj
 0002:00001230       ??_C@_0P@DPPLILLD@?4?4?4?$CD?4aaaa?4?$CD?4?4?4?$AA@ 10006230     plugindesc.obj
 0002:00001240       ??_C@_0P@BDJPMOJJ@?4?4?4?$CD?4?4?4?4?4?4?$CD?4?4?4?$AA@ 10006240     plugindesc.obj
 0002:00001250       ??_C@_0P@JKPGIILG@?4?4?4?$CD?$CD?$CD?$CD?$CD?$CD?$CD?$CD?4?4?4?$AA@ 10006250     plugindesc.obj
 0002:00001264       ??_7config_plugin_desc_base@@6B@ 10006264     plugindesc.obj
 0002:00001278       ??_7plugindesc@@6B@        10006278     plugindesc.obj
 0002:00001288       ??_C@_09IFCEJOKP@navPlugin?$AA@ 10006288     moc_navPlugin.obj
 0002:00001294       ??_C@_06HFKPFKMP@button?$AA@ 10006294     moc_navPlugin.obj
 0002:0000129c       ??_C@_01KBJDNOO@i?$AA@     1000629c     moc_navPlugin.obj
 0002:000012a0       ??_C@_0O@NDCCBDNA@QIconViewItem?$AA@ 100062a0     moc_navPlugin.obj
 0002:000012b0       ??_C@_05BBEJFBFA@point?$AA@ 100062b0     moc_navPlugin.obj
 0002:000012b8       ??_C@_01CAKFMAIO@?$AO?$AA@ 100062b8     moc_navPlugin.obj
 0002:000012c8       ??_C@_0M@PFGNPNAB@iconClicked?$AA@ 100062c8     moc_navPlugin.obj
 0002:000012ec       ??_C@_06CGCGDHF@onItem?$AA@ 100062ec     moc_navPlugin.obj
 0002:00001300       ??_C@_0L@BPIOMCCP@onViewport?$AA@ 10006300     moc_navPlugin.obj
 0002:0000133c       ??_C@_0CO@FJACMMNI@iconClicked?$CIint?0QIconViewItem?$CK?0c@ 1000633c     moc_navPlugin.obj
 0002:0000136c       ??_C@_0BM@IJMGBOII@iconClicked?$CIQIconViewItem?$CK?$CJ?$AA@ 1000636c     moc_navPlugin.obj
 0002:00001388       ??_C@_0BH@FEHOHNKK@onItem?$CIQIconViewItem?$CK?$CJ?$AA@ 10006388     moc_navPlugin.obj
 0002:000013a0       ??_C@_0N@BFGOAMMM@onViewport?$CI?$CJ?$AA@ 100063a0     moc_navPlugin.obj
 0002:000013bc       ??_C@_07KMMNMMFF@command?$AA@ 100063bc     moc_navPlugin.obj
 0002:000013d0       ??_C@_0BJ@FEFNJDLM@command?$CIQString?0QString?$CJ?$AA@ 100063d0     moc_navPlugin.obj
 0002:000013ec       ??_C@_0BB@GDONBMLJ@navPluginDlgBase?$AA@ 100063ec     moc_navPlugindlg.obj
 0002:0000140c       ??_C@_0P@DMEOIADN@languageChange?$AA@ 1000640c     moc_navPlugindlg.obj
 0002:00001428       ??_C@_0BB@PFEIHPGD@languageChange?$CI?$CJ?$AA@ 10006428     moc_navPlugindlg.obj
 0002:0000143c       ??_C@_0N@HOOCFJND@navPluginDlg?$AA@ 1000643c     moc_navPlugindlgimpl.obj
 0002:00001468       ??_7navPluginDlgBase@@6BQObject@@@ 10006468     navPlugindlg.obj
 0002:00001620       ??_7navPluginDlgBase@@6BQPaintDevice@@@ 10006620     navPlugindlg.obj
 0002:00001644       ??_SQLabel@@6BQObject@@@   10006644     navPlugindlg.obj
 0002:0000183c       ??_SQLabel@@6BQPaintDevice@@@ 1000683c     navPlugindlg.obj
 0002:00001864       ??_SQIconView@@6BQObject@@@ 10006864     navPlugindlg.obj
 0002:00001b5c       ??_SQIconView@@6BQPaintDevice@@@ 10006b5c     navPlugindlg.obj
 0002:00001b84       ??_SQVBoxLayout@@6BQObject@@@ 10006b84     navPlugindlg.obj
 0002:00001bec       ??_SQVBoxLayout@@6BQLayoutItem@@@ 10006bec     navPlugindlg.obj
 0002:00001c2c       ??_C@_0BH@DILMGEPC@navPluginDlgBaseLayout?$AA@ 10006c2c     navPlugindlg.obj
 0002:00001c44       ??_C@_0N@CJBMCOMC@textLabel1_4?$AA@ 10006c44     navPlugindlg.obj
 0002:00001c54       ??_C@_09FDMFAAHN@iconView1?$AA@ 10006c54     navPlugindlg.obj
 0002:00001c64       ??_7type_info@@6B@         10006c64     MSVCRT:ti_inst.obj
 0002:00001c68       __pDefaultRawDllMain       10006c68     MSVCRT:crtdll.obj
 0002:00001c68       __pRawDllMain              10006c68     MSVCRT:crtdll.obj
 0002:00001c78       __load_config_used         10006c78     MSVCRT:loadcfg.obj
 0002:00001cc0       ??_R1A@?0A@EA@QGList@@8    10006cc0     config.obj
 0002:00001cdc       ??_R3QGList@@8             10006cdc     config.obj
 0002:00001cec       ??_R2QGList@@8             10006cec     config.obj
 0002:00001cf8       ??_R1A@?0A@EA@QPtrCollection@@8 10006cf8     config.obj
 0002:00001d14       ??_R3QPtrCollection@@8     10006d14     config.obj
 0002:00001d24       ??_R2QPtrCollection@@8     10006d24     config.obj
 0002:00001d2c       ??_R1A@?0A@EA@QGDict@@8    10006d2c     config.obj
 0002:00001d48       ??_R3QGDict@@8             10006d48     config.obj
 0002:00001d58       ??_R2QGDict@@8             10006d58     config.obj
 0002:00001d64       ??_R4?$QPtrList@VnavEntry@@@@6B@ 10006d64     config.obj
 0002:00001d78       ??_R3?$QPtrList@VnavEntry@@@@8 10006d78     config.obj
 0002:00001d88       ??_R2?$QPtrList@VnavEntry@@@@8 10006d88     config.obj
 0002:00001d98       ??_R1A@?0A@EA@?$QPtrList@VnavEntry@@@@8 10006d98     config.obj
 0002:00001db4       ??_R4config@@6B@           10006db4     config.obj
 0002:00001dc8       ??_R3config@@8             10006dc8     config.obj
 0002:00001dd8       ??_R2config@@8             10006dd8     config.obj
 0002:00001de0       ??_R1A@?0A@EA@config@@8    10006de0     config.obj
 0002:00001dfc       ??_R4?$QDict@V?$QPtrList@VnavEntry@@@@@@6B@ 10006dfc     config.obj
 0002:00001e10       ??_R3?$QDict@V?$QPtrList@VnavEntry@@@@@@8 10006e10     config.obj
 0002:00001e20       ??_R2?$QDict@V?$QPtrList@VnavEntry@@@@@@8 10006e20     config.obj
 0002:00001e30       ??_R1A@?0A@EA@?$QDict@V?$QPtrList@VnavEntry@@@@@@8 10006e30     config.obj
 0002:00001e4c       ??_R4navIconViewItem@@6B@  10006e4c     navIconViewItem.obj
 0002:00001e60       ??_R3navIconViewItem@@8    10006e60     navIconViewItem.obj
 0002:00001e70       ??_R2navIconViewItem@@8    10006e70     navIconViewItem.obj
 0002:00001e80       ??_R1A@?0A@EA@navIconViewItem@@8 10006e80     navIconViewItem.obj
 0002:00001e9c       ??_R1A@?0A@EA@QIconViewItem@@8 10006e9c     navIconViewItem.obj
 0002:00001eb8       ??_R3QIconViewItem@@8      10006eb8     navIconViewItem.obj
 0002:00001ec8       ??_R2QIconViewItem@@8      10006ec8     navIconViewItem.obj
 0002:00001ed4       ??_R13?0A@EA@Qt@@8         10006ed4     navIconViewItem.obj
 0002:00001ef0       ??_R3Qt@@8                 10006ef0     navIconViewItem.obj
 0002:00001f00       ??_R2Qt@@8                 10006f00     navIconViewItem.obj
 0002:00001f08       ??_R1A@?0A@EA@Qt@@8        10006f08     navIconViewItem.obj
 0002:00001f24       ??_R4QDockWindowList@@6B@  10006f24     navPlugin.obj
 0002:00001f38       ??_R3QDockWindowList@@8    10006f38     navPlugin.obj
 0002:00001f48       ??_R2QDockWindowList@@8    10006f48     navPlugin.obj
 0002:00001f5c       ??_R1A@?0A@EA@QDockWindowList@@8 10006f5c     navPlugin.obj
 0002:00001f78       ??_R1A@?0A@EA@?$QPtrList@VQDockWindow@@@@8 10006f78     navPlugin.obj
 0002:00001f94       ??_R3?$QPtrList@VQDockWindow@@@@8 10006f94     navPlugin.obj
 0002:00001fa4       ??_R2?$QPtrList@VQDockWindow@@@@8 10006fa4     navPlugin.obj
 0002:00001fb4       ??_R4QPopupMenuList@@6B@   10006fb4     navPlugin.obj
 0002:00001fc8       ??_R3QPopupMenuList@@8     10006fc8     navPlugin.obj
 0002:00001fd8       ??_R2QPopupMenuList@@8     10006fd8     navPlugin.obj
 0002:00001fec       ??_R1A@?0A@EA@QPopupMenuList@@8 10006fec     navPlugin.obj
 0002:00002008       ??_R1A@?0A@EA@?$QPtrList@VQPopupMenu@@@@8 10007008     navPlugin.obj
 0002:00002024       ??_R3?$QPtrList@VQPopupMenu@@@@8 10007024     navPlugin.obj
 0002:00002034       ??_R2?$QPtrList@VQPopupMenu@@@@8 10007034     navPlugin.obj
 0002:00002044       ??_R4?$QPtrList@VQPopupMenu@@@@6B@ 10007044     navPlugin.obj
 0002:00002058       ??_R4config_plugin_base@@6BQObject@@@ 10007058     navPlugin.obj
 0002:0000206c       ??_R3config_plugin_base@@8 1000706c     navPlugin.obj
 0002:0000207c       ??_R2config_plugin_base@@8 1000707c     navPlugin.obj
 0002:00002094       ??_R1A@?0A@EA@config_plugin_base@@8 10007094     navPlugin.obj
 0002:000020b0       ??_R1A@?0A@EA@QWidget@@8   100070b0     navPlugin.obj
 0002:000020cc       ??_R3QWidget@@8            100070cc     navPlugin.obj
 0002:000020dc       ??_R2QWidget@@8            100070dc     navPlugin.obj
 0002:000020f0       ??_R1A@?0A@EA@QObject@@8   100070f0     navPlugin.obj
 0002:0000210c       ??_R3QObject@@8            1000710c     navPlugin.obj
 0002:0000211c       ??_R2QObject@@8            1000711c     navPlugin.obj
 0002:00002128       ??_R1CI@?0A@EA@QPaintDevice@@8 10007128     navPlugin.obj
 0002:00002144       ??_R3QPaintDevice@@8       10007144     navPlugin.obj
 0002:00002154       ??_R2QPaintDevice@@8       10007154     navPlugin.obj
 0002:0000215c       ??_R1A@?0A@EA@QPaintDevice@@8 1000715c     navPlugin.obj
 0002:00002178       ??_R4config_plugin_base@@6BQPaintDevice@@@ 10007178     navPlugin.obj
 0002:0000218c       ??_R4navPlugin@@6BQObject@@@ 1000718c     navPlugin.obj
 0002:000021a0       ??_R3navPlugin@@8          100071a0     navPlugin.obj
 0002:000021b0       ??_R2navPlugin@@8          100071b0     navPlugin.obj
 0002:000021cc       ??_R1A@?0A@EA@navPlugin@@8 100071cc     navPlugin.obj
 0002:000021e8       ??_R4navPlugin@@6BQPaintDevice@@@ 100071e8     navPlugin.obj
 0002:000021fc       ??_R4navPluginDlg@@6BQObject@@@ 100071fc     navPlugindlgimpl.obj
 0002:00002210       ??_R3navPluginDlg@@8       10007210     navPlugindlgimpl.obj
 0002:00002220       ??_R2navPluginDlg@@8       10007220     navPlugindlgimpl.obj
 0002:0000223c       ??_R1A@?0A@EA@navPluginDlg@@8 1000723c     navPlugindlgimpl.obj
 0002:00002258       ??_R1A@?0A@EA@navPluginDlgBase@@8 10007258     navPlugindlgimpl.obj
 0002:00002274       ??_R3navPluginDlgBase@@8   10007274     navPlugindlgimpl.obj
 0002:00002284       ??_R2navPluginDlgBase@@8   10007284     navPlugindlgimpl.obj
 0002:0000229c       ??_R4navPluginDlg@@6BQPaintDevice@@@ 1000729c     navPlugindlgimpl.obj
 0002:000022b0       ??_R4config_plugin_desc_base@@6B@ 100072b0     plugindesc.obj
 0002:000022c4       ??_R3config_plugin_desc_base@@8 100072c4     plugindesc.obj
 0002:000022d4       ??_R2config_plugin_desc_base@@8 100072d4     plugindesc.obj
 0002:000022dc       ??_R1A@?0A@EA@config_plugin_desc_base@@8 100072dc     plugindesc.obj
 0002:000022f8       ??_R4plugindesc@@6B@       100072f8     plugindesc.obj
 0002:0000230c       ??_R3plugindesc@@8         1000730c     plugindesc.obj
 0002:0000231c       ??_R2plugindesc@@8         1000731c     plugindesc.obj
 0002:00002328       ??_R1A@?0A@EA@plugindesc@@8 10007328     plugindesc.obj
 0002:00002344       ??_R4QVBoxLayout@@6BQObject@@@ 10007344     navPlugindlg.obj
 0002:00002358       ??_R3QVBoxLayout@@8        10007358     navPlugindlg.obj
 0002:00002368       ??_R2QVBoxLayout@@8        10007368     navPlugindlg.obj
 0002:00002384       ??_R1A@?0A@EA@QVBoxLayout@@8 10007384     navPlugindlg.obj
 0002:000023a0       ??_R1A@?0A@EA@QBoxLayout@@8 100073a0     navPlugindlg.obj
 0002:000023bc       ??_R3QBoxLayout@@8         100073bc     navPlugindlg.obj
 0002:000023cc       ??_R2QBoxLayout@@8         100073cc     navPlugindlg.obj
 0002:000023e4       ??_R1A@?0A@EA@QLayout@@8   100073e4     navPlugindlg.obj
 0002:00002400       ??_R3QLayout@@8            10007400     navPlugindlg.obj
 0002:00002410       ??_R2QLayout@@8            10007410     navPlugindlg.obj
 0002:00002424       ??_R1CI@?0A@EA@QLayoutItem@@8 10007424     navPlugindlg.obj
 0002:00002440       ??_R3QLayoutItem@@8        10007440     navPlugindlg.obj
 0002:00002450       ??_R2QLayoutItem@@8        10007450     navPlugindlg.obj
 0002:00002458       ??_R1A@?0A@EA@QLayoutItem@@8 10007458     navPlugindlg.obj
 0002:00002474       ??_R4QVBoxLayout@@6BQLayoutItem@@@ 10007474     navPlugindlg.obj
 0002:00002488       ??_R4QLabel@@6BQObject@@@  10007488     navPlugindlg.obj
 0002:0000249c       ??_R3QLabel@@8             1000749c     navPlugindlg.obj
 0002:000024ac       ??_R2QLabel@@8             100074ac     navPlugindlg.obj
 0002:000024c8       ??_R1A@?0A@EA@QLabel@@8    100074c8     navPlugindlg.obj
 0002:000024e4       ??_R1A@?0A@EA@QFrame@@8    100074e4     navPlugindlg.obj
 0002:00002500       ??_R3QFrame@@8             10007500     navPlugindlg.obj
 0002:00002510       ??_R2QFrame@@8             10007510     navPlugindlg.obj
 0002:00002528       ??_R4QLabel@@6BQPaintDevice@@@ 10007528     navPlugindlg.obj
 0002:0000253c       ??_R4QIconView@@6BQObject@@@ 1000753c     navPlugindlg.obj
 0002:00002550       ??_R3QIconView@@8          10007550     navPlugindlg.obj
 0002:00002560       ??_R2QIconView@@8          10007560     navPlugindlg.obj
 0002:00002580       ??_R1A@?0A@EA@QIconView@@8 10007580     navPlugindlg.obj
 0002:0000259c       ??_R1A@?0A@EA@QScrollView@@8 1000759c     navPlugindlg.obj
 0002:000025b8       ??_R3QScrollView@@8        100075b8     navPlugindlg.obj
 0002:000025c8       ??_R2QScrollView@@8        100075c8     navPlugindlg.obj
 0002:000025e4       ??_R4QIconView@@6BQPaintDevice@@@ 100075e4     navPlugindlg.obj
 0002:000025f8       ??_R4navPluginDlgBase@@6BQObject@@@ 100075f8     navPlugindlg.obj
 0002:0000260c       ??_R4navPluginDlgBase@@6BQPaintDevice@@@ 1000760c     navPlugindlg.obj
 0002:00002620       ??_R4type_info@@6B@        10007620     MSVCRT:ti_inst.obj
 0002:00002634       ??_R3type_info@@8          10007634     MSVCRT:ti_inst.obj
 0002:00002644       ??_R2type_info@@8          10007644     MSVCRT:ti_inst.obj
 0002:0000264c       ??_R1A@?0A@EA@type_info@@8 1000764c     MSVCRT:ti_inst.obj
 0002:00002668       ___rtc_iaa                 10007668     MSVCRT:initsect.obj
 0002:0000266c       ___rtc_izz                 1000766c     MSVCRT:initsect.obj
 0002:00002670       ___rtc_taa                 10007670     MSVCRT:initsect.obj
 0002:00002674       ___rtc_tzz                 10007674     MSVCRT:initsect.obj
 0002:00002ef0       __IMPORT_DESCRIPTOR_qt-mt323 10007ef0     qt-mt323:qt-mt323.dll
 0002:00002f04       __IMPORT_DESCRIPTOR_MSVCR120 10007f04     MSVCRT:MSVCR120.dll
 0002:00002f18       __IMPORT_DESCRIPTOR_KERNEL32 10007f18     kernel32:KERNEL32.dll
 0002:00002f2c       __NULL_IMPORT_DESCRIPTOR   10007f2c     qt-mt323:qt-mt323.dll
 0003:00000098       ___security_cookie         1000d098     MSVCRT:gs_cookie.obj
 0003:0000009c       ___security_cookie_complement 1000d09c     MSVCRT:gs_cookie.obj
 0003:000000a0       ___native_dllmain_reason   1000d0a0     MSVCRT:natstart.obj
 0003:000000a4       ??_R0?AVQGList@@@8         1000d0a4     config.obj
 0003:000000bc       ??_R0?AVQPtrCollection@@@8 1000d0bc     config.obj
 0003:000000dc       ??_R0?AVQGDict@@@8         1000d0dc     config.obj
 0003:000000f4       ??_R0?AV?$QPtrList@VnavEntry@@@@@8 1000d0f4     config.obj
 0003:0000011c       ??_R0?AVconfig@@@8         1000d11c     config.obj
 0003:00000134       ??_R0?AV?$QDict@V?$QPtrList@VnavEntry@@@@@@@8 1000d134     config.obj
 0003:00000164       ??_R0?AVnavIconViewItem@@@8 1000d164     navIconViewItem.obj
 0003:00000184       ??_R0?AVQIconViewItem@@@8  1000d184     navIconViewItem.obj
 0003:000001a0       ??_R0?AVQt@@@8             1000d1a0     navIconViewItem.obj
 0003:000001b4       ??_R0?AVQDockWindowList@@@8 1000d1b4     navPlugin.obj
 0003:000001d4       ??_R0?AV?$QPtrList@VQDockWindow@@@@@8 1000d1d4     navPlugin.obj
 0003:000001fc       ??_R0?AVQPopupMenuList@@@8 1000d1fc     navPlugin.obj
 0003:0000021c       ??_R0?AV?$QPtrList@VQPopupMenu@@@@@8 1000d21c     navPlugin.obj
 0003:00000244       ??_R0?AVconfig_plugin_base@@@8 1000d244     navPlugin.obj
 0003:00000268       ??_R0?AVQWidget@@@8        1000d268     navPlugin.obj
 0003:00000280       ??_R0?AVQObject@@@8        1000d280     navPlugin.obj
 0003:00000298       ??_R0?AVQPaintDevice@@@8   1000d298     navPlugin.obj
 0003:000002b4       ??_R0?AVnavPlugin@@@8      1000d2b4     navPlugin.obj
 0003:000002cc       ??_R0?AVnavPluginDlg@@@8   1000d2cc     navPlugindlgimpl.obj
 0003:000002e8       ??_R0?AVnavPluginDlgBase@@@8 1000d2e8     navPlugindlgimpl.obj
 0003:00000308       ??_R0?AVconfig_plugin_desc_base@@@8 1000d308     plugindesc.obj
 0003:00000330       ??_R0?AVplugindesc@@@8     1000d330     plugindesc.obj
 0003:0000034c       ??_R0?AVQVBoxLayout@@@8    1000d34c     navPlugindlg.obj
 0003:00000368       ??_R0?AVQBoxLayout@@@8     1000d368     navPlugindlg.obj
 0003:00000384       ??_R0?AVQLayout@@@8        1000d384     navPlugindlg.obj
 0003:0000039c       ??_R0?AVQLayoutItem@@@8    1000d39c     navPlugindlg.obj
 0003:000003b8       ??_R0?AVQLabel@@@8         1000d3b8     navPlugindlg.obj
 0003:000003d0       ??_R0?AVQFrame@@@8         1000d3d0     navPlugindlg.obj
 0003:000003e8       ??_R0?AVQIconView@@@8      1000d3e8     navPlugindlg.obj
 0003:00000400       ??_R0?AVQScrollView@@@8    1000d400     navPlugindlg.obj
 0003:0000041c       ??_R0?AVtype_info@@@8      1000d41c     MSVCRT:ti_inst.obj
 0003:00000438       ?metaObj@navPlugin@@0PAVQMetaObject@@A 1000d438     moc_navPlugin.obj
 0003:00000464       ?metaObj@navPluginDlgBase@@0PAVQMetaObject@@A 1000d464     moc_navPlugindlg.obj
 0003:0000046c       ?metaObj@navPluginDlg@@0PAVQMetaObject@@A 1000d46c     moc_navPlugindlgimpl.obj
 0003:000007c0       ?__type_info_root_node@@3U__type_info_node@@A 1000d7c0     MSVCRT:tncleanup.obj
 0003:000007c8       ___native_startup_lock     1000d7c8     <common>
 0003:000007cc       ___native_startup_state    1000d7cc     <common>
 0003:000007d0       ___dyn_tls_init_callback   1000d7d0     <common>
 0003:000007d4       ___onexitend               1000d7d4     <common>
 0003:000007d8       ___onexitbegin             1000d7d8     <common>

 entry point at        0001:00002b44

 Static symbols

 0001:00000000       ??__EcleanUp_navPlugin@@YAXXZ 10001000 f   moc_navPlugin.obj
 0001:00000021       ??__EcleanUp_navPluginDlgBase@@YAXXZ 10001021 f   moc_navPlugindlg.obj
 0001:00000042       ??__EcleanUp_navPluginDlg@@YAXXZ 10001042 f   moc_navPlugindlgimpl.obj
 0001:00002901       _pre_c_init                10003901 f   MSVCRT:crtdll.obj
 0001:00002b67       ___DllMainCRTStartup       10003b67 f   MSVCRT:crtdll.obj
 0001:00002de0       $$000000                   10003de0     MSVCRT:sehprolg4.obj
 0001:000030fc       __unwindfunclet$??0config@@QAE@ABVQString@@@Z$0 100040fc f   config.obj
 0001:00003107       __unwindfunclet$??0config@@QAE@ABVQString@@@Z$1 10004107 f   config.obj
 0001:00003113       __ehhandler$??0config@@QAE@ABVQString@@@Z 10004113 f   config.obj
 0001:0000312e       __unwindfunclet$??0navEntry@@QAE@ABVQString@@0ABVQPixmap@@@Z$0 1000412e f   config.obj
 0001:00003137       __unwindfunclet$??0navEntry@@QAE@ABVQString@@0ABVQPixmap@@@Z$1 10004137 f   config.obj
 0001:00003143       __unwindfunclet$??0navEntry@@QAE@ABVQString@@0ABVQPixmap@@@Z$2 10004143 f   config.obj
 0001:0000314f       __ehhandler$??0navEntry@@QAE@ABVQString@@0ABVQPixmap@@@Z 1000414f f   config.obj
 0001:0000316a       __unwindfunclet$??1?$QDict@V?$QPtrList@VnavEntry@@@@@@UAE@XZ$0 1000416a f   config.obj
 0001:00003173       __ehhandler$??1?$QDict@V?$QPtrList@VnavEntry@@@@@@UAE@XZ 10004173 f   config.obj
 0001:0000318e       __unwindfunclet$??1?$QPtrList@VQPopupMenu@@@@UAE@XZ$0 1000418e f   config.obj
 0001:0000318e       __unwindfunclet$??1?$QPtrList@VnavEntry@@@@UAE@XZ$0 1000418e f   config.obj
 0001:00003197       __ehhandler$??1?$QPtrList@VnavEntry@@@@UAE@XZ 10004197 f   config.obj
 0001:00003197       __ehhandler$??1?$QPtrList@VQPopupMenu@@@@UAE@XZ 10004197 f   config.obj
 0001:000031b2       __unwindfunclet$??1config@@UAE@XZ$0 100041b2 f   config.obj
 0001:000031bd       __ehhandler$??1config@@UAE@XZ 100041bd f   config.obj
 0001:000031d8       __unwindfunclet$??1navEntry@@QAE@XZ$0 100041d8 f   config.obj
 0001:000031e1       __unwindfunclet$??1navEntry@@QAE@XZ$1 100041e1 f   config.obj
 0001:000031ed       __ehhandler$??1navEntry@@QAE@XZ 100041ed f   config.obj
 0001:00003208       __unwindfunclet$?getKeys@config@@QAE?AVQStringList@@XZ$0 10004208 f   config.obj
 0001:00003211       __unwindfunclet$?getKeys@config@@QAE?AVQStringList@@XZ$1 10004211 f   config.obj
 0001:0000321a       __unwindfunclet$?getKeys@config@@QAE?AVQStringList@@XZ$2 1000421a f   config.obj
 0001:00003223       __unwindfunclet$?getKeys@config@@QAE?AVQStringList@@XZ$3 10004223 f   config.obj
 0001:0000322c       __unwindfunclet$?getKeys@config@@QAE?AVQStringList@@XZ$4 1000422c f   config.obj
 0001:00003246       __unwindfunclet$?getKeys@config@@QAE?AVQStringList@@XZ$5 10004246 f   config.obj
 0001:0000324f       __unwindfunclet$?getKeys@config@@QAE?AVQStringList@@XZ$6 1000424f f   config.obj
 0001:00003258       __unwindfunclet$?getKeys@config@@QAE?AVQStringList@@XZ$7 10004258 f   config.obj
 0001:00003261       __unwindfunclet$?getKeys@config@@QAE?AVQStringList@@XZ$8 10004261 f   config.obj
 0001:0000326a       __unwindfunclet$?getKeys@config@@QAE?AVQStringList@@XZ$9 1000426a f   config.obj
 0001:00003273       __unwindfunclet$?getKeys@config@@QAE?AVQStringList@@XZ$10 10004273 f   config.obj
 0001:0000327c       __ehhandler$?getKeys@config@@QAE?AVQStringList@@XZ 1000427c f   config.obj
 0001:00003297       __unwindfunclet$?getNavEntry@config@@QAE?AV?$QPtrList@VnavEntry@@@@ABVQString@@AAV3@@Z$0 10004297 f   config.obj
 0001:000032a2       __unwindfunclet$?getNavEntry@config@@QAE?AV?$QPtrList@VnavEntry@@@@ABVQString@@AAV3@@Z$1 100042a2 f   config.obj
 0001:000032ab       __unwindfunclet$?getNavEntry@config@@QAE?AV?$QPtrList@VnavEntry@@@@ABVQString@@AAV3@@Z$2 100042ab f   config.obj
 0001:000032b4       __unwindfunclet$?getNavEntry@config@@QAE?AV?$QPtrList@VnavEntry@@@@ABVQString@@AAV3@@Z$3 100042b4 f   config.obj
 0001:000032c0       __unwindfunclet$?getNavEntry@config@@QAE?AV?$QPtrList@VnavEntry@@@@ABVQString@@AAV3@@Z$4 100042c0 f   config.obj
 0001:000032d9       __unwindfunclet$?getNavEntry@config@@QAE?AV?$QPtrList@VnavEntry@@@@ABVQString@@AAV3@@Z$5 100042d9 f   config.obj
 0001:000032e2       __unwindfunclet$?getNavEntry@config@@QAE?AV?$QPtrList@VnavEntry@@@@ABVQString@@AAV3@@Z$6 100042e2 f   config.obj
 0001:000032eb       __unwindfunclet$?getNavEntry@config@@QAE?AV?$QPtrList@VnavEntry@@@@ABVQString@@AAV3@@Z$7 100042eb f   config.obj
 0001:000032f4       __unwindfunclet$?getNavEntry@config@@QAE?AV?$QPtrList@VnavEntry@@@@ABVQString@@AAV3@@Z$9 100042f4 f   config.obj
 0001:000032fd       __unwindfunclet$?getNavEntry@config@@QAE?AV?$QPtrList@VnavEntry@@@@ABVQString@@AAV3@@Z$10 100042fd f   config.obj
 0001:00003306       __unwindfunclet$?getNavEntry@config@@QAE?AV?$QPtrList@VnavEntry@@@@ABVQString@@AAV3@@Z$11 10004306 f   config.obj
 0001:0000330f       __unwindfunclet$?getNavEntry@config@@QAE?AV?$QPtrList@VnavEntry@@@@ABVQString@@AAV3@@Z$12 1000430f f   config.obj
 0001:00003318       __unwindfunclet$?getNavEntry@config@@QAE?AV?$QPtrList@VnavEntry@@@@ABVQString@@AAV3@@Z$8 10004318 f   config.obj
 0001:00003321       __unwindfunclet$?getNavEntry@config@@QAE?AV?$QPtrList@VnavEntry@@@@ABVQString@@AAV3@@Z$13 10004321 f   config.obj
 0001:0000332a       __unwindfunclet$?getNavEntry@config@@QAE?AV?$QPtrList@VnavEntry@@@@ABVQString@@AAV3@@Z$14 1000432a f   config.obj
 0001:00003333       __unwindfunclet$?getNavEntry@config@@QAE?AV?$QPtrList@VnavEntry@@@@ABVQString@@AAV3@@Z$15 10004333 f   config.obj
 0001:0000333c       __unwindfunclet$?getNavEntry@config@@QAE?AV?$QPtrList@VnavEntry@@@@ABVQString@@AAV3@@Z$17 1000433c f   config.obj
 0001:00003345       __unwindfunclet$?getNavEntry@config@@QAE?AV?$QPtrList@VnavEntry@@@@ABVQString@@AAV3@@Z$18 10004345 f   config.obj
 0001:0000334e       __unwindfunclet$?getNavEntry@config@@QAE?AV?$QPtrList@VnavEntry@@@@ABVQString@@AAV3@@Z$19 1000434e f   config.obj
 0001:00003357       __unwindfunclet$?getNavEntry@config@@QAE?AV?$QPtrList@VnavEntry@@@@ABVQString@@AAV3@@Z$20 10004357 f   config.obj
 0001:00003360       __unwindfunclet$?getNavEntry@config@@QAE?AV?$QPtrList@VnavEntry@@@@ABVQString@@AAV3@@Z$21 10004360 f   config.obj
 0001:00003369       __unwindfunclet$?getNavEntry@config@@QAE?AV?$QPtrList@VnavEntry@@@@ABVQString@@AAV3@@Z$22 10004369 f   config.obj
 0001:00003372       __unwindfunclet$?getNavEntry@config@@QAE?AV?$QPtrList@VnavEntry@@@@ABVQString@@AAV3@@Z$23 10004372 f   config.obj
 0001:0000337b       __unwindfunclet$?getNavEntry@config@@QAE?AV?$QPtrList@VnavEntry@@@@ABVQString@@AAV3@@Z$24 1000437b f   config.obj
 0001:00003384       __unwindfunclet$?getNavEntry@config@@QAE?AV?$QPtrList@VnavEntry@@@@ABVQString@@AAV3@@Z$25 10004384 f   config.obj
 0001:0000338d       __unwindfunclet$?getNavEntry@config@@QAE?AV?$QPtrList@VnavEntry@@@@ABVQString@@AAV3@@Z$26 1000438d f   config.obj
 0001:00003396       __unwindfunclet$?getNavEntry@config@@QAE?AV?$QPtrList@VnavEntry@@@@ABVQString@@AAV3@@Z$27 10004396 f   config.obj
 0001:000033a2       __unwindfunclet$?getNavEntry@config@@QAE?AV?$QPtrList@VnavEntry@@@@ABVQString@@AAV3@@Z$28 100043a2 f   config.obj
 0001:000033af       __unwindfunclet$?getNavEntry@config@@QAE?AV?$QPtrList@VnavEntry@@@@ABVQString@@AAV3@@Z$16 100043af f   config.obj
 0001:000033bb       __ehhandler$?getNavEntry@config@@QAE?AV?$QPtrList@VnavEntry@@@@ABVQString@@AAV3@@Z 100043bb f   config.obj
 0001:000033d9       __unwindfunclet$??0navIconViewItem@@QAE@PAVQIconView@@ABVQString@@1ABVQPixmap@@@Z$0 100043d9 f   navIconViewItem.obj
 0001:000033d9       __unwindfunclet$??0navIconViewItem@@QAE@PAVQIconView@@ABVQString@@1@Z$0 100043d9 f   navIconViewItem.obj
 0001:000033e2       __unwindfunclet$??0navIconViewItem@@QAE@PAVQIconView@@ABVQString@@1@Z$1 100043e2 f   navIconViewItem.obj
 0001:000033e2       __unwindfunclet$??0navIconViewItem@@QAE@PAVQIconView@@ABVQString@@1ABVQPixmap@@@Z$1 100043e2 f   navIconViewItem.obj
 0001:000033ee       __ehhandler$??0navIconViewItem@@QAE@PAVQIconView@@ABVQString@@1ABVQPixmap@@@Z 100043ee f   navIconViewItem.obj
 0001:000033ee       __ehhandler$??0navIconViewItem@@QAE@PAVQIconView@@ABVQString@@1@Z 100043ee f   navIconViewItem.obj
 0001:00003409       __unwindfunclet$??1navIconViewItem@@UAE@XZ$0 10004409 f   navIconViewItem.obj
 0001:00003412       __ehhandler$??1navIconViewItem@@UAE@XZ 10004412 f   navIconViewItem.obj
 0001:0000342d       __unwindfunclet$??0config_plugin_base@@QAE@ABVQString@@00@Z$0 1000442d f   navPlugin.obj
 0001:00003436       __unwindfunclet$??0config_plugin_base@@QAE@ABVQString@@00@Z$1 10004436 f   navPlugin.obj
 0001:00003442       __unwindfunclet$??0config_plugin_base@@QAE@ABVQString@@00@Z$2 10004442 f   navPlugin.obj
 0001:0000344e       __unwindfunclet$??0config_plugin_base@@QAE@ABVQString@@00@Z$3 1000444e f   navPlugin.obj
 0001:0000345a       __ehhandler$??0config_plugin_base@@QAE@ABVQString@@00@Z 1000445a f   navPlugin.obj
 0001:00003475       __unwindfunclet$??0navPlugin@@QAE@ABVQString@@00@Z$0 10004475 f   navPlugin.obj
 0001:0000347d       __unwindfunclet$??0navPlugin@@QAE@ABVQString@@00@Z$1 1000447d f   navPlugin.obj
 0001:00003487       __unwindfunclet$??0navPlugin@@QAE@ABVQString@@00@Z$2 10004487 f   navPlugin.obj
 0001:0000348f       __unwindfunclet$??0navPlugin@@QAE@ABVQString@@00@Z$3 1000448f f   navPlugin.obj
 0001:00003498       __unwindfunclet$??0navPlugin@@QAE@ABVQString@@00@Z$4 10004498 f   navPlugin.obj
 0001:000034a0       __unwindfunclet$??0navPlugin@@QAE@ABVQString@@00@Z$5 100044a0 f   navPlugin.obj
 0001:000034a9       __unwindfunclet$??0navPlugin@@QAE@ABVQString@@00@Z$6 100044a9 f   navPlugin.obj
 0001:000034b2       __unwindfunclet$??0navPlugin@@QAE@ABVQString@@00@Z$7 100044b2 f   navPlugin.obj
 0001:000034bc       __unwindfunclet$??0navPlugin@@QAE@ABVQString@@00@Z$8 100044bc f   navPlugin.obj
 0001:000034c6       __ehhandler$??0navPlugin@@QAE@ABVQString@@00@Z 100044c6 f   navPlugin.obj
 0001:000034e1       __unwindfunclet$??1QDockWindowList@@UAE@XZ$0 100044e1 f   navPlugin.obj
 0001:000034ea       __unwindfunclet$??1QDockWindowList@@UAE@XZ$1 100044ea f   navPlugin.obj
 0001:000034f3       __ehhandler$??1QDockWindowList@@UAE@XZ 100044f3 f   navPlugin.obj
 0001:0000350e       __unwindfunclet$??1QPopupMenuList@@UAE@XZ$0 1000450e f   navPlugin.obj
 0001:00003516       __ehhandler$??1QPopupMenuList@@UAE@XZ 10004516 f   navPlugin.obj
 0001:00003531       __unwindfunclet$??1config_plugin_base@@UAE@XZ$0 10004531 f   navPlugin.obj
 0001:0000353a       __unwindfunclet$??1config_plugin_base@@UAE@XZ$1 1000453a f   navPlugin.obj
 0001:00003546       __unwindfunclet$??1config_plugin_base@@UAE@XZ$2 10004546 f   navPlugin.obj
 0001:00003552       __ehhandler$??1config_plugin_base@@UAE@XZ 10004552 f   navPlugin.obj
 0001:0000356d       __unwindfunclet$?about@config_plugin_base@@UAE?AVQString@@XZ$0 1000456d f   navPlugin.obj
 0001:00003576       __unwindfunclet$?about@config_plugin_base@@UAE?AVQString@@XZ$1 10004576 f   navPlugin.obj
 0001:00003590       __ehhandler$?about@config_plugin_base@@UAE?AVQString@@XZ 10004590 f   navPlugin.obj
 0001:000035ab       __unwindfunclet$?about@navPlugin@@UAE?AVQString@@XZ$0 100045ab f   navPlugin.obj
 0001:000035b4       __unwindfunclet$?about@navPlugin@@UAE?AVQString@@XZ$1 100045b4 f   navPlugin.obj
 0001:000035bd       __unwindfunclet$?about@navPlugin@@UAE?AVQString@@XZ$2 100045bd f   navPlugin.obj
 0001:000035c6       __unwindfunclet$?about@navPlugin@@UAE?AVQString@@XZ$3 100045c6 f   navPlugin.obj
 0001:000035cf       __unwindfunclet$?about@navPlugin@@UAE?AVQString@@XZ$4 100045cf f   navPlugin.obj
 0001:000035e9       __ehhandler$?about@navPlugin@@UAE?AVQString@@XZ 100045e9 f   navPlugin.obj
 0001:00003604       __unwindfunclet$?iconClicked@navPlugin@@QAEXPAVQIconViewItem@@@Z$0 10004604 f   navPlugin.obj
 0001:0000360d       __ehhandler$?iconClicked@navPlugin@@QAEXPAVQIconViewItem@@@Z 1000460d f   navPlugin.obj
 0001:00003628       __unwindfunclet$?navigate@navPlugin@@UAEXABVQString@@0@Z$0 10004628 f   navPlugin.obj
 0001:00003631       __unwindfunclet$?navigate@navPlugin@@UAEXABVQString@@0@Z$1 10004631 f   navPlugin.obj
 0001:0000363a       __unwindfunclet$?navigate@navPlugin@@UAEXABVQString@@0@Z$2 1000463a f   navPlugin.obj
 0001:00003643       __ehhandler$?navigate@navPlugin@@UAEXABVQString@@0@Z 10004643 f   navPlugin.obj
 0001:0000365e       __unwindfunclet$?onItem@navPlugin@@QAEXPAVQIconViewItem@@@Z$0 1000465e f   navPlugin.obj
 0001:00003667       __ehhandler$?onItem@navPlugin@@QAEXPAVQIconViewItem@@@Z 10004667 f   navPlugin.obj
 0001:00003682       __unwindfunclet$?reply@navPlugin@@UAEXPAVresponse@@@Z$0 10004682 f   navPlugin.obj
 0001:0000368b       __unwindfunclet$?reply@navPlugin@@UAEXPAVresponse@@@Z$1 1000468b f   navPlugin.obj
 0001:00003694       __unwindfunclet$?reply@navPlugin@@UAEXPAVresponse@@@Z$2 10004694 f   navPlugin.obj
 0001:0000369d       __unwindfunclet$?reply@navPlugin@@UAEXPAVresponse@@@Z$3 1000469d f   navPlugin.obj
 0001:000036a6       __unwindfunclet$?reply@navPlugin@@UAEXPAVresponse@@@Z$4 100046a6 f   navPlugin.obj
 0001:000036af       __unwindfunclet$?reply@navPlugin@@UAEXPAVresponse@@@Z$5 100046af f   navPlugin.obj
 0001:000036b8       __unwindfunclet$?reply@navPlugin@@UAEXPAVresponse@@@Z$6 100046b8 f   navPlugin.obj
 0001:000036c1       __unwindfunclet$?reply@navPlugin@@UAEXPAVresponse@@@Z$7 100046c1 f   navPlugin.obj
 0001:000036ca       __unwindfunclet$?reply@navPlugin@@UAEXPAVresponse@@@Z$8 100046ca f   navPlugin.obj
 0001:000036d3       __ehhandler$?reply@navPlugin@@UAEXPAVresponse@@@Z 100046d3 f   navPlugin.obj
 0001:000036ee       __unwindfunclet$?create@plugindesc@@UAEPAVconfig_plugin_base@@ABVQString@@00@Z$0 100046ee f   plugindesc.obj
 0001:000036f8       __ehhandler$?create@plugindesc@@UAEPAVconfig_plugin_base@@ABVQString@@00@Z 100046f8 f   plugindesc.obj
 0001:00003713       __unwindfunclet$?keys@plugindesc@@UAE?AVQStringList@@ABVQString@@0@Z$0 10004713 f   plugindesc.obj
 0001:0000371b       __unwindfunclet$?keys@plugindesc@@UAE?AVQStringList@@ABVQString@@0@Z$1 1000471b f   plugindesc.obj
 0001:00003735       __ehhandler$?keys@plugindesc@@UAE?AVQStringList@@ABVQString@@0@Z 10004735 f   plugindesc.obj
 0001:00003750       __unwindfunclet$?command@navPluginDlg@@IAEXVQString@@0@Z$0 10004750 f   moc_navPlugin.obj
 0001:00003750       __unwindfunclet$?command@navPlugin@@IAEXVQString@@0@Z$0 10004750 f   moc_navPlugin.obj
 0001:00003759       __unwindfunclet$?command@navPlugin@@IAEXVQString@@0@Z$1 10004759 f   moc_navPlugin.obj
 0001:00003759       __unwindfunclet$?command@navPluginDlg@@IAEXVQString@@0@Z$1 10004759 f   moc_navPlugin.obj
 0001:00003762       __unwindfunclet$?command@navPlugin@@IAEXVQString@@0@Z$2 10004762 f   moc_navPlugin.obj
 0001:00003762       __unwindfunclet$?command@navPluginDlg@@IAEXVQString@@0@Z$2 10004762 f   moc_navPlugin.obj
 0001:00003776       __ehhandler$?command@navPlugin@@IAEXVQString@@0@Z 10004776 f   moc_navPlugin.obj
 0001:00003776       __ehhandler$?command@navPluginDlg@@IAEXVQString@@0@Z 10004776 f   moc_navPlugin.obj
 0001:0000379b       __unwindfunclet$?qt_emit@navPluginDlg@@UAE_NHPAUQUObject@@@Z$0 1000479b f   moc_navPlugin.obj
 0001:0000379b       __unwindfunclet$?qt_emit@navPlugin@@UAE_NHPAUQUObject@@@Z$0 1000479b f   moc_navPlugin.obj
 0001:000037a4       __ehhandler$?qt_emit@navPlugin@@UAE_NHPAUQUObject@@@Z 100047a4 f   moc_navPlugin.obj
 0001:000037a4       __ehhandler$?qt_emit@navPluginDlg@@UAE_NHPAUQUObject@@@Z 100047a4 f   moc_navPlugin.obj
 0001:000037bf       __unwindfunclet$??0navPluginDlgBase@@QAE@PAVQWidget@@PBDI@Z$0 100047bf f   navPlugindlg.obj
 0001:000037c8       __unwindfunclet$??0navPluginDlgBase@@QAE@PAVQWidget@@PBDI@Z$1 100047c8 f   navPlugindlg.obj
 0001:000037d2       __unwindfunclet$??0navPluginDlgBase@@QAE@PAVQWidget@@PBDI@Z$2 100047d2 f   navPlugindlg.obj
 0001:000037dc       __unwindfunclet$??0navPluginDlgBase@@QAE@PAVQWidget@@PBDI@Z$3 100047dc f   navPlugindlg.obj
 0001:000037e6       __ehhandler$??0navPluginDlgBase@@QAE@PAVQWidget@@PBDI@Z 100047e6 f   navPlugindlg.obj
 0001:00003801       __unwindfunclet$?db@@YAXABVQString@@@Z$0 10004801 f   navPlugindlg.obj
 0001:00003801       __unwindfunclet$?languageChange@navPluginDlgBase@@MAEXXZ$0 10004801 f   navPlugindlg.obj
 0001:0000380a       __ehhandler$?languageChange@navPluginDlgBase@@MAEXXZ 1000480a f   navPlugindlg.obj
 0001:0000380a       __ehhandler$?db@@YAXABVQString@@@Z 1000480a f   navPlugindlg.obj
 0001:00003825       ??__FcleanUp_navPlugin@@YAXXZ 10004825 f   moc_navPlugin.obj
 0001:00003830       ??__FcleanUp_navPluginDlgBase@@YAXXZ 10004830 f   moc_navPlugindlg.obj
 0001:0000383b       ??__FcleanUp_navPluginDlg@@YAXXZ 1000483b f   moc_navPlugindlgimpl.obj
 0002:000006f4       _cleanUp_navPlugin$initializer$ 100056f4     moc_navPlugin.obj
 0002:000006f8       _cleanUp_navPluginDlgBase$initializer$ 100056f8     moc_navPlugindlg.obj
 0002:000006fc       _cleanUp_navPluginDlg$initializer$ 100056fc     moc_navPlugindlgimpl.obj
 0002:00000708       _pcinit                    10005708     MSVCRT:crtdll.obj
 0002:0000070c       _pinit                     1000570c     MSVCRT:atonexit.obj
 0002:000012bc       ?slot_0@?3??staticMetaObject@navPlugin@@SAPAVQMetaObject@@XZ@4UQUMethod@@B 100062bc     moc_navPlugin.obj
 0002:000012d4       ?slot_1@?3??staticMetaObject@navPlugin@@SAPAVQMetaObject@@XZ@4UQUMethod@@B 100062d4     moc_navPlugin.obj
 0002:000012e0       ?slot_2@?3??staticMetaObject@navPlugin@@SAPAVQMetaObject@@XZ@4UQUMethod@@B 100062e0     moc_navPlugin.obj
 0002:000012f4       ?slot_3@?3??staticMetaObject@navPlugin@@SAPAVQMetaObject@@XZ@4UQUMethod@@B 100062f4     moc_navPlugin.obj
 0002:0000130c       ?slot_tbl@?3??staticMetaObject@navPlugin@@SAPAVQMetaObject@@XZ@4QBUQMetaData@@B 1000630c     moc_navPlugin.obj
 0002:000013b0       ?signal_0@?3??staticMetaObject@navPlugin@@SAPAVQMetaObject@@XZ@4UQUMethod@@B 100063b0     moc_navPlugin.obj
 0002:000013c4       ?signal_tbl@?3??staticMetaObject@navPlugin@@SAPAVQMetaObject@@XZ@4QBUQMetaData@@B 100063c4     moc_navPlugin.obj
 0002:00001400       ?slot_0@?3??staticMetaObject@navPluginDlgBase@@SAPAVQMetaObject@@XZ@4UQUMethod@@B 10006400     moc_navPlugindlg.obj
 0002:0000141c       ?slot_tbl@?3??staticMetaObject@navPluginDlgBase@@SAPAVQMetaObject@@XZ@4QBUQMetaData@@B 1000641c     moc_navPlugindlg.obj
 0002:0000144c       ?signal_0@?3??staticMetaObject@navPluginDlg@@SAPAVQMetaObject@@XZ@4UQUMethod@@B 1000644c     moc_navPlugindlgimpl.obj
 0002:00001458       ?signal_tbl@?3??staticMetaObject@navPluginDlg@@SAPAVQMetaObject@@XZ@4QBUQMetaData@@B 10006458     moc_navPlugindlgimpl.obj
 0002:00001c6c       _GS_ExceptionPointers      10006c6c     MSVCRT:gs_report.obj
 0002:00002678       __unwindtable$??0navEntry@@QAE@ABVQString@@0ABVQPixmap@@@Z 10007678     config.obj
 0002:00002690       __ehfuncinfo$??0navEntry@@QAE@ABVQString@@0ABVQPixmap@@@Z 10007690     config.obj
 0002:000026b4       __unwindtable$??1navEntry@@QAE@XZ 100076b4     config.obj
 0002:000026c4       __ehfuncinfo$??1navEntry@@QAE@XZ 100076c4     config.obj
 0002:000026e8       __unwindtable$??0config@@QAE@ABVQString@@@Z 100076e8     config.obj
 0002:000026f8       __ehfuncinfo$??0config@@QAE@ABVQString@@@Z 100076f8     config.obj
 0002:0000271c       __unwindtable$??1config@@UAE@XZ 1000771c     config.obj
 0002:00002724       __ehfuncinfo$??1config@@UAE@XZ 10007724     config.obj
 0002:00002748       __ehfuncinfo$?getKeys@config@@QAE?AVQStringList@@XZ 10007748     config.obj
 0002:0000276c       __unwindtable$?getKeys@config@@QAE?AVQStringList@@XZ 1000776c     config.obj
 0002:000027cc       __ehfuncinfo$?getNavEntry@config@@QAE?AV?$QPtrList@VnavEntry@@@@ABVQString@@AAV3@@Z 100077cc     config.obj
 0002:000027f0       __unwindtable$?getNavEntry@config@@QAE?AV?$QPtrList@VnavEntry@@@@ABVQString@@AAV3@@Z 100077f0     config.obj
 0002:00002908       __unwindtable$??1?$QDict@V?$QPtrList@VnavEntry@@@@@@UAE@XZ 10007908     config.obj
 0002:00002910       __ehfuncinfo$??1?$QDict@V?$QPtrList@VnavEntry@@@@@@UAE@XZ 10007910     config.obj
 0002:00002934       __unwindtable$??1?$QPtrList@VnavEntry@@@@UAE@XZ 10007934     config.obj
 0002:00002934       __unwindtable$??1?$QPtrList@VQPopupMenu@@@@UAE@XZ 10007934     config.obj
 0002:0000293c       __ehfuncinfo$??1?$QPtrList@VnavEntry@@@@UAE@XZ 1000793c     config.obj
 0002:0000293c       __ehfuncinfo$??1?$QPtrList@VQPopupMenu@@@@UAE@XZ 1000793c     config.obj
 0002:00002960       __unwindtable$??0navIconViewItem@@QAE@PAVQIconView@@ABVQString@@1@Z 10007960     navIconViewItem.obj
 0002:00002960       __unwindtable$??0navIconViewItem@@QAE@PAVQIconView@@ABVQString@@1ABVQPixmap@@@Z 10007960     navIconViewItem.obj
 0002:00002970       __ehfuncinfo$??0navIconViewItem@@QAE@PAVQIconView@@ABVQString@@1@Z 10007970     navIconViewItem.obj
 0002:00002970       __ehfuncinfo$??0navIconViewItem@@QAE@PAVQIconView@@ABVQString@@1ABVQPixmap@@@Z 10007970     navIconViewItem.obj
 0002:00002994       __unwindtable$??1navIconViewItem@@UAE@XZ 10007994     navIconViewItem.obj
 0002:0000299c       __ehfuncinfo$??1navIconViewItem@@UAE@XZ 1000799c     navIconViewItem.obj
 0002:000029c0       __unwindtable$??1QDockWindowList@@UAE@XZ 100079c0     navPlugin.obj
 0002:000029d0       __ehfuncinfo$??1QDockWindowList@@UAE@XZ 100079d0     navPlugin.obj
 0002:000029f4       __unwindtable$??1QPopupMenuList@@UAE@XZ 100079f4     navPlugin.obj
 0002:000029fc       __ehfuncinfo$??1QPopupMenuList@@UAE@XZ 100079fc     navPlugin.obj
 0002:00002a20       __unwindtable$??0config_plugin_base@@QAE@ABVQString@@00@Z 10007a20     navPlugin.obj
 0002:00002a40       __ehfuncinfo$??0config_plugin_base@@QAE@ABVQString@@00@Z 10007a40     navPlugin.obj
 0002:00002a64       __unwindtable$??1config_plugin_base@@UAE@XZ 10007a64     navPlugin.obj
 0002:00002a7c       __ehfuncinfo$??1config_plugin_base@@UAE@XZ 10007a7c     navPlugin.obj
 0002:00002aa0       __unwindtable$?about@config_plugin_base@@UAE?AVQString@@XZ 10007aa0     navPlugin.obj
 0002:00002ab0       __ehfuncinfo$?about@config_plugin_base@@UAE?AVQString@@XZ 10007ab0     navPlugin.obj
 0002:00002ad4       __ehfuncinfo$??0navPlugin@@QAE@ABVQString@@00@Z 10007ad4     navPlugin.obj
 0002:00002af8       __unwindtable$??0navPlugin@@QAE@ABVQString@@00@Z 10007af8     navPlugin.obj
 0002:00002b40       __ehfuncinfo$?reply@navPlugin@@UAEXPAVresponse@@@Z 10007b40     navPlugin.obj
 0002:00002b64       __unwindtable$?reply@navPlugin@@UAEXPAVresponse@@@Z 10007b64     navPlugin.obj
 0002:00002bac       __unwindtable$?navigate@navPlugin@@UAEXABVQString@@0@Z 10007bac     navPlugin.obj
 0002:00002bc4       __ehfuncinfo$?navigate@navPlugin@@UAEXABVQString@@0@Z 10007bc4     navPlugin.obj
 0002:00002be8       __ehfuncinfo$?about@navPlugin@@UAE?AVQString@@XZ 10007be8     navPlugin.obj
 0002:00002c0c       __unwindtable$?about@navPlugin@@UAE?AVQString@@XZ 10007c0c     navPlugin.obj
 0002:00002c34       __unwindtable$?iconClicked@navPlugin@@QAEXPAVQIconViewItem@@@Z 10007c34     navPlugin.obj
 0002:00002c3c       __ehfuncinfo$?iconClicked@navPlugin@@QAEXPAVQIconViewItem@@@Z 10007c3c     navPlugin.obj
 0002:00002c60       __unwindtable$?onItem@navPlugin@@QAEXPAVQIconViewItem@@@Z 10007c60     navPlugin.obj
 0002:00002c68       __ehfuncinfo$?onItem@navPlugin@@QAEXPAVQIconViewItem@@@Z 10007c68     navPlugin.obj
 0002:00002c8c       __unwindtable$?keys@plugindesc@@UAE?AVQStringList@@ABVQString@@0@Z 10007c8c     plugindesc.obj
 0002:00002c9c       __ehfuncinfo$?keys@plugindesc@@UAE?AVQStringList@@ABVQString@@0@Z 10007c9c     plugindesc.obj
 0002:00002cc0       __unwindtable$?create@plugindesc@@UAEPAVconfig_plugin_base@@ABVQString@@00@Z 10007cc0     plugindesc.obj
 0002:00002cc8       __ehfuncinfo$?create@plugindesc@@UAEPAVconfig_plugin_base@@ABVQString@@00@Z 10007cc8     plugindesc.obj
 0002:00002cec       __unwindtable$?qt_emit@navPluginDlg@@UAE_NHPAUQUObject@@@Z 10007cec     moc_navPlugin.obj
 0002:00002cec       __unwindtable$?qt_emit@navPlugin@@UAE_NHPAUQUObject@@@Z 10007cec     moc_navPlugin.obj
 0002:00002cf4       __ehfuncinfo$?qt_emit@navPluginDlg@@UAE_NHPAUQUObject@@@Z 10007cf4     moc_navPlugin.obj
 0002:00002cf4       __ehfuncinfo$?qt_emit@navPlugin@@UAE_NHPAUQUObject@@@Z 10007cf4     moc_navPlugin.obj
 0002:00002d18       __unwindtable$?command@navPluginDlg@@IAEXVQString@@0@Z 10007d18     moc_navPlugin.obj
 0002:00002d18       __unwindtable$?command@navPlugin@@IAEXVQString@@0@Z 10007d18     moc_navPlugin.obj
 0002:00002d30       __ehfuncinfo$?command@navPlugin@@IAEXVQString@@0@Z 10007d30     moc_navPlugin.obj
 0002:00002d30       __ehfuncinfo$?command@navPluginDlg@@IAEXVQString@@0@Z 10007d30     moc_navPlugin.obj
 0002:00002d54       __unwindtable$??0navPluginDlgBase@@QAE@PAVQWidget@@PBDI@Z 10007d54     navPlugindlg.obj
 0002:00002d74       __ehfuncinfo$??0navPluginDlgBase@@QAE@PAVQWidget@@PBDI@Z 10007d74     navPlugindlg.obj
 0002:00002d98       __unwindtable$?db@@YAXABVQString@@@Z 10007d98     navPlugindlg.obj
 0002:00002d98       __unwindtable$?languageChange@navPluginDlgBase@@MAEXXZ 10007d98     navPlugindlg.obj
 0002:00002da0       __ehfuncinfo$?languageChange@navPluginDlgBase@@MAEXXZ 10007da0     navPlugindlg.obj
 0002:00002da0       __ehfuncinfo$?db@@YAXABVQString@@@Z 10007da0     navPlugindlg.obj
 0002:00002dc8       __sehtable$??_L@YGXPAXIHP6EX0@Z1@Z 10007dc8     MSVCRT:ehvecctr.obj
 0002:00002de8       __sehtable$??_M@YGXPAXIHP6EX0@Z@Z 10007de8     MSVCRT:ehvecdtr.obj
 0002:00002e08       __sehtable$?__ArrayUnwind@@YGXPAXIHP6EX0@Z@Z 10007e08     MSVCRT:ehvecdtr.obj
 0002:00002e28       __sehtable$__onexit        10007e28     MSVCRT:atonexit.obj
 0002:00002e48       __sehtable$___DllMainCRTStartup 10007e48     MSVCRT:crtdll.obj
 0002:00002e70       __sehtable$__IsNonwritableInCurrentImage 10007e70     MSVCRT:pesect.obj
 0002:00002e90       .edata                     10007e90     navPlugin.exp
 0002:00002eb8       rgpv                       10007eb8     navPlugin.exp
 0002:00002ebc       rgszName                   10007ebc     navPlugin.exp
 0002:00002ec0       rgwOrd                     10007ec0     navPlugin.exp
 0002:00002ec2       szName                     10007ec2     navPlugin.exp
 0002:00002ed0       $N00001                    10007ed0     navPlugin.exp
 0002:000079d6       .idata$6                   1000c9d6     qt-mt323:qt-mt323.dll
 0002:00007a26       .idata$6                   1000ca26     MSVCRT:MSVCR120.dll
 0002:00007c3a       .idata$6                   1000cc3a     kernel32:KERNEL32.dll
 0003:00000000       _navPlugin_XPM             1000d000     plugindesc.obj
 0003:00000048       ?param_slot_0@?3??staticMetaObject@navPlugin@@SAPAVQMetaObject@@XZ@4QBUQUParameter@@B 1000d048     moc_navPlugin.obj
 0003:00000078       ?param_slot_1@?3??staticMetaObject@navPlugin@@SAPAVQMetaObject@@XZ@4QBUQUParameter@@B 1000d078     moc_navPlugin.obj
 0003:00000088       ?param_slot_2@?3??staticMetaObject@navPlugin@@SAPAVQMetaObject@@XZ@4QBUQUParameter@@B 1000d088     moc_navPlugin.obj
 0003:0000043c       _cleanUp_navPlugin         1000d43c     moc_navPlugin.obj
 0003:00000440       ?$S1@?3??staticMetaObject@navPlugin@@SAPAVQMetaObject@@XZ@4IA 1000d440     moc_navPlugin.obj
 0003:00000444       ?param_signal_0@?3??staticMetaObject@navPlugin@@SAPAVQMetaObject@@XZ@4QBUQUParameter@@B 1000d444     moc_navPlugin.obj
 0003:00000468       _cleanUp_navPluginDlgBase  1000d468     moc_navPlugindlg.obj
 0003:00000470       _cleanUp_navPluginDlg      1000d470     moc_navPlugindlgimpl.obj
 0003:00000474       ?param_signal_0@?3??staticMetaObject@navPluginDlg@@SAPAVQMetaObject@@XZ@4QBUQUParameter@@B 1000d474     moc_navPlugindlgimpl.obj
 0003:00000494       ?$S1@?3??staticMetaObject@navPluginDlg@@SAPAVQMetaObject@@XZ@4IA 1000d494     moc_navPlugindlgimpl.obj
 0003:00000498       ___proc_attached           1000d498     MSVCRT:crtdll.obj
 0003:000004a0       _GS_ExceptionRecord        1000d4a0     MSVCRT:gs_report.obj
 0003:000004f0       _GS_ContextRecord          1000d4f0     MSVCRT:gs_report.obj
 0003:000007bc       _DebuggerWasPresent        1000d7bc     MSVCRT:gs_report.obj
 0004:000000a0       $R000000                   1000e0a0     Script1.res
 0004:00000528       $R000488                   1000e528     Script1.res
